:100000000C946B0A0C948C0A0C948C0A0C94E40FDC
:100010000C941E100C948C0A0C948C0A0C948C0A70
:100020000C948C0A0C948C0A0C948C0A0C948C0AF8
:100030000C948C0A0C948C0A0C948C0A0C941A1351
:100040000C948C0A0C948C0A0C948C0A0C948C0AD8
:100050000C948C0A0C94696F0C948C0A0C948C0A86
:100060000C948C0A0C94E46F0C948C0A0C948C0AFB
:100070000C948C0A0C948C0A0C948C0A0C948C0AA8
:100080000C94D6840C948C0A0C948C0A0C948C0AD4
:100090000C9413700C948C0A0C948C0A0C948C0A9B
:1000A0000C948C0A0C948C0A0C948C0A0C948C0A78
:1000B0000C948C0A0C948C0A0C948C0A0C948C0A68
:1000C0000C948C0A0C948C0A0C948C0A0C948C0A58
:1000D0000C948C0A0C948C0A0C948C0A0C948C0A48
:1000E0000C948C0A0C94AF760C94A5760C94B9768B
:1000F0000C9443760C94C3760C949B760C948F7678
:100100000C9483760C948C0A0C948C0A0C948C0AB4
:100110000C948C0A0C948C0A0C948C0A0C948C0A07
:100120000C948C0A0C948C0A0C948C0A0C948C0AF7
:100130000C948C0AFB8A1A8B898B7A8C9A8CBA8CD9
:10014000C28C6F8C084AD73B3BCE016E84BCBFFD8E
:10015000C12F3D6C74319ABD56833DDA3D00C77F97
:1001600011BED9E4BB4C3E916BAAAABE0000008030
:100170003F07634236B79BD8A71A39685618AEBAFC
:10018000AB558C1D3CB7CC5763BD6DEDFD753EF690
:10019000177231BF000000803F08000000BE9224AB
:1001A00049123EABAAAA2ABECDCCCC4C3E000000E0
:1001B00080BEABAAAAAA3E00000000BF00000080DB
:1001C0003F0000000000084178D3BB4387D1133DB6
:1001D000190E3CC3BD4282AD2B3E68EC8276BED97F
:1001E0008FE1A93E4C80EFFFBE01C4FF7F3F0000BE
:1001F000000000000C94FC7C0C946E390C94C571CA
:100200000C943D840C94CC7F0C947E830C944D74A0
:100210000C947A8C0C947B7F0C9401930C94F87062
:100220000C94227D0C94228E0C94D37C0C948A7DA9
:100230000C949A8C0C94C28C0C94756E0C94CA75A8
:100240000C9422840C94FB150C94E7730C94898B0A
:100250000C94A41D0C9474700C943E730C944D4F2C
:100260000C9406500C941F600C946F7F0C94E37FE9
:100270000C94AF7D0C94796E0C94E07F0C941A8BE7
:100280000C94CC700C943E8F0C949B810C94A8849D
:100290000C944C780C94720E0C94D17F0C94B18415
:1002A0000C94BA710C94E9100C946D8D0C943F77FA
:1002B0000C9464500C946F8C0C94F67D0C94FB8A17
:1002C0000C940D150C9483720C94D67F0C94397E8B
:1002D0000C9486830C94DB7F0C947D6E0C94806E62
:1002E0000C945F7D0C948C720C9483830C94580E48
:1002F0000C94A0740C94BA8C6E616E00696E6600EA
:1003000000407A10F35A00A0724E18090010A5D4CC
:10031000E80000E87648170000E40B54020000CA29
:100320009A3B000000E1F50500008096980000006F
:1003300040420F000000A0860100000010270000CE
:100340000000E803000000006400000000000A0054
:10035000000000000100000000002C76D888DC6757
:100360004F0823DFC1DFAE59E1B1B796E5E3E453AF
:10037000C63AE651997696E8E6C28426EB898C9BCC
:1003800062ED407C6FFCEFBC9C9F40F2BAA56FA56C
:10039000F490055A2AF75C936B6CF9676DC11BFCEE
:1003A000E0E40D47FEF520E6B500D0ED902E030009
:1003B000943577050080841E080000204E0A000056
:1003C00000C80C333333330F986E12831141EF8D15
:1003D0002114893BE65516CFFEE6DB18D1844B3855
:1003E0001BF77C1D901DA4BBE424203284725E2286
:1003F0008100C9F124ECA1E53D274E414E494E490B
:100400005459494E46CDCCCC3D0AD7233C17B7D1E1
:100410003877CC2B329595E6241FB14F0A00002087
:10042000410000C84200401C4620BCBE4CCA1B0E06
:100430005AAEC59D74256300496E76616C6964206F
:1004400069326320737065656420696E204545508C
:10045000524F4D2E2053657474696E6720313020E1
:100460006B6269742F730025730A00776474206EC1
:100470006F7420656E61626C65640A005854414C6B
:100480005F5452494D3D25640025730A0025730AC7
:10049000005465737420362025730A005465737404
:1004A00020352025730A0054657374203420257389
:1004B0000A005465737420332025730A0054657351
:1004C0007420322025730A0054657374203120256E
:1004D000730A006368616E3D25640A007478707762
:1004E000723D25640A003530306B0A003235306BBE
:1004F0000A003131356B0A0035366B0A0033386B30
:100500000A0025730A00765F6C6F773D252D332E28
:1005100032660A0025730A0073656E743D252D75D9
:10052000206475703D252D752069676E6F72656456
:100530003D252D752074746C5F7A65726F3D252D95
:10054000750A0025372E33662025372E33660025A1
:10055000352E326620004572726F72203020566F41
:100560006C74004E6F7420737570706F7274656474
:100570000A004572726F72203020566F6C7400450D
:1005800072726F72203020566F6C740062756C6BE3
:100590005F64656C61793D252D750062756C6B3DFE
:1005A000252D750056616C7565206E6F7420616C29
:1005B0006C6F7765640062756C6B3A206D61783D95
:1005C00025752073746172743D25752C20656E64E9
:1005D0003D25752C20696E5F7573653D25750A0094
:1005E0007062323D25730A007062313D25730A0046
:1005F000256C7500416C6C6F776564207370656560
:100600006420312F31302F3130302F343030206B97
:100610006269742F730025630074746C3D252D642A
:10062000200074746C3D252D6420004E6577207485
:10063000746C3D252D6420002563004D5335363103
:100640003120503D252D372E326620252D372E3274
:10065000666D0A00424D5030383520256C642043C9
:100660002000424D5030383520256C6420506120E8
:1006700020252D372E32666D00256300545F4845D6
:1006800041545F4944583D252D352E326620005493
:100690005F4445573D252D352E3266200041483DAB
:1006A000252D352E32662000545F53485432583D74
:1006B000252D352E3266200052485F53485432585B
:1006C0003D252D352E32662000545F52483D252DA4
:1006D000342E3166200052483D252D342E316620BF
:1006E0000025630025630025630025630025630062
:1006F0007265706F72745F616C6C3D007265706FD3
:1007000072743D006175746F0025630025630025D8
:100710006300256300204F534343414C3D25642033
:100720000020467573653A2065653D253032782096
:1007300068663D25303278206C663D253032782061
:100740006C623D25303278004D43553D2530366C86
:10075000780025630074785F6C656E3D252D6C759F
:100760002C765F6C6F773D252D6C752C7368743219
:10077000783D252D6C752C62756C6B3D252D6C7547
:10078000002563004F4B0A002563002563002563A5
:1007900000256300256300256300256300256300B1
:1007A00064656275675F616C6C3D00646562756766
:1007B0003D0064656275673D0025730A00646565E8
:1007C000700A006E6F6E650A00707772733D007775
:1007D00064743D25730A007062323D25730A00700F
:1007E00062313D25730A00696E74725F7365635FE1
:1007F00070313D252D372E33660A00696E74725FA5
:1008000070313D252D6C640A00696E74725F7365EA
:10081000635F70303D252D372E33660A00696E7494
:10082000725F70303D252D6C640A00765F6D6375D4
:100830003D252D352E32660A00745F6D63753D25AA
:100840002D352E32660A00707077723D25730A00CE
:1008500064656275673D0072636D643D25730A00CF
:1008600025730A006175746F0A006C6F675F6D6FA6
:1008700064653D007573625F7077723D25730A0091
:1008800072656C61793D25730A0074746C3D252D89
:10089000640A0052494D455F616464723D252D64D0
:1008A0002E252D640A006E65696768626F725F7439
:1008B00061626C655F73697A653D25640A00765FE5
:1008C0006C6F773D252D332E32660A007478707771
:1008D0003D25640A006368616E3D25640A00696411
:1008E0003D006932635F6275733D006932635F7317
:1008F000706565643D252D6C750A007478743D251E
:10090000730A0053797374656D2053756D6D617250
:10091000790A002530366C780041744D6567613284
:100920003536524652320041744D65676131323876
:10093000524652320041744D656761363452465218
:10094000320041744D6567613132385246413100A1
:100950004D43553D006D61736B3D002C00696E7415
:10096000657276616C3D252D750023252D642C0064
:10097000626F6F745F636175736500705F626D6550
:100980003238300072685F626D6532383000745FF3
:10099000626D65323830007062320070623100740E
:1009A0005F686561745F69647800745F646577008F
:1009B000616800705F6D73353631310072685F7346
:1009C0006874327800745F73687432780070610004
:1009D00070006164340061643300616432006164FA
:1009E0003100613300613200613100765F696E0071
:1009F00072680065727200757074696D650070319F
:100A00005F6C73740070315F740070310070305F20
:100A10006C73740070305F7400703000765F6D63CB
:100A20007500745F6D637500743100740069640053
:100A300065363400747874002D002B006E6F6E657F
:100A40000062756C6B00706F7765725F73617665BD
:100A50005F6C656472790072656C61795F6C656466
:100A60007900636F6D7061737300616363656C001F
:100A70007072657300705F707772006165730070EB
:100A8000315F6C6564790070305F6C65647200651D
:100A900076656E74006C6564006F7700706B74002F
:100AA00074785F6C6564790072785F6C656472005D
:100AB0006F706572006E6F6E65002530327800765B
:100AC0005F6164343D252D382E3666002000765F48
:100AD0006164333D252D382E3666002000765F6137
:100AE00064323D252D382E3666002000765F616425
:100AF000313D252D382E3666002000765F6C696703
:100B000068743D252D382E3666002000765F6132F0
:100B10003D252D372E3366002000765F61313D255F
:100B20002D372E3366002000765F696E3D252D350A
:100B30002E326600204E657665722D7573656420D1
:100B4000737461636B203E20256420627974657341
:100B50000A00757074696D653D252D642D64617999
:100B6000732D253032643A253032643A25303264B0
:100B70002D686F7572730A0074657374205B6F66FD
:100B8000667C317C327C337C347C355D20202020B7
:100B9000202020202D2074657374206D6F64657390
:100BA0000A0D007478205B706B74207061796C6F33
:100BB00061645D2020202020202020202020202D66
:100BC0002073656E6420726164696F20706B74209D
:100BD0006B6579626F6172640A0D00776474205BE3
:100BE0006F6E7C6F66667C746573745D2020202058
:100BF000202020202020202D207761746368646FDE
:100C0000670A0D00765F6C6F77205B765F6C6F779D
:100C10005D20202020202020202020202020202097
:100C20002D206C6F77657374207265706F727420FD
:100C3000766F6C746167650A0D00757067722020AD
:100C400020202020202020202020202020202020A4
:100C50002020202020202D207265626F6F74207666
:100C6000696120626F6F746C6F616465720A0D0058
:100C700075617274205B33386B7C35366B7C313137
:100C8000356B7C3235306B7C3530306B5D202D2000
:100C9000736574207465726D2F7561727420737042
:100CA0006565640A0D00626F6F742020202020208B
:100CB0002020202020202020202020202020202034
:100CC00020202D207265626F6F740A0D007077729C
:100CD00073205B646565707C6E6F6E655D2020209F
:100CE0002020202020202020202D206D63752073BF
:100CF0006C656570206D6F64650A0D0072657374B4
:100D000020656570726F6D2020202020202020201B
:100D100020202020202020202D20726573746F72E7
:100D20006520656570726F6D0A0D007070777220B6
:100D30005B6F6E7C6F66665D202020202020202067
:100D4000202020202020202D2070726F6772616D7E
:100D50006D61626C65207077720A0D0070623220DE
:100D6000205B6F6E7C6F66665D2020202020202037
:100D700020202020202020202D2070726F6772619B
:100D80006D6D61626C652070696E2062320A0D00C3
:100D900070623120205B6F6E7C6F66665D20202064
:100DA0002020202020202020202020202D2062759F
:100DB0006C6B204750494F2070696E0A0D007478A3
:100DC00074205B737472696E675D20202020202080
:100DD000202020202020202020202D20536574203A
:100DE0007265706F727420746578742073747269A0
:100DF0006E670A0D0074787077205B31352D305D99
:100E000020202020202020202020202020202020E2
:100E1000202D205458205077722E2048696768652D
:100E20007374203020283364426D290A0D007474D5
:100E30006C205B302D31355D2020202020202020AB
:100E4000202020202020202020202D2074696D6566
:100E50002D746F2D6C69766520666F7220706163EA
:100E60006B6574730A0D00737320202020202020EE
:100E70002020202020202020202020202020202072
:100E80002020202D2073797374656D2073756D6D2E
:100E90006172790A0D00727320202020202020200A
:100EA0002020202020202020202020202020202042
:100EB00020202D20726164696F2073746174730A3D
:100EC0000D007269205B236E5D205B696E745D208E
:100ED00020202020202020202020202020202D2005
:100EE0007265706F727420696E74657276616C0AD7
:100EF0000D0072636D64205B6F6E7C6F66665D20B3
:100F000020202020202020202020202020202D20D4
:100F1000616C6C6F7720636D642066726F6D206EFC
:100F200065746F726B0A0D007265205B236E5D2025
:100F30005B2B7C2D5D205B6D61736B7C6175746FC9
:100F40002C6D61736B5D202D206D6F746520726553
:100F5000706F7274207365742F6D6F646966790A9F
:100F60000D006F772020202020202020202020200E
:100F700020202020202020202020202020202D2064
:100F80006F6E652D776972652073656E736F72730E
:100F90000A0D006C6F67205B6175746F7C6F6E7CEF
:100FA0006F66665D20202020202020202020202D1C
:100FB000206D6F7465732064617461206F6E2055BD
:100FC00053420A0D006E65205B666C7573685D2088
:100FD0002020202020202020202020202020202011
:100FE000202D206E65696768626F72207461626C83
:100FF000650A0D006572722020202020202020200C
:1010000020202020202020202020202020202020E0
:101010002D206572726F722073746174730A0D00F3
:101020006D637520202020202020202020202020DB
:101030002020202020202020202020202D206D6313
:101040007520696E666F0A0D00693263205B7072ED
:101050006F62657C737065656420236E5D2020205F
:1010600020202020202D206932632070726F62655D
:10107000206275737C73657420627573207370656C
:1010800065640A0D006964205B72657365745D2098
:101090002020202020202020202020202020202050
:1010A000202D2069642068616E646C696E670A0D8A
:1010B0000068756D20202020202020202020202066
:1010C000202020202020202020202020202D2068CB
:1010D000756D69646974792073656E736F720A0D3A
:1010E0000072656C6179205B6F6E7C6F66667C73E5
:1010F000746174735D20202020202020202D207218
:10110000656C6179206E6574776F726B20726570A3
:101110006F7274730A0D006465205B6D61736B5DA3
:1011200020202020202020202020202020202020BF
:101130002020202D2064656275670A0D00636861B8
:101140006E205B31312D32365D2020202020202082
:101150002020202020202020202D206368616E2068
:1011600031312D32362028322E3430352D3234387C
:1011700030204D687A290A0D0063616C69205B5B41
:10118000765F696E7C61317C61325D20766F6C7454
:101190007C72657365747C6E6F6E655D202D206357
:1011A000616C6962726174650A0D0062756C6B2016
:1011B0005B5B73686F777C666C7573685D205B73CF
:1011C00065742074687273682064656C61795D5D14
:1011D00020202D2062756C6B696E67207061636BD7
:1011E000657473200A0D0061646320202020202094
:1011F00020202020202020202020202020202020EF
:101200002020202D2073686F7720765F696E2C2058
:1012100061312C20613220766F6C74616765730ACE
:101220000D0075202020202020202020202020209C
:1012300020202020202020202020202020202D20A1
:10124000757074696D650A0D0076202020202020BD
:10125000202020202020202020202020202020208E
:1012600020202020202D2076657273696F6E0A0D74
:101270000068202020202020202020202020202046
:10128000202020202020202020202020202D206809
:10129000656C700A0D00256300756E6B6E6F776E5E
:1012A00020636D640A00484D433538383300257398
:1012B000002573000A00202573002025362E326693
:1012C0002000253032780074656D705F6578746534
:1012D000726E3D252D362E326600202573002025A6
:1012E000362E3266204F6E2D426F617264002530BB
:1012F00032780074656D705F626F6172643D252D98
:10130000362E32660042756C6B2072656D3A207322
:10131000746172743D25752C20656E643D25752CB5
:1013200020696E5F7573653D25750A0042756C6BAB
:10133000206164643A2073746172743D25752C20B9
:10134000656E643D25752C20696E5F7573653D255E
:10135000750A0042756C6B207468726573683A2078
:1013600074696D65723D25750A00503A20256C64DC
:101370002050612020252D372E3266206D0A005224
:101380004553455454494E4720454550524F4D21F1
:10139000004932433A20004F6E6C696E650A005274
:1013A0006F7574696E6720456E61626C65640A00D2
:1013B00052504C20456E61626C65640A00257320B2
:1013C00025732C206368616E6E656C202575202C5A
:1013D00020636865636B2072617465202575204801
:1013E0007A20747820706F7765722025750A000A5C
:1013F0002A2A2A2A2A2A2A426F6F74696E672025B0
:10140000732A2A2A2A2A2A2A0A00726E67206973F6
:10141000737565732025640A00454550524F4D2071
:10142000697320636F72727570742C2072657772A5
:101430006974696E67207769746820646566617590
:101440006C74732E0A006C6F63616C686F73740048
:1014500041544D45474132353672667232000200C2
:1014600000FFFE000001452025642E256420636CEA
:101470006F636B20256C752063707520256C75205B
:101480006C706D20256C752069727120256C75203B
:10149000676C656420256C7520796C656420256C0B
:1014A0007520726C656420256C7520747820256C1D
:1014B00075206C697374656E20256C752073656E7C
:1014C000736F727320256C752073657269616C206F
:1014D000256C750A000011241FBECFEFD1E8DEBFD6
:1014E000CDBF00E00CBF1BE0A0E0B2E0E2EFFFE305
:1014F00001E00BBF02C007900D92A037B107D9F7EA
:101500002BE3A0E7BBE001C01D92A336B207E1F7D1
:101510000E94D36D0C94F79F0C9400002F923F9281
:101520004F925F926F927F928F929F92AF92BF92F3
:10153000CF92DF92EF92FF920F931F93CF93DF939F
:10154000CDB7DEB760970FB6F894DEBF0FBECDBF44
:101550007C011B016A01FC0117821682838181FFD5
:1015600044C39E012F5F3F4F3901F7019381F10181
:1015700093FD859193FF81911F01882309F431C365
:10158000853239F493FD859193FF81911F01853256
:1015900039F4B70190E00E94D39C56016501E5CF74
:1015A00010E0512C912CFFE1F915D8F08B3279F035
:1015B00038F4803279F08332A1F4F92DF0612EC035
:1015C0008D3261F0803369F4292D21602DC0392DD1
:1015D0003260932E892D8460982E2AC0E92DE86010
:1015E00015C097FC2DC020ED280F2A3088F496FEF8
:1015F00006C03AE0139F200D1124122F19C08AE073
:10160000589E200D1124522EE92DE0629E2E10C00E
:101610008E3231F496FCE5C2F92DF0649F2E08C09D
:101620008C3621F4292D2068922E02C0883641F490
:10163000F10193FD859193FF81911F018111B3CF3A
:101640009BEB980F933020F4992D9061805E07C03A
:101650009BE9980F933008F066C1992D9F7E96FF05
:1016600016E09F73992E853619F49064992E08C060
:10167000863621F4392F3068932E02C01111115093
:1016800097FE07C01C3350F444244394410E27E0D6
:101690000BC0183038F027E017E005C027E09CE3C6
:1016A000492E02C0212F412C560184E0A80EB11C06
:1016B000F6016081718182819381042DA3010E94D2
:1016C0004A9B6C01F981FC87F0FF02C0F3FF06C062
:1016D00091FC06C092FE06C000E205C00DE203C008
:1016E0000BE201C000E08C858C7019F001115AC228
:1016F0009BC297FE10C04C0CFC85F4FF04C08A818D
:10170000813309F44A94141474F528E0241578F50B
:1017100088E0482E2CC096FC2AC0812F90E08C15C2
:101720009D059CF03CEFC3163FEFD30674F0892D66
:101730008068982E0AC0E2E0F0E0EC0FFD1FE10F98
:10174000F11D8081803319F411501111F4CF97FEEF
:101750000EC044244394410E812F90E0C816D90650
:101760002CF41C1904C04424439401C010E097FEDB
:1017700006C01C141D0434F4C601019605C085E0A2
:1017800090E002C081E090E001110196112331F058
:10179000212F30E02F5F3F4F820F931F252D30E028
:1017A0008217930714F4581A01C0512C892D89709F
:1017B00049F4552039F0B70180E290E00E94D39CB3
:1017C0005A94F7CF002329F0B701802F90E00E94B0
:1017D000D39C93FC09C0552039F0B70180E390E019
:1017E0000E94D39C5A94F7CF97FE4CC04601D7FE77
:1017F00002C0812C912CC60188199909F301E80FC8
:10180000F91FFE87ED87960124193109388B2F8740
:10181000012F10E01195019511093FEF83169306F2
:1018200029F4B7018EE290E00E94D39CC814D90439
:101830004CF08F8598898815990524F4ED85FE85EF
:10184000818101C080E3F1E08F1A91082D853E85EA
:101850002F5F3F4F3E872D87801691062CF0B701F2
:1018600090E00E94D39CD9CFC814D90441F49A8146
:10187000963320F4953319F43C8534FF81E3B701A6
:1018800090E04EC08A81813319F09C859F7E9C87B1
:10189000B70190E00E94D39C111105C094FC18C0C0
:1018A00085E690E017C0B7018EE290E00E94D39CDD
:1018B0001E5F82E001E0080FF301E80FF11D808157
:1018C000B70190E00E94D39C802F0113F3CFE6CFA5
:1018D00085E490E0B7010E94D39CD7FC06C0C114F8
:1018E000D10441F4EC85E4FF05C0D194C194D10842
:1018F0008DE201C08BE2B70190E00E94D39C80E3AF
:101900002AE0C216D1042CF08F5FFAE0CF1AD1087A
:10191000F7CFB70190E00E94D39CB701C601C096F3
:101920000E94D39C54C1833631F0833779F08335DC
:1019300009F056C020C0560132E0A30EB11CF601DA
:101940008081898301E010E0630112C05601F2E05A
:10195000AF0EB11CF601C080D18096FE03C0612F8E
:1019600070E002C06FEF7FEFC6010E947F9C8C0188
:10197000F92DFF7714C0560122E0A20EB11CF6012A
:10198000C080D18096FE03C0612F70E002C06FEF6F
:101990007FEFC6010E94349C8C01F92DF0689F2EC8
:1019A000F3FD1AC0852D90E008171907A8F4B701B8
:1019B00080E290E00E94D39C5A94F4CFF60197FC09
:1019C000859197FE81916F01B70190E00E94D39CB1
:1019D00051105A94015011090115110579F7F7C0FA
:1019E000843611F0893661F5560197FE09C024E06E
:1019F000A20EB11CF60160817181828193810AC0BF
:101A0000F2E0AF0EB11CF60160817181072E000C6F
:101A1000880B990BF92DFF769F2E97FF09C09095A3
:101A20008095709561957F4F8F4F9F4FF0689F2EE7
:101A30002AE030E0A3010E94E79DC82EC6183FC0EF
:101A4000092D853721F40F7E2AE030E01DC0097F83
:101A50008F3691F018F4883559F0C3C0803719F0EB
:101A6000883711F0BEC0006104FF09C0046007C0E0
:101A700094FE08C0066006C028E030E005C020E102
:101A800030E002C020E132E0560107FF09C084E0E7
:101A9000A80EB11CF601608171818281938108C01A
:101AA000F2E0AF0EB11CF6016081718180E090E040
:101AB000A3010E94E79DC82EC6180F77902E96FEB0
:101AC0000BC0092D0E7FC11650F494FE0AC092FC83
:101AD00008C0092D0E7E05C0DC2C092D03C0DC2CAE
:101AE00001C0D12E04FF0DC0FE01EC0DF11D80815F
:101AF000803311F4097E09C002FF06C0D394D39449
:101B000004C0802F867809F0D39403FD11C000FF34
:101B100006C01C2DD51480F4150D1D190DC0D5144B
:101B200058F4B70180E290E00E94D39CD394F7CFA1
:101B3000D51410F45D1801C0512C04FF10C0B7017A
:101B400080E390E00E94D39C02FF17C001FD03C018
:101B500088E790E002C088E590E0B7010CC0802FD4
:101B6000867859F001FF02C08BE201C080E207FDD8
:101B70008DE2B70190E00E94D39CC11638F4B70102
:101B800080E390E00E94D39C1150F7CFCA94F301F8
:101B9000EC0DF11D8081B70190E00E94D39CC11033
:101BA000F5CF15C0F4E0F51560F584E0581A93FE02
:101BB0001FC0011127C02C8523FF2AC008EF12E0A7
:101BC000392D3071932EF8018491811124C0552054
:101BD00009F4E4CCB70180E290E00E94D39C5A94CF
:101BE000F6CFF7018681978126C08FEF9FEF23C044
:101BF000B70180E290E00E94D39C5A945110F8CF34
:101C0000D8CF512CB701802F90E00E94D39CD3CF26
:101C10000CEF12E0D5CF91108052B70190E00E94F6
:101C2000D39C0F5F1F4FCFCF23E0251510F483E027
:101C3000BDCF512CC0CF60960FB6F894DEBF0FBE5B
:101C4000CDBFDF91CF911F910F91FF90EF90DF906B
:101C5000CF90BF90AF909F908F907F906F905F904C
:101C60004F903F902F9008958115910511F00197A5
:101C7000F1F7089589EC97E09F938F930E94239D3D
:101C80008091660290916702A0916802B09169020A
:101C90000F900F9093FF03C083EC97E002C08DEB91
:101CA00097E09F938F930E94239D0F900F9008952C
:101CB000E091491EEF73F0E0E656F14E808380918B
:101CC000491E8F5F8093491E8091F636886080930D
:101CD000F6364CE452E061E1CA010E943E7A80E0AF
:101CE00090E00895CF93DF93EC018091C914909117
:101CF000CA14A091CB14B091CC1486FF1DC08E8164
:101D00001F928F938D811F928F938C811F928F933F
:101D10008B811F928F938A811F928F9387EF92E01E
:101D20009F938F930E940F9D8DB79EB70C960FB611
:101D3000F8949EBF0FBE8DBFBE018BEB9BE00E944F
:101D4000357BBE0188E092E0DF91CF910C94907CCE
:101D500052985A981DBAE9E6F0E08081806280834B
:101D6000EA9A53985B98EB9A808180688083E8E6D2
:101D7000F0E08081816080830895EFEFFEE11182C1
:101D8000128210820895CF92DF92EF92FF920F930A
:101D90001F93CF93DF93EC019B018091FF1E843151
:101DA00008F0BBC08091011F64E10E94EC91909308
:101DB000011FC0901C32D0901D32E0901E32F09076
:101DC0001F32092F10E08DE8989FD0011124A150F7
:101DD000B14E1396CD92DD92ED92FC92169741157D
:101DE000510559F0FA018081FD01EA57FF4F8083C8
:101DF000FA018181A957BF4F8C932097A9F089815F
:101E00009DE8909FF001919FF00D1124E150F14E5B
:101E1000DF01A657BF4F8C93E557FF4F88818F7026
:101E2000808388818F70808321153105E1F1D9018C
:101E300016964C9116975DE8509FC001519F900DEA
:101E400011248150914EFC01E757FF4F40831596B6
:101E50004C9115973197408334961B964D915D9127
:101E60006D917C911E97452F562F672F77275183B1
:101E700040837C01BEE8EB0EF11CF901238534851B
:101E800045855685A4E6B0E00E948792672F782F9B
:101E9000892F992724E630E040E050E00E9420920C
:101EA000D7016D937C938DE8809FD001819FB00D09
:101EB0001124AA5FB04EFE0132968FE701900D9279
:101EC0008A95E1F78091011F8F5F8093011F9091A8
:101ED000FF1E9F5F9093FF1E4091C9145091CA143A
:101EE0006091CB147091CC1460FF2DC01F929F9312
:101EF0001F928F938091001F1F928F938CE293E12A
:101F00009F938F930E94239DEDB7FEB738960FB62F
:101F1000F894FEBF0FBEEDBF16C080912C32909199
:101F20002D32A0912E32B0912F320196A11DB11DFC
:101F300080932C3290932D32A0932E32B0932F3277
:101F400080E090E002C081E090E0DF91CF911F91AE
:101F50000F91FF90EF90DF90CF9008952091FF1E9A
:101F6000222361F18091001F8F5F21502093FF1E7B
:101F700064E10E94EC919093001F4091C91450912C
:101F8000CA146091CB147091CC1460FF1AC01F92D8
:101F90002F938091011F1F928F931F929F9385E033
:101FA00093E19F938F930E94239D8DB79EB70896D0
:101FB0000FB6F8949EBF0FBE8DBF03C080E090E0C7
:101FC000089581E090E008951F920F920FB60F924E
:101FD00011248F939F93AF93BF938091680080FFEC
:101FE00024C08091C5369091C636A091C736B09175
:101FF000C8360196A11DB11D8093C5369093C63693
:10200000A093C736B093C8368091C9149091CA1472
:10201000A091CB14B091CC1487FF07C0749882E0D4
:1020200090E09093920280939102BF91AF919F9123
:102030008F910F900FBE0F901F9018951F920F92C7
:102040000FB60F9211248F939F93AF93BF938091FC
:10205000680080FF24C08091C9369091CA36A09153
:10206000CB36B091CC360196A11DB11D8093C936F7
:102070009093CA36A093CB36B093CC368091C914D6
:102080009091CA14A091CB14B091CC1490FF07C0CA
:10209000739882E090E09093920280939102BF91B6
:1020A000AF919F918F910F900FBE0F901F90189539
:1020B00080937C0080917B00877F80937B00809160
:1020C0007C00806C80937C0085E080937A00809116
:1020D0007A00806880937A0080917B0087FFFCCF34
:1020E00080917B0085FFFCCF80917A008064809393
:1020F0007A0080917A0086FDFCCF109279001092D0
:10210000780084E090E060E070E020917A00206444
:1021100020937A0020917A0026FDFCCF2091780050
:1021200030917900620F731F019779F710927C004C
:1021300080917A008F7780937A007695679576956F
:10214000679580E090E00E94CA95089580E00E9423
:1021500058102091890230918A0240918B0250914F
:102160008C020E94C49721EE3AE744E95EE30E94A4
:10217000359408950F931F93CF93DF930FE110E0F1
:10218000CBE5DEE00093510182E991E00E94340E3C
:102190008091510185FD0DC00031110521F02CF019
:1021A000CB54D10903C0C4ECD9E0E2970150110926
:1021B000E9CFBE0180E090E00E94CA9520E030E0C7
:1021C0004AE754E40E941895DF91CF911F910F9137
:1021D0000895CF93DF93EC0188819981009799F05E
:1021E0008F3C924121F01982188283E011C0623144
:1021F00071F40E94BA106093183270931932809370
:102200001A3290931B328FEC92E19983888381E09C
:10221000DF91CF91089580917B00886080937B004F
:1022200089EC80937C0085E080937A0080917A002D
:10223000806880937A0080917B0087FFFCCF80913B
:102240007B0085FFFCCF80917A00806480937A00C8
:1022500080917A0086FDFCCF80917A008064809323
:102260007A0080917A0086FDFCCF609178007091B1
:10227000790080917A008F7780937A0080E090E0F7
:102280000E94CA9527ED33EA40E95FE30E94C497B4
:1022900026E636E648E853E40E9434940895AF9267
:1022A000BF92CF92DF92EF92FF921F93CF93DF9373
:1022B000CDB7DEB729970FB6F894DEBF0FBECDBFFE
:1022C0005C011092C3148FEF898782E5E82E8EE1BE
:1022D000F82E10E06E0189E0C80ED11C8985882394
:1022E000D1F11830D1F1BE016F5F7F4FC6010E945E
:1022F000DD6389858F3F11F08E3F19F48093C314FD
:102300002AC0CE010196A114B10479F40E94F663AB
:102310008093E736FE013196AFEDB6E381918D9360
:10232000EC15FD05D9F781E019C00E94F663F701AD
:102330008087FE01319680E090E02191D701A80FBF
:10234000B91F2C93019688309105B9F71F5FF9E00A
:10235000EF0EF11CC3CF812F01C088E029960FB684
:10236000F894DEBF0FBECDBFDF91CF911F91FF90DC
:10237000EF90DF90CF90BF90AF9008952F923F9253
:102380004F925F926F927F928F929F92AF92BF9285
:10239000CF92DF92EF92FF920F931F93CF93DF9331
:1023A000EC015B01009711F427E003C0019749F4A9
:1023B00026E04AE250E06BE270E089E290E00E94A1
:1023C000BD62CE010E944F119E012C533B4E69010C
:1023D000F9018083CD2B69F0C2E5DEE1E12CF12C1F
:1023E00096EB292E92E1392E24EB822E22E1922EB9
:1023F000C2C08FED96E30E948364BC01990F880BE5
:10240000990B0E94CC956B017C01AB2801F120E077
:1024100030E048EC52E40E9418959F938F937F938D
:102420006F9383EF92E19F938F930E94239D84EBA0
:1024300092E19F938F930E94239D2DB73EB7285F13
:102440003F4F0FB6F8943EBF0FBE2DBFCBC0CFEDB0
:10245000D6E387EEA82E86E3B82E0EEE12E1899120
:102460001F928F931F930F930E94239D0F900F90A5
:102470000F900F90AC16BD0691F720E030E048ECCD
:1024800052E4C701B6010E9418959F938F937F93E2
:102490006F938EED92E19F938F930E94239D0F90F7
:1024A0000F900F900F900F900F908091E736811151
:1024B00003C088EA93E002C086E293E09F938F9383
:1024C0008AED92E19F938F930E94239D84EB92E18A
:1024D0009F938F930E94239D0F900F900F900F90CA
:1024E0000F900F907FC000E010E0FE01E00FF11FA1
:1024F00080811F928F93E2ECF2E1FF93EF930E94B1
:10250000239D0F5F1F4F0F900F900F900F9008307B
:10251000110559F720E030E048EC52E4C301B20164
:102520000E9418959F938F937F936F938AEB92E10C
:102530009F938F930E94239D0F900F900F900F9069
:102540000F900F90888581114AC088EA93E09F938D
:102550008F933F922F920E94239D9F928F920E9471
:10256000239DFFEFEF1AFF0A29960F900F900F900F
:102570000F900F900F90F601808190E0E816F90619
:102580008CF5CE010E948364BC01990F880B990BD6
:102590000E94CC952B013C01A114B10409F4A3CFF6
:1025A00020E030E048EC52E40E9418959F938F930E
:1025B0007F936F9387EC92E19F938F930E94239D6B
:1025C00084EB92E19F938F930E94239D8DB79EB7DA
:1025D00008960FB6F8949EBF0FBE8DBF03C086E26B
:1025E00093E0B5CFDF91CF911F910F91FF90EF90C6
:1025F000DF90CF90BF90AF909F908F907F906F9023
:102600005F904F903F902F900895CF93DF931F924C
:102610001F92CDB7DEB7EFEDF6E381818983878125
:102620008A83CE0101960E9482810F900F90DF91E4
:10263000CF9108951F920F920FB60F9211240BB6EF
:102640000F92FF920F931F932F933F934F935F939C
:102650006F937F938F939F93AF93BF93CF93DF93AA
:10266000EF93FF938091F63682608093F6368091E7
:10267000660286FD2B9A8091660287FD2B9A8091D7
:102680009102909192021816190614F4749A739A92
:102690008091C9149091CA14A091CB14B091CC141C
:1026A00085FF02C07498739880910602909107028A
:1026B00001979093070280930602892B09F073C15A
:1026C00080917E0B90917F0B019690937F0B80936E
:1026D0007E0B80911C3290911D32A0911E32B091E0
:1026E0001F320196A11DB11D80931C3290931D32A3
:1026F000A0931E32B0931F3280E190E090930702C6
:10270000809306028091660280FD02C01D9B05C079
:102710001092C8141092C71406C081E090E0909304
:10272000C8148093C7148091C9149091CA14A091C1
:10273000CB14B091CC1497FF08C08091C71490912E
:10274000C814892B49F0749A739809EF1DE1C1E30D
:10275000D2E3FF24F39441C0739A7498F6CF80912A
:102760007E0B90917F0B0196BF010E94F891892BFF
:10277000E1F5D80112964C91417020E030E050E034
:1027800060E070E080E090E0A0E00E94289469F1B1
:1027900077988091C9149091CA14A091CB14B091EC
:1027A000CC1492FF05C0749810929202109291027C
:1027B000F8016085718561157105C1F4D80118961D
:1027C0006D917C9119976115710511F5065F1F4F89
:1027D0002596B2E3C534DB0779F1D8011896ED915F
:1027E000FC911997309721F3BACFBF0180917E0BEE
:1027F00090917F0B01960E94F891892BF9F61C822B
:102800001B82AE0162E184E292E00E943E7AD6CF62
:1028100080917E0B90917F0B0E94F891892BB1F6ED
:10282000F8821A8309831C821B82AE0162E182E472
:1028300092E00E943E7ACACF60916C0270916D0264
:1028400061157105A1F180917E0B90917F0B0E9423
:10285000F891892B61F58091C5369091C636A0918B
:10286000C736B091C83640910E2A50910F2A609118
:10287000102A7091112A841B950BA60BB70B80931D
:10288000211E9093221EA093231EB093241E80919C
:10289000C5369091C636A091C736B091C8368093A0
:1028A0000E2A90930F2AA093102AB093112A6091B8
:1028B0006A0270916B0261157105A1F180917E0B26
:1028C00090917F0B0E94F891892B61F58091C93618
:1028D0009091CA36A091CB36B091CC364091122A55
:1028E0005091132A6091142A7091152A841B950B1C
:1028F000A60BB70B8093251E9093261EA093271E30
:10290000B093281E8091C9369091CA36A091CB36DB
:10291000B091CC368093122A9093132AA093142A54
:10292000B093152AE091980AF091990A80E090E01E
:102930001995892BD9F481E08093313289EF9DE19B
:102940009093333280933232109235321092343277
:10295000749882E090E0909392028093910241E318
:1029600052E362E182E492E00E943E7A8091660244
:1029700086FD2B988091660290916702A091680273
:10298000B091690291FF0FC00E947C738A3119F0E7
:10299000C1E0C80F01C0CBE00E94BA718C2F0E9429
:1029A0008D730E94837240E050E060E089EB92E01A
:1029B0000E943E7AFF91EF91DF91CF91BF91AF914D
:1029C0009F918F917F916F915F914F913F912F9147
:1029D0001F910F91FF900F900BBE0F900FBE0F90A5
:1029E0001F9018958091491E90913032891B08954F
:1029F0000E94F214882371F0E0913032EF73F0E01E
:102A0000E656F14E808190E0209130322F5F209386
:102A1000303208958FEF9FEF0895CF93DF93EC014D
:102A20001092AF0B1092AE0B888199810097C1F084
:102A30008B30944021F01982188283E0B8C0613154
:102A400009F0B4C00E94F81499279093AA0B8093C0
:102A5000A90B8D30910509F444C08F3F910549F4CD
:102A60000E94F2148111EECF8BE094E09983888369
:102A70009DC08231910509F45AC08F37910509F044
:102A800052C08091A70B9091A80B181619060CF54F
:102A900060915D3B70915E3B88E090E00E94D39C2A
:102AA00060915D3B70915E3B80E290E00E94D39C20
:102AB00060915D3B70915E3B88E090E00E94D39C0A
:102AC0008091A70B9091A80B01979093A80B8093EE
:102AD000A70B8091A70B9091A80B8F37910509F058
:102AE000BFCF109230321092491E8091A70B909167
:102AF000A80BFC01EB5BFD4C10829093AF0B809315
:102B0000AE0B1092A80B1092A70B8091E836909113
:102B1000E936009709F4A4CF40E050E06091C11479
:102B20000E943E7A9DCF8830910571F5AACF6091C1
:102B30005D3B70915E3B8DE090E00E94D39C1092D3
:102B4000A60B1092A50B8091A50B9091A60B20913E
:102B5000A70B3091A80B821793070CF0BACFFC019A
:102B6000EB5BFD4C808160915D3B70915E3B90E042
:102B70000E94D39C8091A50B9091A60B01969093F7
:102B8000A60B8093A50BDFCF60915D3B70915E3B00
:102B90000E94D39C8091A70B9091A80B2091A90B28
:102BA000FC01EB5BFD4C208301968FCF81E0DF9130
:102BB000CF9108958091C7149091C814892BD1F0BA
:102BC0008091660290916702A0916802B0916902BB
:102BD00093FD10C00E94BA7183B7817F866083BF66
:102BE000F89483B7816083BF7894889583B78E7F8C
:102BF00083BF78940895CF93DF93FC0120813181C6
:102C00002115310551F02630334129F0FC011182A4
:102C1000108283E015C0653891F4EC010E94BA700F
:102C20000E94DA1540E050E065E8809133169091FB
:102C300034160E943E7A86E093E19983888381E08E
:102C4000DF91CF910895CF93DF93EB01892B61F052
:102C50005F934F9381EB92E19F938F930E94239D0B
:102C60000F900F900F900F90DF93CF938EEA92E129
:102C70009F938F930E94239D0F900F900F900F9022
:102C8000DF91CF910895CF93DF93D62FC42F0E9469
:102C900046658D2F0E9477658C2F0E947765DF91A6
:102CA000CF910C946F65CF92DF92EF92FF920F93CA
:102CB0001F93CF93DF93C82FD62FF42E152F022FFB
:102CC0000E9446658D2F0E9477658C2F81600E943F
:102CD0006D65CF2DD12F10E0E12CF12C680181E042
:102CE000C81AD108E016F10671F0CE14DF0419F409
:102CF0000E94926502C00E94886588838FEFE81A5F
:102D0000F80A2196EFCFDF91CF911F910F91FF909D
:102D1000EF90DF90CF900C946F65CF93DF931F926D
:102D20001F92CDB7DEB728E030E04AE95EE168E9FE
:102D300070E080EB90E00E945316EAE9FEE18781A3
:102D4000898386818A83CE0101960E9482810F90B9
:102D50000F90DF91CF910895CF93DF93EC012091F5
:102D6000DF363091E0364091E1365091E2366091A5
:102D7000E3367091E4368091E5369091E636AFEF18
:102D80000E94289429F527E04AE250E06BE270E0C7
:102D900089E290E00E94BD6280E090E00E944F11C5
:102DA000FE01EC53FB4E8083CD2B71F4882361F040
:102DB00049E050E06EE070E08FED96E30E94DA9F0C
:102DC000DF91CF910C940513DF91CF910C948D1668
:102DD000DF91CF910895CF92DF92EF92FF920F9300
:102DE0001F93CF93DF931F92CDB7DEB70E94BA70C7
:102DF00080EB0E94126581111CC00E946F6580915A
:102E0000162E9091172E81609093172E8093162E78
:102E10008FE293E09F938F938EEA92E19F938F933B
:102E20000E94239D0F900F900F900F9001E010E0F3
:102E300002C000E010E08EB18470F82E729A64E255
:102E400078E680E090E00E94EF640E94BA708EE421
:102E50000E941265811117C00E946F658091162E25
:102E60009091172E82609093172E8093162E6801F2
:102E70008FEFC81AD80A47EE59E067E373E0C8013C
:102E80000E9423168601F11001C0729864E278E670
:102E900080E090E00E94EF640E94BA708EEE0E9483
:102EA0001265811159C019820E946F6521E030E0DE
:102EB000AE014F5F5F4F60ED70E08EEE90E00E94DC
:102EC000531689818535A9F48091162E9091172E7D
:102ED00084609093172E8093162E78018FEFE81A56
:102EE000F80A47EE59E06FE373E0C8010E94231629
:102EF000870189818835A9F48091162E9091172E2B
:102F000080619093172E8093162E78018FEFE81A28
:102F1000F80A47EE59E066E473E0C8010E94231600
:102F2000870189818036C1F48091162E9091172EE9
:102F300080629093172E8093162E78018FEFE81AF7
:102F4000F80A47EE59E06DE473E0C8010E942316C9
:102F500081E00E947C68870164E278E680E090E08E
:102F60000E94EF640E94BA7086EA0E941265811185
:102F700017C00E946F658091162E9091172E806465
:102F80009093172E8093162E78018FEFE81AF80A87
:102F900047EE59E064E573E0C8010E9423168701FB
:102FA00064E278E680E090E00E94EF640E94BA70EC
:102FB0008CE30E94126581111FC00E946F65809191
:102FC000162E9091172E80689093172E8093162EB0
:102FD00078018FEFE81AF80A47EE59E06CE573E0E4
:102FE000C8010E94231686EA92E19F938F930E9464
:102FF000239D0F900F90870164E278E680E090E0D7
:103000000E94EF640E94BA7082ED0E9412658111E5
:1030100017C00E946F658091162E9091172E9160B7
:103020009093172E8093162E78018FEFE81AF80AE6
:1030300047EE59E064E673E0C8010E942316870159
:1030400064E278E680E090E00E94EF640E94BA704B
:1030500080E80E941265811117C00E946F658091FF
:10306000162E9091172E98609093172E8093162EFF
:1030700078018FEFE81AF80A47EE59E06DE673E041
:10308000C8010E942316870164E278E680E090E0A0
:103090000E94EF640E94BA7080ED0E941265811157
:1030A00017C00E946F658091162E9091172E946024
:1030B0009093172E8093162E78018FEFE81AF80A56
:1030C00047EE59E063E773E0C8010E9423168701C9
:1030D00064E278E680E090E00E94EF640E94BA70BB
:1030E0008CEE0E941265811117C00E946F6580915D
:1030F000162E9091172E90619093172E8093162E76
:1031000078018FEFE81AF80A47EE59E06BE773E0B1
:10311000C8010E942316870187E0E82EF12C64E2A3
:1031200078E680E090E00E94EF640E94BA708CE73D
:103130000E941265811113C00E946F658091162E46
:103140009091172E92609093172E8093162E47EE33
:1031500059E062E873E0C8010E94231604C081E0D0
:10316000E81AF108E1F60E946F6584EB92E19F9303
:103170008F930E94239D0F900F900F90DF91CF911E
:103180001F910F91FF90EF90DF90CF900895AF9235
:10319000BF92CF92DF92EF92FF920F931F93CF9344
:1031A000DF93CDB7DEB760970FB6F894DEBF0FBEE2
:1031B000CDBFF82EE42E6623E9F18E010F5F1F4F7D
:1031C00080E1F80111928A95E9F728E0A80168E901
:1031D00080EB0E945316FF2041F08BE893E09F9311
:1031E0008F930E940F9D0F900F905E01F8E0AF0E3D
:1031F000B11C92E9C92E93E0D92EF80181918F017B
:103200001F928F93DF92CF920E940F9D0F900F908D
:103210000F900F900A151B0581F788851F928F93D9
:1032200087EE93E09F938F930E940F9D0F900F90D6
:103230000F900F90EE20E9F18E010F5F1F4F80E19C
:10324000F80111928A95E9F720E1A80160E880EB86
:103250000E945316FF2041F087E993E09F938F93DC
:103260000E940F9D0F900F906E01F0E1CF0ED11CC8
:1032700082E9E82E83E0F82EF80181918F011F92F8
:103280008F93FF92EF920E940F9D0F900F900F90DF
:103290000F90C016D10681F788891F928F9387EE11
:1032A00093E09F938F930E940F9D0F900F900F902C
:1032B0000F9060960FB6F894DEBF0FBECDBFDF91C2
:1032C000CF911F910F91FF90EF90DF90CF90BF9023
:1032D000AF9008950F931F93CF93DF931F921F9288
:1032E000CDB7DEB71A82198222E0AE014F5F5F4F81
:1032F0006AEA8EEE0E9453160AED1EE189819A81D8
:10330000982789279827F8019183808322E0AE01CE
:103310004F5F5F4F6CEA8EEE0E94531689819A814F
:10332000982789279827F8019383828322E0AE01AA
:103330004F5F5F4F6EEA8EEE0E94531689819A812D
:10334000982789279827F8019583848322E0AE0186
:103350004F5F5F4F60EB8EEE0E94531689819A811A
:10336000982789279827F801938B828B22E0AE015A
:103370004F5F5F4F62EB8EEE0E94531689819A81F8
:10338000982789279827F801958B848B22E0AE0136
:103390004F5F5F4F64EB8EEE0E94531689819A81D6
:1033A000982789279827F801978B868B22E0AE0112
:1033B0004F5F5F4F66EB8EEE0E94531689819A81B4
:1033C000982789279827F8019783868322E0AE0102
:1033D0004F5F5F4F68EB8EEE0E94531689819A8192
:1033E000982789279827F8019187808722E0AE01E6
:1033F0004F5F5F4F6AEB8EEE0E94531689819A8170
:10340000982789279827F8019587848722E0AE01BD
:103410004F5F5F4F6CEB8EEE0E94531689819A814D
:10342000982789279827F8019787868722E0AE0199
:103430004F5F5F4F6EEB8EEE0E94531689819A812B
:10344000982789279827F801918B808B0F900F90F0
:10345000DF91CF911F910F9108952F923F924F923C
:103460005F926F927F928F929F92AF92BF92CF9214
:10347000DF92EF92FF920F931F93CF93DF93CDB71D
:10348000DEB769970FB6F894DEBF0FBECDBF182F19
:10349000D62E042F2F8B9E012F5F3F4F790183E0A3
:1034A000F90111928A95E9F78091FE1E811105C0FC
:1034B0000E946A1981E08093FE1EDD2009F46DC030
:1034C0004EE264EF8EEE0E94431662E174E380E008
:1034D00090E00E94EF6422E0A70166EF8EEE0E946A
:1034E000531629813A81322723273227A90160E028
:1034F00070E08091F01E9091F11E9A01AB01281BA3
:10350000390B41095109A091EE1EB091EF1E0E94A6
:1035100087926B017C013FE0F594E794D794C794C0
:103520003A95D1F76091E81E7091E91ECB01770FB3
:10353000AA0BBB0BBC01CD014BE0660F771F881FA8
:10354000991F4A95D1F72091EA1E3091EB1E49014F
:10355000330FAA08BB08A50194012C0D3D1D4E1D7B
:103560005F1D0E944292C20ED31ED092E51EC092F1
:10357000E41EF8E0CF0ED11C54E0D594C7945A95C0
:10358000E1F70D2C000CEE08FF08C092F21ED0925D
:10359000F31EE092F41EF092F51E812F8295880FA3
:1035A000880F807C8C5C8A87212F30E039872887C0
:1035B000A3E0B0E0012E02C0AA0FBB1F0A94E2F7FD
:1035C0002AE63AE00E9480929B01AC012E5F3F4FB9
:1035D0004F4F5F4F2B873C874D875E8780E593EC8D
:1035E000A0E0B0E09C01AD0104C05595479537952A
:1035F00027951A95D2F72B8B3C8B4D8B5E8B10E069
:10360000412C512C320188E090E0AC01E885F9852D
:103610004E1B5F0B598F488F101709F439C14A852B
:1036200064EF8EEE0E9443166B857C858D859E85AA
:103630000E94EF6423E0AE014F5F5F4F66EF8EEEB6
:103640000E9453162090E41E3090E51EF0EA2F1AD7
:10365000FFE03F0A9101D1010E9469926C837D8352
:103660008E839F83E091DC1EF091DD1EF88BEF8747
:10367000E091DA1EF091DB1EFA8BE98BE091DE1E01
:10368000F091DF1EA091E01EB091E11E9B01AC0104
:103690008CE055954795379527958A95D1F70E94E7
:1036A00092926C01FF24D7FCF094EF2C9101DF0182
:1036B0000E946992DC01CB013DE0B595A7959795F5
:1036C00087953A95D1F78C0D9D1DAE1DBF1D0296B5
:1036D000A11DB11D42E0B595A795979587954A958F
:1036E000D1F79C01AD0130584F4F5F4FA091EC1EB8
:1036F000B091ED1E0E9487924B015C015FE0B69491
:10370000A794979487945A95D1F78981CA80D12C30
:10371000E12CF12CFE2CED2CDC2CCC24E82A8B8126
:10372000C82A088C04C0F594E794D794C7940A94E7
:10373000D2F7A091E21EB091E31E2C813D814E8113
:103740005F810E9492929B01AC0177E1559547956C
:10375000379527957A95D1F72C833D834E835F83E8
:103760009101AF85B8890E946992DC01CB01EBE041
:10377000B595A79597958795EA95D1F72C813D81C9
:103780004E815F81820F931FA41FB51FE989FA89BB
:10379000AF01FF0F660B770BF2E0440F551F661F5A
:1037A000771FFA95D1F7840F951FA61FB71F0884BE
:1037B00004C0880F991FAA1FBB1F0A94D2F7029654
:1037C000A11DB11D22E0B595A795979587952A95DE
:1037D000D1F7A7019601281B390B4A0B5B0B6B89AC
:1037E0007C898D899E890E94DC9197FD0BC0660FB4
:1037F000771F881F991FA50194010E9420924901FB
:103800005A010AC0A50194010E94209249015A015F
:10381000880C991CAA1CBB1C9927B7FC9A958B2D68
:103820007A2D692D9B01AC010E94DC919B01AC01BA
:10383000AEEDBBE00E9487926B017C01A3E4B3EE86
:10384000A50194010E949592BB2797FDB095AB2FDF
:103850006701FF24D7FCF094EF2CC80ED91EEA1E96
:10386000FB1EFFECCF0EFEE0DF1EE11CF11C44E06E
:10387000F594E794D794C7944A95D1F78C0C9D1C86
:10388000AE1CBF1C480C591C6A1C7B1C1F5FC4CE9D
:10389000112381F0212F30E040E050E0C301B2015C
:1038A0000E9420922093F61E3093F71E4093F81E3C
:1038B0005093F91E2F89222389F16091F61E709191
:1038C000F71E8091F81E9091F91E61157105810512
:1038D000910521F10E94CC9520E836EE45EC57E4A5
:1038E0000E94189521E03EED42E45EE30E9431988B
:1038F0009B01AC0160E070E080E89FE30E9434949B
:103900002BE43AE34DEB57E30E9418956093FA1EBF
:103910007093FB1E8093FC1E9093FD1E69960FB65C
:10392000F894DEBF0FBECDBFDF91CF911F910F91F5
:10393000FF90EF90DF90CF90BF90AF909F908F90CF
:103940007F906F905F904F903F902F9008950F93CE
:103950001F93CF93DF9300D000D0CDB7DEB78E0199
:103960000F5F1F4F86E0F80111928A95E9F7809169
:10397000F01D811113C040E061E386EA0E94431606
:103980004AE06CE286EA0E94431681E08093F01DD3
:1039900068EF7CE780E090E00E94EF6448E06DE231
:1039A00086EA0E94431668EF7CE780E090E00E9480
:1039B000EF6426E0A80162E386EA0E94531647E01E
:1039C0006DE286EA0E94431689819A818093EA1DFE
:1039D0009093EB1D2B813C812093EC1D3093ED1DCA
:1039E0004D815E814093EE1D5093EF1D5F934F9389
:1039F0003F932F939F938F938BE993E09F938F93A4
:103A00000E940F9D0FB6F894DEBF0FBECDBF269665
:103A10000FB6F894DEBF0FBECDBFDF91CF911F91DF
:103A20000F9108958F929F92AF92BF92CF92DF92A3
:103A3000EF92FF920F931F93CF93DF9300D000D0AC
:103A4000CDB7DEB78E010F5F1F4F86E0F8011192F0
:103A50008A95E9F741E062E08CE30E94431648E56D
:103A600060E08CE30E94431664E278E680E090E038
:103A70000E94EF6426E0A80163E08CE30E945316E5
:103A800043E062E08CE30E94431609811A8110270B
:103A900001271027EAECFDE111830083EB80FC8015
:103AA000FE24EF24FE24F382E282CD80DE80DC243B
:103AB000CD24DC24D582C482B801012E000C880BF1
:103AC000990B0E94CC954B015C01B7010F2C000CA7
:103AD000880B990B0E94CC95A50194010E94B49487
:103AE00020EE3EE245E652E40E94C49720E030E03A
:103AF00044E353E40E9435949F938F937F936F9395
:103B0000DF92CF92FF92EF921F930F9389EA93E097
:103B10009F938F930E940F9D0FB6F894DEBF0FBE48
:103B2000CDBF26960FB6F894DEBF0FBECDBFDF9196
:103B3000CF911F910F91FF90EF90DF90CF90BF90AA
:103B4000AF909F908F900895CF93DF93EC01888181
:103B500099810097A9F18B3E924121F01982188238
:103B600083E083C08CE89BE00E940F78892BA1F151
:103B70008091C9149091CA14A091CB14B091CC1427
:103B800093FD2CC08091C9149091CA14A091CB14BC
:103B9000B091CC1493FD53C08091C9149091CA1474
:103BA000A091CB14B091CC1494FD51C08091C91454
:103BB0009091CA14A091CB14B091CC1495FD4EC035
:103BC00040E850E060E070E08CE89BE00E94F17714
:103BD0008BEE92E19983888381E047C08091162E15
:103BE00082FFD0CF21E048E061E083E00E942D1AFF
:103BF0008091FD1E8F938091FC1E8F938091FB1E00
:103C00008F938091FA1E8F938091F91E8F938091EC
:103C1000F81E8F938091F71E8F938091F61E8F93DD
:103C20008AE693E19F938F930E94239D8DB79EB761
:103C30000A960FB6F8949EBF0FBE8DBFA3CF80919A
:103C4000162E85FFA9CF81E00E947269A5CF8091D1
:103C5000162E86FFABCF0E94A71CA8CF8091162EF0
:103C600087FFAECF0E94121DABCFDF91CF91089599
:103C7000CF93DF93C82F8CEE0E946D658C2F0E942E
:103C800077656AE67AE080E090E00E94EF648DEE6E
:103C90000E946D650E948865D82F0E949265C82F8A
:103CA0000E946F658C2F90E09D2BDF91CF9108953E
:103CB0001F93CF93DF93C82F8CEE0E946D658C2FDE
:103CC0000E94776564E278E680E090E00E94EF640D
:103CD0008CEE0E946D6580E00E9477656AE67AE06E
:103CE00080E090E00E94EF648DEE0E946D650E947E
:103CF0008865182F0E948865C82F0E949265D82F6A
:103D00000E946F658C2F90E0A0E0B0E0BA2FA92F41
:103D1000982F8827A12BBC01CD016D2BDF91CF916E
:103D20001F9108952F923F924F925F926F927F92D0
:103D30008F929F92AF92BF92CF92DF92EF92FF92BB
:103D40000F931F93CF93DF93CDB7DEB7CE54D10936
:103D50000FB6F894DEBF0FBECDBF809104029091E4
:103D60000502892BE1F110920502109204028CEEFB
:103D70000E946D658EE10E9477650E946F6566E323
:103D80007CE980E090E00E94EF6482EA0E94381EA5
:103D900090937D0B80937C0B84EA0E94381E909355
:103DA0007B0B80937A0B86EA0E94381E9093790BE6
:103DB0008093780B88EA0E94381E9093770B80934B
:103DC000760B8AEA0E94381E9093750B8093740BD1
:103DD0008CEA0E94381E9093730B8093720B88E4D8
:103DE0000E94581E6AAF7BAF8CAF9DAF88E50E94E2
:103DF000581E2091740B3091750B4B015C01A90189
:103E000060E070E080E090E0DC0127962FAF27971C
:103E100028965FAF289729966FAF29972A967FAF8C
:103E20002A972B968FAF2B972C969FAF2C972D967A
:103E3000AFAF2D972E96BFAF2E97AB0160E070E02D
:103E400080E090E008E00E94CA932A833983B42F6F
:103E5000A52FF62FE72F8C019401A50160E070E0FB
:103E600080E090E0AA80B980CB2EDA2EEF2EFE2ED5
:103E70000E94169429014A016DA37CA389839A8329
:103E8000315041095F4F6F4F7F4F8F4F9F4F6624D7
:103E90006394712C21153F4F4F4F514061057105BF
:103EA0008105910509F010F4612C712C13014091EA
:103EB000720B5091730B52016401EDA0FCA00981BB
:103EC0001A819A0140E050E060E070E080E090E00C
:103ED0000E949A92F22E032F142FB52FF62FE72F60
:103EE000D82EE92EA0E00E94289484F421503109B4
:103EF00040485F4F6F4F7F4F8F4F9F4FF22E032FE2
:103F0000142FB52FF62FE72FD82EE92E2F2D302F77
:103F1000412F5B2F6F2F7E2F8D2D9E2D07E10E944D
:103F2000E3932C8F3D8F4E8F5F8F68A379A38AA375
:103F30009BA32053384F4F4F5F4F6F4F7F4F8F4F93
:103F40009F4F2C8B3D8B4E8B5F8B688F798F8A8F29
:103F50009B8F2056304F4F4F5F4F6F4F7F4F8F4F8C
:103F60009F4F243D30434105510561057105810591
:103F7000910529F020F01301EFEF2E1A3E0A40912F
:103F8000760B5091770B52016401EDA0FCA00981E2
:103F90001A819A0140E050E060E070E080E090E03B
:103FA0000E949A92F22E032F142FB52FF62FE72F8F
:103FB000D82EE92EA0E00E9428945CF4AFE70E947E
:103FC0000A94F22E032F142FB52FF62FE72FD82E99
:103FD000E92E2F2D302F412F5B2F6F2F7E2F8D2D10
:103FE0009E2D07E00E94E3932B833C833A01B62F7A
:103FF000A72FF82FE92FA0907A0BB0907B0B95019B
:1040000040E050E060E070E080E090E000E10E947D
:10401000CA9359016A017B018C012B813C81A30168
:104020006B2F7A2F8F2F9E2F0E9401942B833C831E
:1040300049875A876B877C878D879E872E5F3F4F86
:10404000434051096E4F7F4F8F4F9F4F22303105B4
:10405000494F5F4F644071058105910521F018F0CB
:104060002FEF221A320A40917C0B50917D0B5E8318
:104070004D834091780B5091790B52016401EDA072
:10408000FCA009811A819A0140E050E060E070E0F4
:1040900080E090E00E949A92F22E032F142FB52F09
:1040A000F62FE72FD82EE92EA0E00E94289484F462
:1040B00021503F4F4F4F5F4F6F4F7F4F8F4F9F4F5D
:1040C000F22E032F142FB52FF62FE72FD82EE92E1F
:1040D0002F2D302F412F5B2F6F2F7E2F8D2D9E2D5B
:1040E00008E00E94E3932F8338873A01B62FA72F69
:1040F000F82FE92F6D817E81C12CD12C9B01A60167
:1041000060E070E080E090E00FE00E94CA93590107
:104110006A017B018C012F813885A3016B2F7A2FD7
:104120008F2F9E2F0E9401942D833F8348875F87A6
:10413000688B798B8A8B9B8B2F5F3F4F4140510956
:104140006F4F7F4F8F4F9F4F213030484C4F5F470D
:10415000624071058105910521F018F0BFEF2B1A1F
:104160003B0A2C893D894E895F89688D798D8A8DBE
:104170009B8D2F3C37404105510561057105810537
:10418000910511F00CF0D3C152016401EDA0FCA027
:1041900009811A819201A401B701C8010E949A9273
:1041A000122F3A834983B52FF62FE72FF82E092FC8
:1041B000A0E00E94289484F421503109410950481C
:1041C0006F4F7F4F8F4F9F4F122F3A834983B52FE9
:1041D000F62FE72FF82E092F212F3A8149815B2FE7
:1041E0006F2F7E2F8F2D902F0FE10E94E3932EAF24
:1041F0003FAF21964FAF219722965FAF229723962C
:104200006FAF239724967FAF249725968FAF25977E
:1042100026969FAF269745E0A42EB12CC12CD12C19
:10422000E12CF12C00E010E02C8D3D8D4E8D5F8D4A
:1042300068A179A18AA19BA10E949A92AC8CBD8CA5
:10424000CE8CDF8CE8A0F9A00AA11BA10E949A9253
:10425000122F3BAB4AABB52FF62FE72F7C01922EE6
:10426000A32EB42EC52ED62E072F782E8F2CA0E08D
:104270000E9428945CF4A1E00E940A94922EA32E3E
:10428000B42EC52ED62E072F782E892E292D3A2D05
:104290004B2D5C2D6D2D702F872D982D01E00E94E8
:1042A000E3932AA73BA74CA75DA76EA77FA788AB80
:1042B00099AB29833A834CA35DA36EA37FA388A700
:1042C00099A7212F3BA94AA95B2F6F2F7E2FC701EA
:1042D000A0E00E94289454F4A3E00E940A94122FB4
:1042E0003BAB4AABB52FF62FE72F7C01212F3BA923
:1042F0004AA95B2F6F2F7E2FC70102E00E94E39334
:104300002AAB3BAB4CAB5DAB6EAB7FAB88AF99AF31
:104310002F962FAF2F9727963FAF2797B42FA52F14
:10432000F62FE72F4C012C893D894E895F89688DD6
:10433000798D8A8D9B8D24323A4F4F4F5F4F6F4F4F
:104340007F4F8F4F9F4F0CF088C02C8D3D8D4E8D31
:104350005F8D68A179A18AA19BA12455324F4F4F4F
:104360005F4F6F4F7F4F8F4F9F4F29013A014B0196
:104370008D8F9C8F27E0A22EB12CC12CD12CE12C4B
:10438000F12C00E010E092010E949A925201630128
:1043900074010D8D1C8D0E949A92AAA4BBA4CCA47A
:1043A000DDA4EEA4FFA408A919A90E940194298301
:1043B0003A834CA35DA36EA37FA388A799A73BE094
:1043C000A32EB12CC12CD12CE12CF12C00E010E05B
:1043D0009201A301B4018D8D9C8D0E949A9252018D
:1043E000630174010D8D1C8D0E949A92122F3D8FD6
:1043F0004C8FB52FF62FE72FF82E092FA0E00E9443
:1044000028945CF4A1E00E940A94122F3D8F4C8FF7
:10441000B52FF62FE72FF82E092F212F3D8D4C8D2C
:104420005B2F6F2F7E2F8F2D902F01E00E94E39343
:10443000AAA8BBA8CCA8DDA8EEA8FFA808AD19AD16
:104440000E9401942F962FAF2F9727963FAF279763
:10445000B42FA52FF62FE72F4C012B813C814985E6
:104460005A856B857C858D859E85A980BA80CCA078
:10447000DDA0EEA0FFA008A519A50E9416942B832D
:104480003C8349875A876B877C878D879E872D81E0
:104490003F8148855F85688979898A899B892F96BC
:1044A000AFAC2F972796BFAC2797CB2EDA2EEF2EE7
:1044B000FE2E84010E9416942D833F8348875F87D8
:1044C000688B798B8A8B9B8B2C893D894E895F8980
:1044D000688D798D8A8D9B8DAEACBFAC2196CFACAB
:1044E00021972296DFAC22972396EFAC2397249650
:1044F000FFAC249725960FAD259726961FAD2697DE
:104500000E9416942056304F4F4F5F4F6F4F7F4F92
:104510008F4F9F4F243D3043410551056105710583
:104520008105910521F018F0BFEF2B1A3B0A4AAD27
:104530005BAD6CAD7DAD9A01AB0160E070E0CB018D
:1045400027962FAF279728963FAF289729964FAFEA
:1045500029972A965FAF2A972B966FAF2B972C96A9
:104560007FAF2C972D968FAF2D972E969FAF2E97BE
:10457000AD80BF80C884DF84E888F9880A891B89F8
:1045800060E070E080E090E00E949A92122F3A83FF
:104590004983B52FF62FE72FF82E092FA0E00E94B0
:1045A000289484F421503109404E5F4F6F4F7F4F64
:1045B0008F4F9F4F122F3A834983B52FF62FE72F46
:1045C000F82E092F212F3A8149815B2F6F2F7E2FE3
:1045D0008F2D902F05E10E94E393AB80BC80C984AE
:1045E000DA84EB84FC840D851E850E941694122FBC
:1045F0003A834983B52FF62FE72FF82E092FA0E035
:104600000E94289484F4215030484F4F5F4F6F4FE1
:104610007F4F8F4F9F4F122F3A834983B52FF62F2D
:10462000E72FF82E092F212F3A8149815B2F6F2F19
:104630007E2F8F2D902F0FE00E94E39359016A0186
:104640007B018C01722E6B2CB42FAD2DF62F5F2CBD
:104650004C01285E33404109510961097109810902
:104660009109283D304D4140510561057105810595
:10467000910509F010F4232869F09501A601B7010E
:10468000C8010E948393722E632EB42FA52FF62F9C
:10469000572E4C01272D362D4B2F5A2F6F2F752D4E
:1046A000C4010E94C49520E030E048EC52E40E942E
:1046B0001895C25BDF4F0FB6F894DEBF0FBECDBFBB
:1046C000DF91CF911F910F91FF90EF90DF90CF90EE
:1046D000BF90AF909F908F907F906F905F904F9022
:1046E0003F902F9008954F925F926F927F928F929A
:1046F0009F92AF92BF92CF92DF92EF92FF922B01E7
:104700003C0169017A0123EC35EF4CE851E4C70123
:10471000B6010E94C4974B015C0128EB3EE143E7E0
:1047200053E4C701B6010E9435949B01AC01C50159
:10473000B4010E9418950E9492954B015C0120E003
:1047400030E048EC52E4C301B2010E94189521E820
:1047500035E943EC50E40E94C497A50194010E94FE
:10476000C4974B015C0123E333E948E853E4C701F4
:10477000B6010E9435949B01AC01C501B4010E94B1
:10478000189523E333EB48E553E40E94C497FF9068
:10479000EF90DF90CF90BF90AF909F908F907F90E1
:1047A0006F905F904F9008954F925F926F927F92BB
:1047B0008F929F92AF92BF92CF92DF92EF92FF9231
:1047C00069017A010E9438974B015C0123EC35EFB7
:1047D0004CE851E4C701B6010E94C4972B013C018B
:1047E00028EB3EE143E753E4C701B6010E9435944C
:1047F0009B01AC01C301B2010E9418956B017C01C1
:1048000020E030E040E050E4C501B4010E9434945F
:1048100022E93CE54EED5EE30E9418959B01AC0158
:10482000C701B6010E9435946B017C0128EB3EE183
:1048300043E753E40E94C4974B015C01A701960132
:1048400063EC75EF8CE891E40E9434949B01AC0119
:10485000C501B4010E941895FF90EF90DF90CF90B2
:10486000BF90AF909F908F907F906F905F904F9090
:1048700008954F925F926F927F928F929F92AF9224
:10488000BF92CF92DF92EF92FF922B013C01690120
:104890007A0123EC35EF4CE851E4C701B6010E94E0
:1048A000C4974B015C0128EB3EE143E753E4C701A9
:1048B000B6010E9435949B01AC01C501B4010E9470
:1048C00018950E9492954B015C0120E030E048EC85
:1048D00052E4C301B2010E941895A50194010E94FF
:1048E000C49720E030E040E251E40E94349424EE8A
:1048F00038E34EE05FE30E94C497A70196010E944F
:104900003594FF90EF90DF90CF90BF90AF909F9045
:104910008F907F906F905F904F90089580E80E94F5
:104920006D6581110DC08EEF0E947765811108C001
:1049300066E37CE980E090E00E94EF640C946F6590
:104940000E946F658091283290912932A0912A327D
:10495000B0912B320196A11DB11D80932832909306
:104960002932A0932A32B0932B320895FC01DC0146
:10497000AC014E5F5F4F90E031E38D91982788E066
:10498000292F220F97FF03C0922F932701C0922F48
:104990008150B1F7A417B50781F721E030E082819B
:1049A000891711F020E030E0C9010895DF92EF92FD
:1049B000FF920F931F93CF93DF930E948E2480E882
:1049C0000E946D6581116DC08AEF0E94776581112B
:1049D00068C08FE00E947765811163C06AE67AE063
:1049E00080E090E00E94EF6481E80E946D65811193
:1049F00058C00E948865D82F0E9488650E948865EB
:104A0000182F0E9488650E948865082F0E9488657B
:104A10000E949265F82E80E80E946D65811141C068
:104A20008CEF0E94776581113CC089EC0E9477650C
:104A3000811137C06AE67AE080E090E00E94EF647E
:104A400081E80E946D650E948865E82E0E94886555
:104A5000D82E0E9488650E948865C82F0E949265A2
:104A60001F92DF921F92EF921F92FF921F920F935D
:104A70001F921F931F92DF931F928F931F92CF93CA
:104A80008EEB93E09F938F930E940F9D0E946F6522
:104A90008DB79EB742960FB6F8949EBF0FBE8DBFDE
:104AA00017C00E946F658091283290912932A091A1
:104AB0002A32B0912B320196A11DB11D809328326C
:104AC00090932932A0932A32B0932B320E948E24E5
:104AD00020E030E040E050E060E070E080E090E016
:104AE000DF91CF911F910F91FF90EF90DF9008958C
:104AF000EF92FF920F931F93CF93DF9300D0CDB728
:104B0000DEB78C0180E80E946D65811154C00115EB
:104B1000110551F085EE0E94776581114CC062E06D
:104B20007EE281E090E009C083EE0E94776581110A
:104B300042C062E375E783E090E00E94EF6481E8A1
:104B40000E946D65811137C00E948865E82E8983B7
:104B50000E948865F82E8A830E9492658B830E944A
:104B60006F65CE0101960E94B624892B21F16F2D2D
:104B700070E07E296C7F80E090E0012B69F00E945C
:104B8000CA9520E030E04AEF5AE30E94C49720E043
:104B900030E040EC50E40CC00E94CA9522E538EBAE
:104BA0004FE25BE30E94C49726E636E64BE352E40D
:104BB0000E9434941BC00E946F65809128329091AE
:104BC0002932A0912A32B0912B320196A11DB11D3C
:104BD0008093283290932932A0932A32B0932B32BB
:104BE0000E948E2460EF7FEF89E794E40F900F908E
:104BF0000F90DF91CF911F910F91FF90EF9008954B
:104C00000F931F93CF93DF93729A8091660283FF75
:104C100008C08EE40E941265811165C0C0E5D0E035
:104C200009C0C0E5D0E08FED97E00E94340E2197D7
:104C3000D1F7EFCF8FED97E00E94340E2197D1F797
:104C40008FE40E9412650E948865D82FDF730E944E
:104C50008865082F0E948865C82F0E949265182FCA
:104C60000E946F658091660283FF72986D2F70E0DD
:104C7000762F6627600F711D80E090E00E94CA9534
:104C800020E134E048EC5BE30E94C49760930A2A79
:104C900070930B2A80930C2A90930D2A6C2F70E04E
:104CA000762F6627610F711D7695679576956795C6
:104CB00080E090E00E94CA9524EA3CEF44E25CE385
:104CC0000E94C49720E030E040E252E40E94349415
:104CD0006093F7367093F8368093F9369093FA36EE
:104CE00080E090E002C081E090E0DF91CF911F91E1
:104CF0000F9108957298729A8EE40E94126580EA6C
:104D00000E94776580E00E94776580E00E94776569
:104D10008FE40E9412650E9488658EE40E941265ED
:104D200080E80E94776580E00E94776580E00E94BD
:104D300077650E946F6580E090E0089589E992E1CF
:104D40009F938F930E94239D809180020F900F90DC
:104D5000882361F01F928F9386E992E19F938F934E
:104D60000E94239D0F900F900F900F90089581E760
:104D700092E19F938F930E94239D89E492E19F93F8
:104D80008F930E94239D82E292E19F938F930E94D2
:104D9000239D87EE91E19F938F930E94239D8BEA41
:104DA00091E19F938F930E94239D89E791E19F93C7
:104DB0008F930E94239D8DE391E19F938F930E9497
:104DC000239D87E191E19F938F930E94239D81EE24
:104DD00090E19F938F930E94239D8091162E909136
:104DE000172E827098702DB73EB72E5E3F4F0FB6CC
:104DF000F8943EBF0FBE2DBF892B41F081EB90E1AF
:104E00009F938F930E94239D0F900F9085E890E1D0
:104E10009F938F930E94239D89E490E19F938F93AA
:104E20000E94239D80E290E19F938F930E94239D97
:104E300084EF9FE09F938F930E94239D85EC9FE0DA
:104E40009F938F930E94239D83E99FE09F938F936D
:104E50000E94239D82E69FE09F938F930E94239D53
:104E600088E29FE09F938F930E94239D82EF9EE0B4
:104E70009F938F930E94239D82EC9EE09F938F933C
:104E80000E94239D86E99EE09F938F930E94239D1D
:104E900087E69EE09F938F930E94239D8EE29EE083
:104EA0009F938F930E94239D85EF9DE09F938F9307
:104EB0000E94239D8EEB9DE09F938F930E94239DE4
:104EC00080E99DE09F938F930E94239D8DB79EB7AD
:104ED00080960FB6F8949EBF0FBE8DBF8CE59DE007
:104EE0009F938F930E94239D8BE29DE09F938F93CE
:104EF0000E94239D8CEF9CE09F938F930E94239DA3
:104F00008DEC9CE09F938F930E94239D86EA9CE00A
:104F10009F938F930E94239D80E79CE09F938F93A4
:104F20000E94239D8AE39CE09F938F930E94239D80
:104F300084E09CE09F938F930E94239D8BED9BE0E8
:104F40009F938F930E94239D83EA9BE09F938F936F
:104F50000E94239D88E79BE09F938F930E94239D4F
:104F60002DB73EB72A5E3F4F0FB6F8943EBF0FBE37
:104F70002DBF08958DEE93E00C944B9D4F925F9260
:104F80006F927F928F929F92AF92BF92CF92DF9259
:104F9000EF92FF92CF93DF93CDB7DEB728970FB68E
:104FA000F894DEBF0FBECDBF80911C3290911D32B0
:104FB000A0911E32B0911F3289839A83AB83BC8348
:104FC00040901C3250901D3260901E3270901F3203
:104FD00080911C3290911D32A0911E32B0911F32EF
:104FE0008D839E83AF83B88760911C3270911D3290
:104FF00080911E3290911F322CE3822E912CA12C95
:10500000B12CA50194010E9420927F936F9330E10F
:10501000C32E3EE0D32EE12CF12C6D817E818F8159
:105020009885A70196010E942092A50194010E94F3
:1050300020923F932F9340E8842E41E5942EAA249A
:10504000A394B12CC301B201A50194010E94209246
:10505000A70196010E9420923F932F9369817A8144
:105060008B819C81A50194010E9420923F932F93F4
:1050700082E59BE09F938F930E94239D0FB6F89447
:10508000DEBF0FBECDBF28960FB6F894DEBF0FBEB1
:10509000CDBFDF91CF91FF90EF90DF90CF90BF9089
:1050A000AF909F908F907F906F905F904F900895FA
:1050B000E3E6FBE3808191818234924479F0E35608
:1050C000FB43FF93EF9384E39BE09F938F930E94B6
:1050D000239D0F900F900F900F9008953A96E53F03
:1050E00081E8F80738F30895CF93DF93EC018C9AA9
:1050F0000E94A6109F938F937F936F9388E29BE00B
:105100009F938F930E94239D0F900F900F900F906D
:105110000F900F90209719F084EB92E102C086E285
:105120009BE09F938F930E94239D0F900F9081E0AF
:105130000E9458102091850230918602409187028A
:10514000509188020E94C4979F938F937F936F938F
:105150008AE19BE09F938F930E94239D0F900F9075
:105160000F900F900F900F90209719F084EB92E121
:1051700002C088E19BE09F938F930E94239D0F9034
:105180000F9082E00E94581020918102309182029B
:1051900040918302509184020E94C4979F938F9301
:1051A0007F936F938CE09BE09F938F930E94239D4E
:1051B0000F900F900F900F900F900F90209719F075
:1051C00084EB92E102C08AE09BE09F938F930E9460
:1051D000239D0F900F9083E00E9458109F938F9310
:1051E0007F936F938BEF9AE09F938F930E94239D01
:1051F0008C980F900F900F900F900F900F9020971A
:1052000019F084EB92E102C089EF9AE09F938F93AB
:105210000E94239D0F900F908091162E9091172E33
:1052200092FF88C021E042E161E080ED0E94D966F2
:105230009F938F937F936F938CEE9AE09F938F93BE
:105240000E94239D0F900F900F900F900F900F9042
:10525000209719F084EB92E102C08AEE9AE09F93C6
:105260008F930E94239D0F900F9021E042E162E016
:1052700080ED0E94D9669F938F937F936F938DEDFE
:105280009AE09F938F930E94239D0F900F900F9011
:105290000F900F900F90209719F084EB92E102C0CD
:1052A0008BED9AE09F938F930E94239D0F900F9018
:1052B00021E042E163E080ED0E94D9669F938F93E5
:1052C0007F936F938EEC9AE09F938F930E94239D20
:1052D0000F900F900F900F900F900F90CD2B19F013
:1052E00084EB92E102C08CEC9AE09F938F930E9432
:1052F000239D0F900F9021E042E164E080ED0E9439
:10530000D9669F938F937F936F938FEB9AE09F93D0
:105310008F930E94239D0F900F900F900F900F90EE
:105320000F9084EB92E19F938F930E94239D0F90A7
:105330000F9002C0CD2BA9F3DF91CF9108950F9369
:105340001F93CF93DF93882389F049E050E06FEFFC
:1053500070E08FED96E30E94599C49E050E06EE0CA
:1053600070E08FED96E30E94DA9F13C0CFEDD6E395
:105370000AEB1AE089911F928F931F930F930E945B
:10538000239D0F900F900F900F9086E3C73ED80794
:1053900089F784EB92E19F938F930E94239D0F9056
:1053A0000F90DF91CF911F910F910895882311F0F5
:1053B000299A089529980895882311F02A9A089522
:1053C0002A980895CF92DF92EF92FF92CF93DF93C6
:1053D0006B017C0160FF11C08AE294E09F938F9380
:1053E0008EEA92E19F938F930E94239D0F900F90DE
:1053F0000F900F9081E090E002C080E090E0C1FE4D
:1054000009C0EC01219647EE59E06FE274E00E947A
:105410002316CE01C2FE09C0EC01219647EE59E0E9
:1054200067E374E00E942316CE01C3FE09C0EC01BD
:10543000219647EE59E06FE374E00E942316CE01F7
:10544000C4FE09C0EC01219647EE59E06FEF75E00C
:105450000E942316CE01C5FE09C0EC01219647EE3D
:1054600059E063E474E00E942316CE01C6FE09C031
:10547000EC01219647EE59E067E474E00E942316A0
:10548000CE01C7FE09C0EC01219647EE59E06DE45C
:1054900074E00E942316CE01D0FE09C0EC012196D3
:1054A00047EE59E065E574E00E942316CE01D1FE77
:1054B00009C0EC01219647EE59E06DE574E00E94C9
:1054C0002316CE01D2FE09C0EC01219647EE59E029
:1054D00061E674E00E942316CE012091162E3091D1
:1054E000172E24703071232B59F0D3FE09C0EC0124
:1054F000219647EE59E067E674E00E942316CE013C
:105500002091162E26FF0BC0D4FE09C0EC01219677
:1055100047EE59E06CE674E00E942316CE0120911C
:10552000162E27FF0BC0D5FE09C0EC01219647EED1
:1055300059E062E774E00E942316CE01D6FE09C04E
:10554000EC01219647EE59E06AE774E00E942316C9
:10555000CE01D7FE09C0EC01219647EE59E065E87F
:1055600074E00E942316CE01E0FE0CC047EE59E025
:1055700066E974E0DF91CF91FF90EF90DF90CF90DC
:105580000C942316CD28CE28CF2841F485EB9AE041
:105590009F938F930E94239D0F900F90DF91CF9147
:1055A000FF90EF90DF90CF900895CF92DF92EF922F
:1055B000FF92CF93DF93EC01C12CD12C7601209781
:1055C00009F4A3C060EB7AE0CE010E942B9C892BEA
:1055D00011F46894C0F868EA7AE0CE010E942B9C2E
:1055E000892B11F46894C1F860EA7AE0CE010E9438
:1055F0002B9C892B11F46894C2F86CE97AE0CE01F7
:105600000E942B9C892B11F46894C3F869E97AE015
:10561000CE010E942B9C892B11F46894C4F865E993
:105620007AE0CE010E942B9C892B11F46894C5F876
:105630006FE87AE0CE010E942B9C892B11F46894CC
:10564000C6F867E87AE0CE010E942B9C892B11F402
:105650006894C7F86FE77AE0CE010E942B9C892BF3
:1056600011F46894D0F86BE77AE0CE010E942B9C8D
:10567000892B11F46894D1F865E77AE0CE010E9495
:105680002B9C892B11F46894D2F860E77AE0CE0164
:105690000E942B9C892B11F46894D3F86AE67AE077
:1056A000CE010E942B9C892B11F46894D4F862E6F9
:1056B0007AE0CE010E942B9C892B11F46894D5F8D6
:1056C00067E57AE0CE010E942B9C892B11F4689447
:1056D000D6F866E47AE0CE010E942B9C892B11F467
:1056E0006894D7F861E47AE0CE010E942B9C892B64
:1056F00011F46894E0F860917E0270917F0280E07E
:1057000090E00E943F9CEC015ACFC701B601DF91A7
:10571000CF91FF90EF90DF90CF900895AF92BF921E
:10572000CF92DF92EF92FF920F931F93CF93DF936D
:10573000122FD32FC42F052FF62EE72ED82EC92EC9
:10574000217030E040E050E060E070E080E090E008
:10575000A0E00E94289489F08BE994E09F938F93B6
:105760008EEA92E19F938F930E94239D0F900F905A
:105770000F900F90E1E0F0E002C0E0E0F0E08091F7
:10578000162E80FF19C0212F247030E040E050E039
:1057900060E070E080E090E0A0E00E94289461F07A
:1057A0005F018FEFA81AB80A47EE59E06FE974E07D
:1057B000CF010E942316F501212F227030E040E036
:1057C00050E060E070E080E090E0A0E00E9428946B
:1057D00061F05F018FEFA81AB80A47EE59E063EA5B
:1057E00074E0CF010E942316F501212F287030E0CC
:1057F00040E050E060E070E080E090E0A0E00E94D7
:10580000289461F05F018FEFA81AB80A47EE59E0BB
:105810006BEB74E0CF010E942316F501212F20715C
:1058200030E040E050E060E070E080E090E0A0E038
:105830000E94289461F05F018FEFA81AB80A47EE22
:1058400059E066EA74E0CF010E942316F501212F8A
:10585000207230E040E050E060E070E080E090E0F6
:10586000A0E00E94289461F05F018FEFA81AB80AA7
:1058700047EE59E069EA74E0CF010E942316F50172
:10588000212F207430E040E050E060E070E080E0E4
:1058900090E0A0E00E94289461F05F018FEFA81AC9
:1058A000B80A47EE59E06FEA74E0CF010E94231670
:1058B000F501212F207830E040E050E060E070E01A
:1058C00080E090E0A0E00E94289461F05F018FEFFB
:1058D000A81AB80A47EE59E065EB74E0CF010E94C0
:1058E0002316F50120E03D2F317040E050E060E0EC
:1058F00070E080E090E0A0E00E94289461F05F01F9
:105900008FEFA81AB80A47EE59E068EB74E0CF01B0
:105910000E942316F50120E03D2F327040E050E058
:1059200060E070E080E090E0A0E00E94289461F0E8
:105930005F018FEFA81AB80A47EE59E06DEB74E0EB
:10594000CF010E942316F50120E03D2F347040E086
:1059500050E060E070E080E090E0A0E00E942894D9
:1059600061F05F018FEFA81AB80A47EE59E064ECC6
:1059700074E0CF010E942316F50120E03D2F38701E
:1059800040E050E060E070E080E090E0A0E00E9445
:10599000289461F05F018FEFA81AB80A47EE59E02A
:1059A00067EC74E0CF010E942316F50120E03D2F43
:1059B000307140E050E060E070E080E090E0A0E016
:1059C0000E94289461F05F018FEFA81AB80A47EE91
:1059D00059E06CEC74E0CF010E942316F50120E041
:1059E0003D2F307240E050E060E070E080E090E0F9
:1059F000A0E00E94289461F05F018FEFA81AB80A16
:105A000047EE59E063ED74E0CF010E942316F501E3
:105A100020E030E040E050E06F2D647070E080E006
:105A200090E0A0E00E94289461F05F018FEFA81A37
:105A3000B80A47EE59E06AED74E0CF010E942316E0
:105A4000F5018091162E81FF19C020E03D2F3074A2
:105A500040E050E060E070E080E090E0A0E00E9474
:105A6000289461F05F018FEFA81AB80A47EE59E059
:105A70006EED74E0CF010E942316F5018091162E81
:105A80009091172E93FF19C020E030E040E0502F96
:105A9000507160E070E080E090E0A0E00E94289407
:105AA00061F05F018FEFA81AB80A47EE59E061EE86
:105AB00074E0CF010E942316F5018091162E90917B
:105AC000172E93FF19C020E030E040E0502F5072B5
:105AD00060E070E080E090E0A0E00E94289461F037
:105AE0005F018FEFA81AB80A47EE59E064EE74E040
:105AF000CF010E942316F5018091162E9091172E4A
:105B000093FF19C020E030E040E0502F507460E077
:105B100070E080E090E0A0E00E94289461F05F01D6
:105B20008FEFA81AB80A47EE59E06AEE74E0CF0189
:105B30000E942316F50120E03D2F307840E050E030
:105B400060E070E080E090E0A0E00E94289461F0C6
:105B50005F018FEFA81AB80A47EE59E065EF74E0CD
:105B6000CF010E942316F50120E030E04C2F417058
:105B700050E060E070E080E090E0A0E00E942894B7
:105B800061F05F018FEFA81AB80A47EE59E06AEF9B
:105B900074E0CF010E942316F50120E030E04C2F85
:105BA000427050E060E070E080E090E0A0E00E9491
:105BB000289461F05F018FEFA81AB80A47EE59E008
:105BC0006DEF74E0CF010E942316F50120E030E074
:105BD0004C2F447050E060E070E080E090E0A0E086
:105BE0000E94289461F05F018FEFA81AB80A47EE6F
:105BF00059E060E075E0CF010E942316F50120E036
:105C000030E040E050E06F2D687070E080E090E0A0
:105C1000A0E00E94289461F05F018FEFA81AB80AF3
:105C200047EE59E063E075E0CF010E942316F501CD
:105C300020E030E040E050E06F2D607170E080E0E7
:105C400090E0A0E00E94289461F05F018FEFA81A15
:105C5000B80A47EE59E067E075E0CF010E942316CD
:105C6000F50120E030E040E050E060E07E2D717012
:105C700080E090E0A0E00E94289461F05F018FEF47
:105C8000A81AB80A47EE59E06BE075E0CF010E9410
:105C90002316F5018091162E9091172E92FF19C0B0
:105CA00020E030E04C2F487050E060E070E080E091
:105CB00090E0A0E00E94289461F05F018FEFA81AA5
:105CC000B80A47EE59E066E175E0CF010E9423165D
:105CD000F5018091162E9091172E92FF19C020E0A9
:105CE00030E04C2F407150E060E070E080E090E0E8
:105CF000A0E00E94289461F05F018FEFA81AB80A13
:105D000047EE59E06AE175E0CF010E942316F501E4
:105D10008091162E9091172E92FF19C020E030E04E
:105D20004C2F407250E060E070E080E090E0A0E036
:105D30000E94289461F05F018FEFA81AB80A47EE1D
:105D400059E06EE175E0CF010E942316F5018091C4
:105D5000162E9091172E92FF19C020E030E04C2FA4
:105D6000407450E060E070E080E090E0A0E00E94CD
:105D7000289461F05F018FEFA81AB80A47EE59E046
:105D800062E275E0CF010E942316F5018091162E84
:105D900082FF19C020E030E04C2F407850E060E0F6
:105DA00070E080E090E0A0E00E94289461F05F0144
:105DB0008FEFA81AB80A47EE59E063E976E0CF0101
:105DC0000E942316F5018091162E82FF19C020E053
:105DD00030E040E0502F517060E070E080E090E0F3
:105DE000A0E00E94289461F05F018FEFA81AB80A22
:105DF00047EE59E066E275E0CF010E942316F501F7
:105E00008091162E9091172E93FF19C020E030E05C
:105E100040E0502F527060E070E080E090E0A0E041
:105E20000E94289461F05F018FEFA81AB80A47EE2C
:105E300059E069E275E0CF010E942316F5018091D7
:105E4000162E9091172E93FF19C020E030E040E00D
:105E5000502F547060E070E080E090E0A0E00E947D
:105E6000289461F05F018FEFA81AB80A47EE59E055
:105E700061E375E0CF010E942316F5018091162E93
:105E80009091172E94FF19C020E030E040E0502F91
:105E9000587060E070E080E090E0A0E00E942894FC
:105EA00061F05F018FEFA81AB80A47EE59E06AE384
:105EB00075E0CF010E942316F5018091162E85FF13
:105EC00019C020E030E040E050E06F2D607270E0DB
:105ED00080E090E0A0E00E94289461F05F018FEFE5
:105EE000A81AB80A47EE59E063E475E0CF010E94B2
:105EF0002316F5018091162E85FF19C020E030E0B1
:105F000040E050E06F2D607470E080E090E0A0E031
:105F10000E94289461F05F018FEFA81AB80A47EE3B
:105F200059E06CE475E0CF010E942316F5018091E1
:105F3000162E85FF1EC020E030E040E050E06F2DBF
:105F4000607870E080E090E0A0E00E94289489F002
:105F500047EE59E066E575E0CF01DF91CF911F91E3
:105F60000F91FF90EF90DF90CF90BF90AF900C9487
:105F70002316212F3D2F4C2F502F6F2D7E2D8D2D31
:105F80009C2DA0E00E94289441F48CE39AE09F931A
:105F90008F930E94239D0F900F90DF91CF911F91BF
:105FA0000F91FF90EF90DF90CF90BF90AF9008954A
:105FB0001F93CF93DF938091162ED0E082FF02C013
:105FC00010E801C010E081FDD0E427E04AE250E093
:105FD0006BE270E089E290E00E94BD6280E090E0B8
:105FE0000E944F11882311F0CDE001C0C5E026E0EA
:105FF0004AE250E06BE270E089E290E00E94BD620C
:1060000081E090E00E944F112C2F882311F0206135
:1060100001C02F7E50E060E08091162E9091172EE7
:10602000FC01E072FF2785FF02C0277F60E293FF3B
:1060300002C0277F56E094FD5860EF2B09F0606C9A
:106040003D2F412F70E080E090E0DF91CF911F91D4
:1060500008950E94D82FE9EFFDE120833183428328
:10606000538364837583868397838CE390E0918761
:10607000808725E4228720E8238727E02487158668
:1060800016861786108A118A938B828B85E0848B03
:1060900080E2858B168A178A108E81E0818F128E9E
:1060A000138E88E592E0958F848F168E178E10A23E
:1060B00011A212A213A214A215A217A216A248E2BC
:1060C00050E062E270E0CF010C94DA9FCF92DF9251
:1060D000EF92FF920F931F93CF93DF93EC018B010D
:1060E000FB0110826AE37AE00E942B9C892B61F409
:1060F00081E0F801808360917E0270917F0280E0F0
:1061000090E00E943F9CEC0168E37AE0CE010E949F
:106110002B9C892B61F48FEFF801808360917E02C4
:1061200070917F0280E090E00E943F9CEC01F12C96
:1061300000E010E0E12CD12CC12C209709F466C1BD
:1061400064E37AE0CE010E942B9C892B19F4FF2D89
:10615000F160FF2E60E37AE0CE010E942B9C892B38
:1061600019F48F2D8460F82E6DE27AE0CE010E9442
:106170002B9C892B19F4EF2DE260FE2E6BE27AE066
:10618000CE010E942B9C892B19F4FF2DF860FF2E65
:1061900068E27AE0CE010E942B9C892B19F48F2DA6
:1061A0008061F82E62E27AE0CE010E942B9C892B5E
:1061B00019F4EF2DE062FE2E6CE17AE0CE010E9430
:1061C0002B9C892B19F4FF2DF064FF2E69E17AE0F6
:1061D000CE010E942B9C892B19F48F2D8068F82EFC
:1061E00064E17AE0CE010E942B9C892B09F40160C6
:1061F0006DE07AE0CE010E942B9C892B09F40260AD
:106200006AE07AE0CE010E942B9C892B09F404609D
:1062100065E07AE0CE010E942B9C892B09F408608E
:106220006EEF79E0CE010E942B9C892B09F400616E
:1062300067EF79E0CE010E942B9C892B09F4006264
:1062400063EF79E0CE010E942B9C892B19F4ED2D90
:10625000E460DE2E60EF79E0CE010E942B9C892B5A
:1062600009F400646BEE79E0CE010E942B9C892B2F
:1062700009F4006868EE79E0CE010E942B9C892B1E
:1062800009F4116065EE79E0CE010E942B9C892B08
:1062900009F4126062EE79E0CE010E942B9C892BFA
:1062A00009F414606EED79E0CE010E942B9C892BDD
:1062B00009F418606AED79E0CE010E942B9C892BCD
:1062C00009F4106166ED79E0CE010E942B9C892BC8
:1062D00009F4106262ED79E0CE010E942B9C892BBB
:1062E00009F4106460ED79E0CE010E942B9C892BAB
:1062F00009F410686DEC79E0CE010E942B9C892B8B
:1063000019F4FE2DF160EF2E65EC79E0CE010E94CC
:106310002B9C892B19F48E2D8260E82E6CEB79E092
:10632000CE010E942B9C892B19F4EE2DE460EE2EF9
:1063300063EB79E0CE010E942B9C892B19F4FE2D92
:10634000F860EF2E60EB79E0CE010E942B9C892B48
:1063500019F48E2D8061E82E6AEA79E0CE010E9460
:106360002B9C892B19F4EE2DE062EE2E6FE979E07B
:10637000CE010E942B9C892B19F4FE2DF064EF2E88
:106380006BE979E0CE010E942B9C892B19F48D2DAD
:106390008860D82E67E979E0CE010E942B9C892B7A
:1063A00019F4ED2DE061DE2E6EE879E0CE010E9459
:1063B0002B9C892B19F4FD2DF062DF2E64E879E027
:1063C000CE010E942B9C892B19F48D2D8064D82E30
:1063D0006BE779E0CE010E942B9C892B19F4ED2DFF
:1063E000E068DE2E60E779E0CE010E942B9C892BCD
:1063F00019F4FC2DF160CF2E60917E0270917F0226
:1064000080E090E00E943F9CEC0197CE2F2D302F32
:10641000412F5E2D6D2D7C2D80E090E0DF91CF919E
:106420001F910F91FF90EF90DF90CF9008953F92D2
:106430004F925F926F927F928F929F92AF92BF9294
:10644000CF92DF92EF92FF920F931F93CF93DF9340
:10645000582EC9EFDDE100E010E08AE6E82E89E081
:10646000F82E852D8170382E852D8270482E95E569
:10647000C92E99E0D92E2DE5A22E29E0B22E3BE5BA
:10648000832E39E0932E44EB642E42E1742E552086
:1064900051F01F930F93FF92EF920E94239D0F9054
:1064A0000F900F900F903320A1F089858F938885EE
:1064B0008F93BF92AF920E94239D0F900F900F90E9
:1064C0000F904420C1F09F928F920E94239D0F90C5
:1064D0000F90442081F0DF92CF920E94239D28816B
:1064E00039814A815B816C817D818E819F810E948F
:1064F0008E2B0F900F907F926F920E94239D0F5FC3
:106500001F4F2A960F900F900430110509F0BFCF4E
:10651000DF91CF911F910F91FF90EF90DF90CF907F
:10652000BF90AF909F908F907F906F905F904F90B3
:106530003F90089580E599E09F938F930E94239D5B
:106540008091062A9091072AA091082AB091092AE1
:106550000F900F90813027EA92072EE1A207B10534
:1065600019F482E499E01DC0823026EA92072EE1F8
:10657000A207B10519F485E399E013C0823027EA38
:1065800092072EE1A207B10519F487E299E009C04C
:10659000823028EA92072EE1A207B10549F489E189
:1065A00099E09F938F930E94239D0F900F900895E1
:1065B000BF93AF939F938F9383E199E09F938F93C2
:1065C0000E94239D0F900F900F900F900F900F90AF
:1065D000089583E099E09F938F930E94239D0E94EA
:1065E000BA270E949A3284EB92E19F938F930E9484
:1065F000239D8EB390E00E94E96C80EE9DE19F9315
:106600008F938BEF98E09F938F930E94239D6091CF
:10661000600270916102809162029091630228EEA3
:1066200033E040E050E00E9420925F934F933F930D
:106630002F938BEE98E09F938F930E94239D82EE81
:1066400098E09F938F930E94239D0E94EB16809168
:10665000162E2DB73EB7205F3F4F0FB6F8943EBFC2
:106660000FBE2DBF80FF05C041E061E081E00E94C8
:10667000C7188EED98E09F938F930E94239D80E032
:106680000E949F290E94BE27809165021F928F93CE
:1066900085ED98E09F938F930E94239D8091C6146F
:1066A0001F928F938CEC98E09F938F930E94239D71
:1066B000809190028F9380918F028F9380918E02B0
:1066C0008F9380918D028F938EEB98E09F938F93A1
:1066D0000E94239D1F9280E48F9386EA98E09F9307
:1066E0008F930E94239D809142391F928F938091B6
:1066F00041391F928F9383E998E09F938F930E9473
:10670000239D809164021F928F938AE898E09F9363
:106710008F930E94239D8091660290916702A091C1
:106720006802B09169022DB73EB7225E3F4F0FB6A7
:10673000F8943EBF0FBE2DBF96FD03C08FE595E0D8
:1067400002C083E99AE09F938F9380E898E09F933B
:106750008F930E94239D83E00E9417320F900F9029
:106760000F900F901D9903C08FE595E002C083E95B
:106770009AE09F938F9384E798E09F938F930E9472
:10678000239D8AE698E09F938F930E94239D80919A
:1067900066020F900F900F900F900F900F9081FF57
:1067A00009C084E698E09F938F930E94239D0F90E9
:1067B0000F9013C080FD03C08FE595E002C083E910
:1067C0009AE09F938F9380E698E09F938F930E9427
:1067D000239D0F900F900F900F90809166029091E3
:1067E0006702A0916802B091690297FD03C08FE52E
:1067F00095E002C083E99AE09F938F9387E598E044
:106800009F938F930E94239D80E598E09F938F93A1
:106810000E94239D6091C9147091CA148091CB1479
:106820009091CC140E94E22984EB92E19F938F9384
:106830000E94239D8DB79EB708960FB6F8949EBF11
:106840000FBE8DBF779B03C08FE595E002C083E943
:106850009AE09F938F9387E498E09F938F930E9491
:10686000239D0E943A0E0E940B119F938F937F935A
:106870006F9389E398E09F938F930E94239D0E94DA
:10688000BA109F938F937F936F938BE298E09F93BF
:106890008F930E94239D81E090E00E947428809154
:1068A000C5369091C636A091C736B091C836BF9311
:1068B000AF939F938F938DE198E09F938F930E9466
:1068C000239D8091DA368F938091D9368F93809172
:1068D000D8368F938091D7368F9389E098E09F9335
:1068E0008F930E94239D8091C9369091CA36A091C2
:1068F000CB36B091CC36BF93AF939F938F938BEFF2
:1069000097E09F938F930E94239D2DB73EB72E5DF6
:106910003F4F0FB6F8943EBF0FBE2DBF8091DE36BD
:106920008F938091DD368F938091DC368F938091A9
:10693000DB368F9387EE97E09F938F930E94239D82
:1069400061E070E080E090E00E94BE1161E070E0E4
:1069500081E090E00E94BE110F900F900F900F9079
:106960000F900F90299903C08FE595E002C083E94D
:106970009AE09F938F938FED97E09F938F930E9460
:10698000239D0F900F900F900F902A9903C08FE5D1
:1069900095E002C083E99AE09F938F9387ED97E09B
:1069A0009F938F930E94239D80916602909167022E
:1069B000A0916802B09169020F900F900F900F9014
:1069C00094FD03C08FE595E002C083E99AE09F93B0
:1069D0008F938FEC97E09F938F930E94239D8091DC
:1069E000162E0F900F900F900F9085FF5FC081E0E3
:1069F0000E9472696091EA367091EB368091EC36B4
:106A00009091ED360E94CC9520E030E048EC52E4C5
:106A10000E9418959F938F937F936F9383E695E0E1
:106A20009F938F930E940F9D6091EE367091EF3689
:106A30008091F0369091F1360E94CA9520E030E0C6
:106A400040E85AE30E94C4979F938F937F936F937C
:106A500082E795E09F938F930E940F9D6091F2369D
:106A60007091F3368091F4369091F5360E94CA9574
:106A700020E030E040E85BE30E94C4979F938F934F
:106A80007F936F9383E895E09F938F930E940F9D70
:106A900084EB92E19F938F930E94239D8DB79EB7C5
:106AA00044960FB6F8949EBF0FBE8DBF0895F8941C
:106AB00091E2E0E0F0E0909357008491E2E0F0E0B2
:106AC000909357002491E4E0F0E090935700E49114
:106AD00090E0A0E0B0E0BC0155274427822F90E071
:106AE000A0E0B0E0BA2FA92F982F8827840F951F18
:106AF000A61FB71F8E0F911DA11DB11D8093062AE1
:106B00009093072AA093082AB093092A78940895AD
:106B1000CF93DF93CDB7DEB761970FB6F894DEBFA2
:106B20000FBECDBF48E250E062E270E089EF9DE128
:106B30000E94BC9F2091F91D3091FA1D4091FB1DD0
:106B40005091FC1D6091FD1D7091FE1D8091FF1DF7
:106B50009091001EAFEF0E94289411F40E942930FA
:106B600044E050E06EE170E0CE010B960E94BC9FC5
:106B70008B859C85AD85BE858F3F2FEF9207A20741
:106B8000B207A9F48AE090E4A0E0B0E08093660246
:106B900090936702A0936802B093690244E050E0CA
:106BA0006EE170E086E692E00E94DA9F08C0809372
:106BB000660290936702A0936802B0936902809185
:106BC000660290916702A0916802B0916902A2FFEB
:106BD00002C02A9A03C080E00E94DC2944E050E011
:106BE0006AE570E0CE010B960E94BC9F8B859C8568
:106BF000AD85BE858F3F2FEF9207A207B20789F4BC
:106C00001092C9141092CA141092CB141092CC1482
:106C100044E050E06AE570E089EC94E10E94DA9F7C
:106C200008C08093C9149093CA14A093CB14B09356
:106C3000CC1449E050E06EE070E08FED96E30E94E6
:106C4000BC9F0E94051344E050E06EE470E0CE016A
:106C50000B960E94BC9F8B859C85AD85BE8544E0CC
:106C600050E06EE470E08F3F9F4FAF4FBF4F29F46D
:106C700085E892E00E94DA9F04C085E892E00E94D5
:106C8000BC9F44E050E06AE470E0CE010B960E94A5
:106C9000BC9F8B859C85AD85BE8544E050E06AE451
:106CA00070E08F3F9F4FAF4FBF4F29F481E892E0D4
:106CB0000E94DA9F04C081E892E00E94BC9F44E0F9
:106CC00050E062E570E0CE010B960E94BC9F8B8580
:106CD0009C85AD85BE8544E050E062E570E08F3F65
:106CE0009F4FAF4FBF4F29F489E892E00E94DA9F8F
:106CF00004C089E892E00E94BC9F41E050E06DE151
:106D000070E0CE0141960E94BC9F898941E050E02D
:106D10006DE170E08F3F29F486EC94E10E94DA9FE8
:106D200004C086EC94E10E94BC9F41E050E06CE11D
:106D300070E0CE0141960E94BC9F898941E050E0FD
:106D40006CE170E08F3F29F485E692E00E94DA9FC3
:106D500004C085E692E00E94BC9F41E050E06BE1F8
:106D600070E0CE0141960E94BC9F898941E050E0CD
:106D70006BE170E08F3F29F484E692E00E94DA9F95
:106D800004C084E692E00E94BC9F4AE050E064E0C8
:106D900070E0CE0101960E94BC9F89814AE050E0DC
:106DA00064E070E08F3F29F480EE9DE10E94DA9F5D
:106DB00004C080EE9DE10E94BC9F44E050E066E587
:106DC00070E0CE010B960E94BC9F8B859C85AD85A3
:106DD000BE8544E050E066E570E08F3F9F4FAF4FC7
:106DE000BF4F29F48DE892E00E94DA9F04C08DE83D
:106DF00092E00E94BC9F44E050E067E170E0CE0169
:106E00000B960E94BC9F8B859C85AD85BE8544E01A
:106E100050E067E170E08F3F9F4FAF4FBF4F29F4C5
:106E200080E692E00E94DA9F04C080E692E00E9431
:106E3000BC9F8091600290916102A0916202B0912A
:106E4000630281389A41A640B105A0F088E394E03E
:106E50009F938F930E94239D80E197E2A0E0B0E092
:106E60008093600290936102A0936202B0936302E8
:106E70000F900F90609160027091610280916202A8
:106E8000909163020E94FC6442E050E062E070E096
:106E9000CE010F960E94BC9F8F85988942E050E0FA
:106EA00062E070E08F3F910529F48FEB94E10E943E
:106EB000DA9F04C08FEB94E10E94BC9F42E050E057
:106EC00060E070E0CE010F960E94BC9F8F8598898C
:106ED00042E050E060E070E08F3F910529F48DEBD7
:106EE00094E10E94DA9F04C08DEB94E10E94BC9F64
:106EF00061960FB6F894DEBF0FBECDBFDF91CF9184
:106F00000895CF92DF92EF92FF920E9429308AE09B
:106F100090E4A0E0B0E08093660290936702A093B3
:106F20006802B093690244E050E06EE170E086E6EA
:106F300092E00E94DA9F1092C9141092CA14109223
:106F4000CB141092CC1444E050E06AE570E089EC78
:106F500094E10E94DA9F82E2C82EDD24DA948CEC60
:106F6000E82E8BE3F82EC0928502D0928602E09242
:106F70008702F092880244E050E06EE470E085E819
:106F800092E00E94DA9FC0928102D0928202E09247
:106F90008302F092840244E050E06AE470E081E809
:106FA00092E00E94DA9F87ED94E3AFEEBCE380931A
:106FB000890290938A02A0938B02B0938C0244E0E2
:106FC00050E062E570E089E892E00E94DA9F8AE989
:106FD00099E9A9E1B0E480938D0290938E02A09389
:106FE0008F02B093900244E050E066E570E08DE8D7
:106FF00092E00E94DA9F1092C61480E00E94927480
:1070000041E050E06DE170E086EC94E10E94DA9F8F
:107010008AE1809365020E947F7341E050E06CE159
:1070200070E085E692E00E94DA9F8FE08093640230
:1070300041E050E06BE170E084E692E00E94DA9F6C
:107040008AE0E0EEFDE1DF011D928A95E9F74AE072
:1070500050E064E070E0CF010E94DA9F80E197E2A7
:10706000A0E0B0E08093600290936102A09362027E
:10707000B093630244E050E067E170E080E692E0A4
:107080000E94DA9F1092C0141092BF1442E050E0A8
:1070900062E070E08FEB94E10E94DA9F1092BE14E0
:1070A0001092BD1442E050E060E070E08DEB94E19E
:1070B0000E94DA9F81E00E949F2980E090E0FF908B
:1070C000EF90DF90CF900C94AC160E94A0706C9A59
:1070D0006B9A6A9A6F9A729A749A739A779A80984E
:1070E00080B3897F80BB8398849887E080937E00FB
:1070F000549A0E9457350E9488358091660290917B
:107100006702A0916802B091690294FD0E94AF707D
:107110000E94A80E80E090E00E94AC166091600290
:107120007091610280916202909163020E94FC64FE
:107130000E94BA10609318327093193280931A32F9
:1071400090931B328091660286FD239A219A229A9F
:10715000239A0E94BD0E1D9B05C01092C814109268
:10716000C714089581E090E09093C8148093C714E9
:107170000895CF93DF9390E04091C9145091CA14C1
:107180006091CB147091CC1441FD08C0209166022F
:1071900020FD04C021FF92C01D9B90C02DE8289FB8
:1071A000E001299FD00D1124CE018A5F904E9F935C
:1071B0008F9383E995E09F938F930E940F9DFE012B
:1071C000E150F14EDF01AA57BF4F2C910F900F9065
:1071D0000F900F90438154816581768180911C329C
:1071E00090911D32A0911E32B0911F32841B950BDD
:1071F000A60BB70B2223D1F1BF93AF939F938F932D
:10720000DF01A257BF4F11968C9111978F938C91EC
:107210008F93129711968C9111978F938C918F93D6
:1072200013978C911F928F9311978C911F928F932C
:1072300013968C911F928F9311978C911F928F931D
:10724000E957FF4F80811F928F931F922F9389E9F7
:1072500095E09F938F930E940F9D8DB79EB74696A2
:107260000FB6F8949EBF0FBE8DBF10C0BF93AF93F3
:107270009F938F9380EE95E09F938F930E940F9D35
:107280000F900F900F900F900F900F9084EB92E162
:107290009F938F930E94239D809180020F900F9067
:1072A000882361F01F928F9385E394E09F938F93DF
:1072B0000E94239D0F900F900F900F90DF91CF9120
:1072C00008958091FF1E882341F08091001F90E077
:1072D0000E94B9380E94AE0FF4CF0895CF93DF9388
:1072E000EC01888199818D372FE09207F1F018F435
:1072F000892BC1F04BC085382FE0920709F44CC0B0
:1073000089389F4009F042C080E89BE00E940F78D6
:10731000892B09F43FC080E89BE00E94FB7780E066
:107320000E94D6298DE79FE02EC0623199F5299AF7
:107330004091BD145091BE145695542F4427579533
:10734000479560E070E080E89BE00E94F1778091D3
:10735000C9149091CA14A091CB14B091CC14A0FF81
:1073600010C08091BE148F938091BD148F9383E5DC
:1073700093E19F938F930E94239D0F900F900F9006
:107380000F9085E89FE09983888304C01982188252
:1073900083E019C081E017C080E89BE00E940F786D
:1073A000892BC1F380E89BE00E94FB770E94613942
:1073B00040E250E060E070E080E89BE00E94F177FE
:1073C00089E89FE0E0CFDF91CF9108952F923F921F
:1073D0004F925F926F927F928F929F92AF92BF92E5
:1073E000CF92DF92EF92FF920F931F93CF93DF9391
:1073F000CDB7DEB72B970FB6F894DEBF0FBECDBF6B
:107400009B878A873A01FC0180819181892B11F049
:107410000C942F4F60917E0270917F02CA010E94EE
:107420003F9C60E870E0C3010E947F9C009759F484
:1074300060915D3B70915E3B8AE090E00E94D39C3E
:1074400081E00C94344F8130910561F4F301108197
:10745000912E990C9908892CE92CF92C092D492C8D
:10746000592CC0C082309105B9F4F3018081082EF7
:10747000000C990B982F88272181820F911D27FDE1
:107480009A95182F992E892E880C8808E82CF82CAC
:10749000082D482C582CA6C083309105C1F5F30166
:1074A0002081922F990F990B392F492F592F692F2E
:1074B000792F892F00E10E94CA9329014A01B62F32
:1074C000A72F382E292E2181922F990F990B392F12
:1074D000492F592F692F792F892F08E00E94CA93CD
:1074E00059016A017B018C019201A4016B2F7A2F53
:1074F000832D922D0E940194A2801A2D110F110B41
:10750000B12EC12ED12EE12EF12E012F59C004979C
:107510000CF460C0F3012081922F990F990B392F41
:10752000492F592F692F792F892F08E10E94CA937B
:1075300029014A01B62FA72F382E292E2181922FFB
:10754000990F990B392F492F592F692F792F892F8F
:1075500000E10E94CA9359016A017B018C019201EA
:10756000A4016B2F7A2F832D922D0E940194A3806A
:107570001A2D110F110BB12EC12ED12EE12EF12E8D
:10758000012F0E94019429014A01B62FA72F382EFE
:10759000292E2281922F990F990B392F492F592F7C
:1075A000692F792F892F08E00E94CA9359016A0137
:1075B0007B018C019201A4016B2F7A2F832D922DD8
:1075C0000E940194122F932E842EE52EF62E072F63
:1075D0002C0108C01AE0912C812CE12CF12C00E048
:1075E000412C512C34EB232E32E1332E3F922F923B
:1075F0000E94239D0F900F90212F392D482D5E2D35
:107600006F2D702FC2012537F3E63F07FDE64F07C8
:107610005105610571058105910511F40C944949E5
:107620002537E3E63E07EDE64E0751056105710596
:107630008105910511F008F0B9C12337F2E73F0742
:1076400041055105610571058105910511F40C9401
:10765000134C2337E2E73E074105510561057105EB
:107660008105910511F008F0BCC02536F4E63F070E
:1076700041055105610571058105910509F4FAC7B8
:107680002536E4E63E074105510561057105810592
:10769000910511F008F042C0A6E70E94289411F469
:1076A0000C94C8450E94289409F070F4A8E60E9442
:1076B000289411F40C949743A5E70E94289411F4A0
:1076C0000C94B2450C942D4F212F392D482D5E2D51
:1076D0006F2D702FC2012436F1E63F074105510599
:1076E000610571058105910511F40C943B4C25371A
:1076F000E2E63E07410551056105710581059105E9
:1077000009F448C52A333642410551056105710522
:107710008105910509F43EC30C942D4F212F392D7D
:10772000482D5E2D6F2D702FC2012737EFE63E07E3
:1077300041055105610571058105910511F40C9410
:10774000B3492737FFE63F0741055105610571053C
:107750008105910509F0C8F42436E9E63E074105A4
:107760005105610571058105910511F40C948B4556
:1077700025363E4641055105610571058105910596
:1077800011F40C94EB490C942D4F212F392D482DD9
:107790005E2D6F2D702FC2012536E2E73E074105B1
:1077A0005105610571058105910511F40C94C64AD6
:1077B0002936F2E73F07410551056105710581054D
:1077C000910511F40C94C24B233331474105510507
:1077D000610571058105910511F00C942D4F0C94F4
:1077E0003B4C212F392D482D5E2D6F2D702FC2015E
:1077F0002236F5E63F07F4E64F07510561057105AE
:107800008105910509F436C72236E5E63E07E4E630
:107810004E075105610571058105910511F008F0CC
:107820005CC02133F4E63F07F1E64F0751056105DF
:1078300071058105910509F4C1C22133E4E63E07D3
:10784000E1E64E075105610571058105910509F0D5
:10785000C0F42337F3E73F07410551056105710582
:107860008105910511F40C94274C283734474105C4
:107870005105610571058105910509F48BC20C94D0
:107880002D4F212F392D482D5E2D6F2D702FC201C8
:107890002837F4E63F07F1E64F075105610571050A
:1078A0008105910509F486C22C36E5E73E07E2E63C
:1078B0004E075105610571058105910509F46AC4FA
:1078C0002336344641465105610571058105910510
:1078D00011F00C942D4F0C943B4C212F392D482D39
:1078E0005E2D6F2D702FC2012D36E5E73E07E8E6CD
:1078F0004E075105610571058105910511F40C9440
:10790000514C2D36F5E73F07F8E64F075105610565
:1079100071058105910509F0E0F42237E2E73E07A1
:10792000E5E64E075105610571058105910511F4E4
:107930000C94F64823363D464846510561057105CD
:107940008105910511F00C942D4F0E94121D0C948D
:107950002F4F212F392D482D5E2D6F2D702FC201F5
:107960002436E3E63E07ECE64E0751056105710556
:107970008105910511F40C9459482736FFE63F071D
:10798000FCE64F075105610571058105910511F46C
:107990000C945C4823363243494651056105710514
:1079A0008105910511F00C942D4F28C2212F392DFE
:1079B000482D5E2D6F2D702FC2012037FCE63F074A
:1079C000F5E64F07F8E65F0761057105810591054A
:1079D00009F4ADC62037ECE63E07E5E64E07E8E6DB
:1079E0005E07610571058105910511F008F0E3C09E
:1079F0002437F8E73F07F4E74F07510561057105A4
:107A00008105910511F40C9434462437E8E73E07CC
:107A1000E4E74E075105610571058105910511F0F7
:107A200008F05EC02033F1E33F07F1E74F0751054F
:107A3000610571058105910511F40C94F648203318
:107A4000E1E33E07E1E74E07510561057105810558
:107A5000910509F0C0F42133F2E63F07F0E74F0744
:107A60005105610571058105910509F4A8C222330C
:107A7000324640475105610571058105910509F4BC
:107A8000F3C20C942D4F212F392D482D5E2D6F2DD3
:107A9000702FC2012037F5E63F07F2E74F07510587
:107AA000610571058105910511F40C94C64A2C36C7
:107AB000E4E73E074E075105610571058105910513
:107AC00011F40C94444E2133314341475105610573
:107AD00071058105910511F00C942D4F0C944949C5
:107AE000212F392D482D5E2D6F2D702FC2012B3681
:107AF000ECE63E07E5E74E07E2E65E076105710545
:107B00008105910509F446C32B36FCE63F07F5E7EE
:107B10004F07F2E65F07610571058105910509F0E0
:107B2000E0F42437E4E63E07E7E74E075105610538
:107B300071058105910511F40C94984E24373F4648
:107B40004F465246610571058105910511F00C946F
:107B50002D4F0C9400000C942F4F212F392D482DC0
:107B60005E2D6F2D702FC2012E36E1E63E07E8E64E
:107B70004E07E3E65E07610571058105910511F485
:107B80000C9408462633F9E63F07F5E74F07F5E67C
:107B90005F07610571058105910509F4CCC529369A
:107BA0003C4641465346610571058105910511F03A
:107BB0000C942D4F99C3212F392D482D5E2D6F2DFB
:107BC000702FC2012437F3E73F07F5E64F07F2E7CE
:107BD0005F07610571058105910511F40C94674AF1
:107BE0002437E3E73E07E5E64E07E2E75E07610577
:107BF00071058105910511F008F063C02337F5E6A2
:107C00003F07F2E74F07F0E75F0761057105810560
:107C1000910511F40C940D4D2337E5E63E07E2E79C
:107C20004E07E0E75E07610571058105910509F0E2
:107C3000D0F42136FDE63F07F5E74F07F8E65F078A
:107C4000610571058105910511F40C94D149223724
:107C5000374740475047610571058105910509F493
:107C600068C20C942D4F212F392D482D5E2D6F2D7C
:107C7000702FC2012436FDE63F07F3E64F07F2E717
:107C80005F07610571058105910509F45FC621361D
:107C9000ECE63E07E5E64E07E2E75E0761057105A3
:107CA0008105910509F464C523373247474750479A
:107CB000610571058105910511F00C942D4F0C940F
:107CC000794A212F392D482D5E2D6F2D702FC2013D
:107CD0002437E2E73E07E1E64E07E5E75E07610588
:107CE00071058105910509F48CC62437F2E73F0739
:107CF000F1E64F07F5E75F0761057105810591051D
:107D000009F0C8F42437E3E73E07E5E64E07E4E769
:107D10005E07610571058105910509F4D0C7273714
:107D2000304748475447610571058105910509F4BD
:107D300045C70C942D4F212F392D482D5E2D6F2DC9
:107D4000702FC2012F36ECE63E07EFE54E07E6E75F
:107D50005E07610571058105910509F4A2C52C3600
:107D6000F1E63F07F4E74F07F8E75F0761057105A4
:107D70008105910511F40C940B4E2237374640478C
:107D80005547610571058105910511F00C942D4F42
:107D90000C94354883E08093CD361092CF36109204
:107DA000CE364DEC56E362E182E492E00E943E7AE8
:107DB0000C942F4F0E94A71C0C942F4F21E042E1FE
:107DC00061E080ED0E94D96621E042E161E080ED52
:107DD0000E94D96621E042E161E080ED0E94D9660F
:107DE00021E042E161E080ED0E94D96621E042E1BC
:107DF00061E080ED0E94D9660C942F4F60917E0265
:107E000070917F0280E090E00E943F9C6CEE75E0F4
:107E10000E94609C892B09F0CEC060917E02709117
:107E20007F0280E090E00E943F9C8C01009709F463
:107E30009DC060E873E00E94609C892BE1F488EEAD
:107E400093E0A0E0B0E08093600290936102A09381
:107E50006202B093630268EE73E080E090E00E94FB
:107E6000FC6444E050E067E170E080E692E00E944C
:107E7000DA9F0C942F4F62EF75E0C8010E94609C5E
:107E8000892BE1F480E197E2A0E0B0E0809360020A
:107E900090936102A0936202B093630260E177E283
:107EA00080E090E00E94FC6444E050E067E170E014
:107EB00080E692E00E94DA9F0C942F4F65EF75E008
:107EC000C8010E94609C892BE1F480EA96E8A1E059
:107ED000B0E08093600290936102A0936202B0933D
:107EE000630260EA76E881E090E00E94FC6444E08E
:107EF00050E067E170E080E692E00E94DA9F0C9427
:107F00002F4F69EF75E0C8010E94609C892BE1F456
:107F100080E89AE1A6E0B0E080936002909361026D
:107F2000A0936202B093630260E87AE186E090E099
:107F30000E94FC6444E050E067E170E080E692E07B
:107F40000E94DA9F0C942F4F84EF95E09F938F93BC
:107F50000E94239D84EB92E19F938F930E94239D27
:107F60000F900F900F900F900C942F4F6091600224
:107F700070916102809162029091630228EE33E079
:107F800040E050E00E9420925F934F933F932F93E5
:107F900080EF95E09F938F930E94239D84EB92E165
:107FA0009F938F930E94239D0FB6F894DEBF0FBE60
:107FB000CDBF0C942F4F0E94EB160C942F4F609165
:107FC0007E0270917F0280E090E00E943F9C8C01D5
:107FD00063E97AE00E94609C892BA1F4809166029B
:107FE00090916702A0916802B0916902A2608093AB
:107FF000660290936702A0936802B0936902299A7F
:108000000C942F4F6FE575E0C8010E94609C892B8E
:10801000B1F48091660290916702A0916802B091DC
:108020006902AD7F8093660290936702A093680215
:10803000B093690280E00E94D6290C942F4F299BAF
:1080400003C083E99AE002C08FE595E09F938F9388
:1080500088EE95E09F938F930E94239D0F900F9041
:108060000F900F900C942F4F60917E0270917F02C1
:1080700080E090E00E943F9C8C0163E97AE00E94DE
:10808000609C892BE1F48091660290916702A09137
:108090006802B0916902A4608093660290936702BF
:1080A000A0936802B09369022A9A44E050E06EE11E
:1080B00070E086E692E00E94DA9F0C942F4F6FE505
:1080C00075E0C8010E94609C892BF1F480916602E2
:1080D00090916702A0916802B0916902AB7F809392
:1080E000660290936702A0936802B093690280E0F1
:1080F0000E94DC2944E050E06EE170E086E692E008
:108100000E94DA9F0C942F4F2A9B03C083E99AE0C8
:1081100002C08FE595E09F938F9380EE95E09F934B
:108120008F930E94239D0F900F900F900F900C94AF
:108130002F4F60917E0270917F0280E090E00E945C
:108140003F9C8C0163E97AE00E94609C892B19F4C2
:1081500077980C942F4F6FE575E0C8010E94609CE2
:10816000892B19F4779A0C942F4F779903C083E9E0
:108170009AE002C08FE595E09F938F9389EB97E09B
:108180009F938F930E94239D0F900F900F900F90BD
:108190000C942F4F60917E0270917F0280E090E0FE
:1081A0000E943F9C8C016DEF75E00E94609C892BC2
:1081B000D1F48091FF1E1F928F938091011F1F9217
:1081C0008F938091001F1F928F931F9284E18F9352
:1081D00086EB95E09F938F930E94239D0FB6F894B2
:1081E000DEBF0FBECDBF62E076E0C8010E94609C9A
:1081F000892B19F40E9461396DC061E77AE0C801EA
:108200000E94609C892BF9F560917E0270917F023B
:1082100080E090E00E943F9C009709F45BC00E94C0
:108220002C9B8531910530F59093C0148093BF1439
:1082300042E050E062E070E08FEB94E10E94DA9F50
:1082400060917E0270917F0280E090E00E943F9CEE
:10825000009709F43FC00E942C9B9093BE1480931A
:10826000BD1442E050E060E070E08DEB94E10E94CC
:10827000DA9F30C084EA95E09F938F930E94239DFC
:108280000F900F9027C08091C0148F938091BF14DE
:108290008F938BE995E09F938F930E94239D04EB2E
:1082A00012E11F930F930E94239D8091BE148F9320
:1082B0008091BD148F938CE895E09F938F930E94DB
:1082C000239D1F930F930E94239D0FB6F894DEBF4A
:1082D0000FBECDBF84EB92E19F938F930E94239DAD
:1082E0000F900F900C942F4F60917E0270917F023F
:1082F00080E090E00E943F9C8C016AEF74E00E9455
:10830000609C892B09F077C060917E0270917F029A
:1083100080E090E00E943F9C8C01009711F40C9447
:108320002F4F6FE67AE00E94609C892BB1F482E2C5
:108330009FEFACECBBE38093850290938602A09301
:108340008702B093880244E050E06EE470E085E874
:1083500092E00E94DA9F0C942F4F68E076E0C8010B
:108360000E94609C892BB1F482E29FEFACECBAE3EF
:108370008093850290938602A0938702B09388022F
:1083800044E050E06EE470E085E892E00E94DA9FFD
:108390000C942F4FC8010E94289B2B013C0120E028
:1083A00030E0A9010E9413958823D9F081E00E9452
:1083B00058109B01AC01C301B2010E941895609353
:1083C000850270938602809387029093880244E02E
:1083D00050E06EE470E085E892E00E94DA9F0C9431
:1083E0002F4F8FE795E09F938F930E94239D0F90CF
:1083F0000F900C942F4F6DEF74E0C8010E94609CA9
:10840000892B09F077C060917E0270917F0280E035
:1084100090E00E943F9C8C01009711F40C942F4F28
:108420006FE67AE00E94609C892BB1F482E29FEFB4
:10843000ACECBBE38093810290938202A093830211
:10844000B093840244E050E06AE470E081E892E096
:108450000E94DA9F0C942F4F68E076E0C8010E94DA
:10846000609C892BB1F482E29FEFACECBAE380937D
:10847000810290938202A0938302B093840244E02D
:1084800050E06AE470E081E892E00E94DA9F0C9488
:108490002F4FC8010E94289B2B013C0120E030E0B7
:1084A000A9010E9413958823D9F082E00E945810F8
:1084B0009B01AC01C301B2010E9418956093810237
:1084C00070938202809383029093840244E050E090
:1084D0006AE470E081E892E00E94DA9F0C942F4FEA
:1084E00082E795E09F938F930E94239D0F900F90BA
:1084F0000C942F4F65EF74E0C8010E94609C892B9B
:1085000009F073C060917E0270917F0280E090E07C
:108510000E943F9C8C01009711F40C942F4F6FE642
:108520007AE00E94609C892BB1F487ED94E3AFEE72
:10853000BCE38093890290938A02A0938B02B0934C
:108540008C0244E050E062E570E089E892E00E942D
:10855000DA9F0C942F4F68E076E0C8010E94609C7F
:10856000892B51F483E695E09F938F930E94239D7E
:108570000F900F900C942F4FC8010E94289B2B0145
:108580003C0120E030E0A9010E941395882319F1F5
:1085900080E00E9458104B015C0121EE3AE744E96B
:1085A0005EE3C301B2010E943494A50194010E94CC
:1085B00018956093890270938A0280938B0290933E
:1085C0008C0244E050E062E570E089E892E00E94AD
:1085D000DA9F0C942F4F86E595E09F938F930E942E
:1085E000239D0F900F900C942F4F0E94A6109F93E5
:1085F0008F937F936F938FE495E09F938F930E9467
:10860000239D82E00E9458102091810230918202C5
:1086100040918302509184020E94C497162F072F25
:10862000F82EE92E81E00E945810EF92FF920F93EE
:108630001F932091850230918602409187025091CC
:1086400088020E94C4979F938F937F936F9383E4D4
:1086500095E09F938F930E94239D84EB92E19F93DB
:108660008F930E94239D0FB6F894DEBF0FBECDBF3F
:108670000C942F4F60917E0270917F0280E090E019
:108680000E943F9C009711F10E94D52A0091C914C5
:108690001091CA142091CB143091CC14601771073B
:1086A0008207930769F16093C9147093CA14809389
:1086B000CB149093CC1444E050E06AE570E089EC70
:1086C00094E10E94DA9F82EB97E002C08BEA97E088
:1086D0009F938F930E94239D6091C9147091CA1437
:1086E0008091CB149091CC140E94E22984EB92E10A
:1086F0009F938F930E94239D0F900F900F900F9048
:1087000080EA97E09F938F930E94239D6FEF7FEF06
:10871000CB010E94E22984EB92E19F938F930E9408
:10872000239D0F900F900F900F900C942F4F0E944D
:10873000B7260C942F4FF3018481843329F440E051
:1087400061E080E00E94C71880918002882311F4C4
:108750000C942F4F1F928F938DE997E09F938F93E7
:108760000E94239D0F900F900F900F900C942F4F0D
:10877000F3018481893709F080C060917E02709195
:108780007F0280E090E00E943F9C8C0163E97AE0E8
:108790000E94609C892B51F480916602909167023F
:1087A000A0916802B0916902906410C06FE575E015
:1087B000C8010E94609C892BD1F48091660290913F
:1087C0006702A0916802B09169029F7B8093660264
:1087D00090936702A0936802B093690244E050E06E
:1087E0006EE170E086E692E00E94DA9F46C06DE09E
:1087F00076E0C8010E94609C892B21F58091F81DCC
:108800008F938091F71D8F938091F61D8F938091A8
:10881000F51D8F938091F41D8F938091F31D8F939D
:108820008091F21D8F938091F11D8F9388E195E0E7
:108830009F938F930E94239D0FB6F894DEBF0FBEC7
:10884000CDBF1BC08091660290916702A091680223
:10885000B091690296FF03C083E99AE002C08FE5F8
:1088600095E09F938F9384E195E09F938F930E946F
:10887000239D0F900F900F900F908091800288237E
:1088800011F40C942F4F1F928F938AE997E09F93D6
:108890008F930E94239D0F900F900F900F900C9438
:1088A0002F4FF30184818737E9F560917E02709143
:1088B0007F0280E090E00E943F9C0097D9F00E94E8
:1088C000289B2B013C0120E030E0A9010E94139578
:1088D000882381F040928D0250928E0260928F0226
:1088E0007092900244E050E066E570E08DE892E01E
:1088F0000E94DA9F809190028F9380918F028F93D4
:1089000080918E028F9380918D028F9386E095E007
:108910009F938F930E94239D0F900F900F900F9025
:108920000F900F9080918002882311F40C942F4FA8
:108930001F928F9387E997E09F938F930E94239DC7
:108940000F900F900F900F900C942F4F60917E021C
:1089500070917F0280E090E00E943F9C8C0163E96F
:108960007AE00E94609C409066025090670260909E
:10897000680270906902892B19F4689457F809C04D
:108980006FE575E0C8010E94609C892B99F4E8941A
:1089900057F84092660250926702609268027092A5
:1089A000690244E050E06EE170E086E692E00E94E9
:1089B000DA9F13C057FE03C083E99AE002C08FE537
:1089C00095E09F938F9382E095E09F938F930E9411
:1089D000239D0F900F900F900F908091800288231D
:1089E00011F40C942F4F1F928F9384E997E09F937B
:1089F0008F930E94239D0F900F900F900F900C94D7
:108A00002F4F60917E0270917F0280E090E00E9483
:108A10003F9C8C0163E176E00E94609C892B11F4FD
:108A200089E108C067E176E0C8010E94609C892B5B
:108A300049F480E18093C4001092C50082E08093E5
:108A4000C00055C06BE176E0C8010E94609C892B94
:108A500011F488E0EFCF60E276E0C8010E94609CEC
:108A6000892B39F065E276E0C8010E94609C892B71
:108A700011F483E0DFCF8091C400893141F48DEFA0
:108A800094E09F938F930E94239D0F900F9080916D
:108A9000C400803141F488EF94E09F938F930E944B
:108AA000239D0F900F908091C400883041F482EF95
:108AB00094E09F938F930E94239D0F900F9080913D
:108AC000C400833041F48CEE94E09F938F930E9416
:108AD000239D0F900F908091C400883041F486EE62
:108AE00094E09F938F930E94239D0F900F9080910D
:108AF0008002882311F40C942F4F1F928F9381E9E9
:108B000097E09F938F930E94239D0F900F900F905B
:108B10000F900C942F4F60917E0270917F0280E045
:108B200090E00E943F9C6FE67AE00E94609C892B57
:108B300011F481E001C080E00E949F2980918002B1
:108B4000882311F40C942F4F1F928F938EE897E097
:108B50009F938F930E94239D0F900F900F900F90E3
:108B60000C942F4F0E94BE2780918002882311F41D
:108B70000C942F4F1F928F938BE897E09F938F93C6
:108B80000E94239D0F900F900F900F900C942F4FE9
:108B90000E94BA2780918002882311F40C942F4FF1
:108BA0001F928F9388E897E09F938F930E94239D55
:108BB0000F900F900F900F900C942F4F60917E02AA
:108BC00070917F0280E090E00E943F9C0E942C9B6D
:108BD000803170F48093C6140E94927441E050E09A
:108BE0006DE170E086EC94E10E94DA9F0C942F4FC7
:108BF0008091C6141F928F938CED94E09F938F9376
:108C00000E94239D0F900F900F900F900C942F4F68
:108C100060917E0270917F0280E090E00E943F9C14
:108C20000E942C9B95EF980F903170F48093650211
:108C30000E947F7341E050E06CE170E085E692E0D5
:108C40000E94DA9F0C942F4F809165021F928F93A0
:108C500083ED94E09F938F930E94239D0F900F903C
:108C60000F900F900C942F4F60917E0270917F02B5
:108C700080E090E00E943F9C009789F04AE050E03D
:108C8000BC0180EE9DE10E94709C4AE050E064E0EF
:108C900070E080EE9DE10E94DA9F0C942F4F80EEF1
:108CA0009DE19F938F938AE296E09F938F930E941A
:108CB0000F9D0F900F900F900F900C942F4F60917D
:108CC0007E0270917F0280E090E00E943F9C8C01C8
:108CD00060E873E00E94609C892BE1F4219A809106
:108CE000660290916702A0916802B091690280616A
:108CF0008093660290936702A0936802B093690222
:108D000044E050E06EE170E086E692E00E94DA9F77
:108D10000C942F4F6EEF74E0C8010E94609C892B69
:108D2000E1F4229A8091660290916702A091680214
:108D3000B091690280628093660290936702A0936B
:108D40006802B093690244E050E06EE170E086E6AC
:108D500092E00E94DA9F0C942F4F62E673E0C80104
:108D60000E94609C892BE1F4239A80916602909185
:108D70006702A0916802B0916902806480936602E4
:108D800090936702A0936802B093690244E050E0B8
:108D90006EE170E086E692E00E94DA9F0C942F4F1D
:108DA00061EA74E0C8010E94609C892BE1F4239A77
:108DB0008091660290916702A0916802B091690269
:108DC00080688093660290936702A0936802B093D4
:108DD000690244E050E06EE170E086E692E00E94B5
:108DE000DA9F0C942F4F6AE573E0C8010E94609CE3
:108DF000892B79F581E08093313289EF9DE1909361
:108E00003332809332321092353210923432809164
:108E1000660290916702A0916802B0916902916028
:108E20008093660290936702A0936802B0936902F0
:108E300044E050E06EE170E086E692E00E94DA9F46
:108E400041E352E362E182E492E00E943E7A0C94B4
:108E50002F4F69E873E0C8010E94609C892B21F5BF
:108E6000E9E2FEE189E49EE1119211928E179F07DB
:108E7000D9F78091660290916702A0916802B09143
:108E8000690292608093660290936702A0936802E1
:108E9000B093690244E050E06EE170E086E692E053
:108EA0000E94DA9F0C942F4F6FE575E0C8010E9475
:108EB000609C4091660250916702609168027091D7
:108EC0006902892BC1F44F705C7F40936602509316
:108ED000670260936802709369022B9A44E050E045
:108EE0006EE170E086E692E00E94DA9F8091D636CD
:108EF0000E948D73B4C744FF03C083E99AE002C0A7
:108F00008FE595E09F938F9388EC94E09F938F93E8
:108F10000E94239D809166020F900F900F900F90FA
:108F200085FF03C083E99AE002C08FE595E09F9337
:108F30008F938DEB94E09F938F930E94239D80915C
:108F400066020F900F900F900F9086FF03C083E989
:108F50009AE002C08FE595E09F938F9382EB94E0B7
:108F60009F938F930E94239D809166020F900F9094
:108F70000F900F9087FF03C083E99AE002C08FE54E
:108F800095E09F938F9387EA94E09F938F930E943D
:108F9000239D8091660290916702A0916802B09132
:108FA00069020F900F900F900F9090FF03C083E91C
:108FB0009AE002C08FE595E09F938F938CE994E04F
:108FC0009F938F930E94239D8091660290916702E8
:108FD000A0916802B09169020F900F900F900F90CE
:108FE00091FF03C083E99AE002C08FE595E09F936B
:108FF0008F9381E994E09F938F930E94239D8091AA
:10900000660290916702A0916802B09169020F9088
:109010000F900F900F9091FF22C782E396E00E947D
:109020004B9D99E2E92E9EE1F92E0BE010E02AE338
:10903000822E26E0922EF70180819181F2E0EF0EE0
:10904000F11C9F938F931F930F939F928F920E9477
:109050000F9D0F5F1F4F0F900F900F900F900F906D
:109060000F900B31110539F7FAC684E897E09F930A
:109070008F930E94239D809180020F900F908823F0
:1090800061F01F928F9381E897E09F938F930E94E6
:10909000239D0F900F900F900F90F89498E088E127
:1090A0000FB6F894A895809360000FBE909360006F
:1090B000FFCF0E948A66D3C660917E0270917F02C4
:1090C00080E090E00E943F9C8C0163E97AE00E947E
:1090D000609C892BE9F40E948372809166029091D2
:1090E0006702A0916802B09169028D7F81608093D0
:1090F000660290936702A0936802B093690244E00D
:1091000050E06EE170E086E692E00E94DA9FA7C62A
:109110006FE575E0C8010E94609C892BE1F40E9414
:10912000BA718091660290916702A0916802B09135
:1091300069028C7F8093660290936702A093680215
:10914000B093690244E050E06EE170E086E692E0A0
:109150000E94DA9F84C665E476E0C8010E94609CA4
:10916000892BE9F40E94BA7180916602909167029E
:10917000A0916802B09169028E7F8260809366023E
:1091800090936702A0936802B093690244E050E0B4
:109190006EE170E086E692E00E94DA9F60C6809100
:1091A000660281FF0FC085E496E09F938F938DE860
:1091B00094E09F938F930E94239D0F900F900F90A8
:1091C0000F904DC680FF03C083E99AE002C08FE58F
:1091D00095E09F938F9389E894E09F938F930E94EB
:1091E000239D0F900F900F900F9039C680912F32D2
:1091F0008F9380912E328F9380912D328F93809117
:109200002C328F9380912B328F9380912A328F93BF
:10921000809129328F93809128328F9380912732C9
:109220008F93809126328F93809125328F938091F6
:1092300024328F93809123328F93809122328F93A7
:10924000809121328F93809120328F9385E597E032
:109250009F938F930E94239D84EB92E19F938F9322
:109260000E94239D809180020FB6F894DEBF0FBE4E
:10927000CDBF882309F4F3C51F928F9382E597E051
:109280009F938F930E94239D0F900F900F900F90AC
:10929000E6C5F89489E021E030E0F90180935700B9
:1092A000C895E02C20E030E0F90180935700C89584
:1092B000F02C7894F89423E030E0F9018093570083
:1092C000C895002D22E030E0F90180935700C89541
:1092D000102D78948091092A8F938091082A8F937A
:1092E0008091072A8F938091062A8F9388E497E0D4
:1092F0009F938F930E94239D1F92EF921F92FF9244
:109300001F920F931F921F9381E297E09F938F9379
:109310000E94239D0E945828809166001F928F937F
:1093200085E197E09F938F930E94239D84EB92E1C8
:109330009F938F930E94239D809180020FB6F89493
:10934000DEBF0FBECDBF882309F489C51F928F935E
:1093500082E197E09F938F930E94239D0F900F903F
:109360000F900F907CC560E070E080E090E00E947C
:10937000BE1160E070E081E090E00E94BE1180913B
:109380008002882309F46BC51F928F938FE097E0CA
:109390009F938F930E94239D0F900F900F900F909B
:1093A0005EC50E947A263F922F920E94239D809153
:1093B00080020F900F90882309F451C51F928F935C
:1093C0008CE097E09F938F930E94239D0F900F90C6
:1093D0000F900F9044C560917E0270917F0280E0F3
:1093E00090E00E943F9C62E076E00E94609C892BA6
:1093F00031F5F8948BEB9BE00E94157B8C01892B57
:1094000069F0C8010F960E94F678B80188E092E0F2
:109410000E94907CC8010E94767BF0CF8BEB9BE092
:109420000E94697B892B29F08BEB9BE00E94297BB2
:10943000F5CF8BEB9BE00E94117B789436C08BEBD1
:109440009BE00E94157B8C018AE4E82E86E0F82ED2
:109450000115110551F1F80186811F928F938085C6
:109460001F928F9385811F928F9381851F928F9377
:1094700087811F928F9384811F928F9383811F9284
:109480008F9382811F928F9382851F928F93FF9279
:10949000EF920E940F9DC8010E94767B8C010FB64F
:1094A000F894DEBF0FBECDBFD3CF8091800288235A
:1094B00009F4D5C41F928F9389E097E09F938F930F
:1094C0000E94239D0F900F900F900F90C8C4609141
:1094D0007E0270917F0280E090E00E943F9C69E8EC
:1094E00076E00E94609C892B09F0B9C40E94813704
:1094F000B6C460917E0270917F0280E090E00E948D
:109500003F9C8C0160E976E00E94609C892BD1F43D
:109510008091660290916702A0916802B091690201
:10952000977F8093660290936702A0936802B0933E
:10953000690244E050E06EE170E086E692E00E944D
:10954000DA9F8DC468E076E0C8010E94609C892B98
:10955000D1F48091660290916702A0916802B09167
:10956000690298608093660290936702A0936802F4
:10957000B093690244E050E06EE170E086E692E06C
:109580000E94DA9F6CC40E943A0E69C460917E0208
:1095900070917F0280E090E00E943F9C8C0164E02B
:1095A00077E00E942B9C892B19F40E94293057C424
:1095B000F80180818332D1F44AE050E060E070E04D
:1095C000C80101960E94ED987B836A8360917E02B8
:1095D00070917F0280E090E00E943F9C8C012A8184
:1095E0003B81243031050CF09EC002C01B821A82E0
:1095F0000115110509F497C01982BE016F5F7F4FF5
:10960000C8010E94663019013A014B01B82FA92FF9
:109610008AE02A813B81829FF001839FF00D112413
:10962000E750F24E4080518032813C8383818D83AC
:1096300094819E8325812F8336813887878189870E
:109640009101A301B4018B2F9A2F5201CC80DD80B0
:10965000EE80FF80088519850E941F9409F466C07A
:109660008981811103C0208231822AC0181684F4B6
:10967000422853289C81692A2D81722A3E81832A9F
:109680008F81982A9885B92B2985A22B408217C0F3
:10969000209430946094709480949094B095A095A8
:1096A000242053203C8163228D8178229E8189224F
:1096B0002F8192223885B3238985A8232082518265
:1096C0006282738284829582B683A78348E250E0E7
:1096D00062E270E089EF9DE10E94DA9F8CEF96E0F4
:1096E0009F938F930E94239D8AE02A813B81829FD2
:1096F000F001839FF00D1124E750F24E208131815B
:109700004281538164817581868197810E948E2B6D
:1097100084EB92E19F938F930E94239D0F900F9073
:109720000F900F9003C082E00E94173280EF96E006
:109730009F938F930E94239D2FEF3FEF4FEF5FEF9B
:109740006FEF7FEF8FEF9FEF0E948E2B84EB92E104
:109750009F938F930E94239D809180020F900F9082
:109760000F900F90882309F47AC31F928F938DEE88
:1097700096E09F938F930E94239D0F900F900F90E0
:109780000F906DC360917E0270917F0280E090E047
:109790000E943F9CFC0120812332A1F44AE050E06A
:1097A00060E070E001960E94ED988B0160917E026E
:1097B00070917F0280E090E00E943F9C0430110590
:1097C000ECF402C000E010E00097C1F04AE050E085
:1097D00060E070E00E941B9A2AE0209FF001219F28
:1097E000F00D1124E750F24E7187608748E250E097
:1097F00062E270E089EF9DE10E94DA9F81E00E94C1
:10980000173280918002882309F429C31F928F9315
:109810008AEE96E09F938F930E94239D0F900F9066
:109820000F900F901CC30E947F7B80918002882341
:1098300009F415C31F928F9387EE96E09F938F9341
:109840000E94239D0F900F900F900F9008C30E94CD
:10985000E93280918002882309F401C31F928F931B
:1098600084EE96E09F938F930E94239D0F900F901C
:109870000F900F90F4C280E090E00E9474288091D5
:109880008002882309F4EBC21F928F9381EE96E049
:109890009F938F930E94239D0F900F900F900F9096
:1098A000DEC28091162E81FF2DC00E940026892BDA
:1098B00049F580910D2A8F9380910C2A8F93809186
:1098C0000B2A8F9380910A2A8F9386ED96E09F93BF
:1098D0008F930E94239D8091FA368F938091F93661
:1098E0008F938091F8368F938091F7368F9389EC20
:1098F00096E09F938F930E94239D0FB6F894DEBF4E
:109900000FBECDBF84EB92E19F938F930E94239D66
:109910008091162E9091172E0F900F9093FF63C099
:1099200081E090E00E9478251B012C0180E090E00E
:109930000E9478257B018C010E94D6245F924F9271
:109940003F922F9288EB96E09F938F930E94239DE6
:109950001F930F93FF92EF9288EA96E09F938F9365
:109960000E94239D370148019701A80171018201DE
:10997000B101C2010E9473239F938F937F936F93D2
:109980008DE996E09F938F930E94239D262D372D7E
:10999000482D592D622D7F2D842D912F0E94D42387
:1099A0009F938F937F936F938FE896E09F938F930E
:1099B0000E94239D262D372D482D592D622D7F2D58
:1099C000842D912F0E9439249F938F937F936F93BF
:1099D0008CE796E09F938F930E94239D0FB6F89497
:1099E000DEBF0FBECDBF84EB92E19F938F930E94A9
:1099F000239D809180020F900F90882309F42FC23D
:109A00001F928F9389E796E09F938F930E94239DE7
:109A10000F900F900F900F9022C28091162E82FF10
:109A200043C021E048E061E083E00E942D1A80916C
:109A3000FD1E8F938091FC1E8F938091FB1E8F9350
:109A40008091FA1E8F938091F91E8F938091F81E5A
:109A50008F938091F71E8F938091F61E8F9382E6ED
:109A600096E09F938F930E94239D3F922F920E9496
:109A7000239D8091F51E8F938091F41E8F9380918A
:109A8000F31E8F938091F21E8F9384E596E09F934F
:109A90008F930E94239D3F922F920E94239D0FB689
:109AA000F894DEBF0FBECDBF8091162E85FF5CC03F
:109AB00081E00E9472696091EA367091EB36809184
:109AC000EC369091ED360E94CC9520E030E048ECE9
:109AD00052E40E9418959F938F937F936F9383E630
:109AE00095E09F938F930E940F9D6091EE36709149
:109AF000EF368091F0369091F1360E94CA9520E0C1
:109B000030E040E85AE30E94C4979F938F937F937D
:109B10006F9382E795E09F938F930E940F9D6091D2
:109B2000F2367091F3368091F4369091F5360E94BA
:109B3000CA9520E030E040E85BE30E94C4979F9321
:109B40008F937F936F9383E895E09F938F930E9409
:109B50000F9D84EB92E19F938F930E94239D0FB6FC
:109B6000F894DEBF0FBECDBF8091162E9091172EB8
:109B700094FF3FC00E94921E20E030E048EC52E487
:109B8000162F072FF82EE92E0E94C49720E836EEF4
:109B900045EC57E40E94189521E03EED42E45EE377
:109BA0000E9431989B01AC0160E070E080E89FE387
:109BB0000E9434942BE43AE34DEB57E30E9418954E
:109BC0009F938F937F936F93EF92FF920F931F93C7
:109BD0008BE396E09F938F930E94239D84EB92E109
:109BE0009F938F930E94239D0FB6F894DEBF0FBE04
:109BF000CDBF80918002882309F431C11F928F93D9
:109C000088E396E09F938F930E94239D0F900F907F
:109C10000F900F9024C160917E0270917F0280E0CE
:109C200090E00E943F9C65E976E00E94609C892B51
:109C300099F460917E0270917F0280E090E00E9432
:109C40003F9C009709F40BC10E942C9B90915201FC
:109C5000892B8093520103C1809152018F701F9212
:109C60008F938CE794E09F938F930E94239D84EBC6
:109C700092E19F938F930E94239D0F900F900F90DE
:109C80000F900F900F90EBC060917E0270917F0259
:109C900080E090E00E943F9C009711F14AE050E084
:109CA00060E070E00E94ED98603198F46093640287
:109CB0001F926F938BE296E09F938F930E94239D58
:109CC00041E050E06BE170E084E692E00E94DA9FB0
:109CD00011C0809164021F928F9382E296E006C0C9
:109CE000809164021F928F9389E196E09F938F93F6
:109CF0000E94239D0F900F900F900F9084EB92E1A4
:109D00009F938F930E94239D809180020F900F90CC
:109D1000882309F4A4C01F928F9386E196E09F9355
:109D20008F930E94239D0F900F900F900F9097C0DC
:109D300060917E0270917F0280E090E00E943F9CE3
:109D40008C0163E97AE00E94609C892BE1F40E9417
:109D5000AF708091660290916702A0916802B09105
:109D6000690290618093660290936702A0936802F3
:109D7000B093690244E050E06EE170E086E692E064
:109D80000E94DA9F6CC06FE575E0C8010E94609C7C
:109D9000892B99F5F8940E94BC700FB6F894A89599
:109DA00080916000886180936000109260000FBE17
:109DB00084B7877F84BF8091600088618093600052
:109DC0001092600078948091660290916702A09151
:109DD0006802B09169029F7E809366029093670249
:109DE000A0936802B093690244E050E06EE170E035
:109DF00086E692E00E94DA9F32C06AE976E0C80106
:109E00000E94609C409166025091670260916802D6
:109E100070916902892B69F454FF02C0F894FFCF56
:109E20008BE694E09F938F930E94239D0F900F9059
:109E300016C054FF03C083E99AE002C08FE595E0A5
:109E40009F938F9387E694E09F938F930E94239D27
:109E50000F900F900F900F9002C00E949E26EA85EF
:109E6000FB851182108283E02B960FB6F894DEBF3B
:109E70000FBECDBFDF91CF911F910F91FF90EF905B
:109E8000DF90CF90BF90AF909F908F907F906F901A
:109E90005F904F903F902F900895CF93DF93EC0108
:109EA00088819981009741F0843C924109F4A0C0D7
:109EB0001982188283E0A7C00E94653880916602EB
:109EC00080FD05C081FF01C01D9B0E94BA71809179
:109ED00070008C7F809370008091B60080628093C8
:109EE000B6001092B20082E08093B1008091B6007B
:109EF0008770E1F78091700081608093700068E561
:109F00007EE080E090E00E9489700E94BA2780E0A5
:109F10000E949F2981E993E19F938F930E94239D43
:109F20000E94EB160F900F908091043790910537A7
:109F3000892B51F48FE793E19F938F930E94239D88
:109F40000E9481370F900F908091162E9091172EBE
:109F500091FD0E9436668091162E9091172E93FDEA
:109F60000E948E248091162E9091172E92FF06C08B
:109F700021E04CE061E080ED0E94D9668091C6143A
:109F80000E949274809165020E947F730E947C738C
:109F90008093AB0B809165020E947F738091C61401
:109FA0001F928F938091AB0B1F928F938FE996E056
:109FB0009F938F930E940F9D1092AD0B1092AC0B4C
:109FC0000F900F900F900F900F900F9086E592E0FA
:109FD0009093E9368093E83683E290E09093C21440
:109FE0008093C11484EC92E19983888381E00BC053
:109FF0006332E1F745E452E360E070E08CEA9BE015
:10A000000E94E639E3CFDF91CF9108950F931F931C
:10A01000CF93DF93EC018A0188819981009711F138
:10A02000893D924121F01982188283E020C062317B
:10A03000E9F4A80162E170E08CEA9BE00E94E63955
:10A0400084E08093CD361092CF361092CE361093A6
:10A05000D1360093D0364DEC56E362E182E492E0D3
:10A060000E943E7A89ED92E19983888381E0DF91B5
:10A07000CF911F910F9108958436910514F19F930C
:10A080008F9385EF96E09F938F930E940F9D809111
:10A09000203290912132A0912232B0912332019648
:10A0A000A11DB11D8093203290932132A0932232C2
:10A0B000B09323320F900F900F900F9081E090E0BB
:10A0C000089580E090E008952F923F924F925F9222
:10A0D0006F927F928F929F92AF92BF92CF92DF92B8
:10A0E000EF92FF920F931F93CF93DF93CDB7DEB71D
:10A0F000C959D1090FB6F894DEBF0FBECDBFCD56FA
:10A10000DF4F99838883C359D040F62E8A0123E814
:10A11000621304C080EB9BE00E94BD7FCD56DF4FF1
:10A12000A881B981C359D0408D919C918B36B2E101
:10A130009B0711F40C94D85F38F4009781F08D35AB
:10A14000904109F4FCC4F0C48D3722E1920709F470
:10A15000CAC48438924111F40C94E05FE5C449EE1E
:10A1600059E061E870E080EB9BE00E94A27F8DE502
:10A1700090E1B0C48C010F5F1F4FE3E0F0E0EC0F03
:10A18000FD1FE00FF11F1082C8010E943C50892B77
:10A1900071F720E030E040E050E0C157DF4F6881C8
:10A1A000CF58D040627070E080E090E0A0E00E9464
:10A1B000289409F0C6C7C557DF4F2881CB58D04037
:10A1C000287030E040E050E060E070E080E090E037
:10A1D000A0E00E94289499F127E04AE250E06BE267
:10A1E00070E089E290E00E94BD628FED96E30E94EC
:10A1F0008364BC01990F880B990B0E94CC9520E0D9
:10A2000030E048EC52E40E9418959F938F937F931F
:10A210006F9388E397E09F938F931F9287E78F93C5
:10A22000CE01800F911F03969F938F930E947B9D79
:10A23000080F191F0FB6F894DEBF0FBECDBFC5576C
:10A24000DF4F2881CB58D040207130E040E050E013
:10A2500060E070E080E090E0A0E00E942894E9F1E6
:10A2600026E04AE250E06BE270E089E290E00E9472
:10A27000BD6281E090E00E944F118093C51482E599
:10A280009EE10E948364BC01990F880B990B0E9488
:10A29000CC9520E030E048EC52E40E9418959F9362
:10A2A0008F937F936F9382E497E09F938F931F9296
:10A2B00087E78F93C801029621E030E02C0F3D1F05
:10A2C000820F931F9F938F930E947B9D080F191FEE
:10A2D0000FB6F894DEBF0FBECDBF2E2D30E040E0AC
:10A2E00050E060E070E080E090E0A0E00E94289400
:10A2F00001F10E940B119F938F937F936F938DE4D5
:10A3000097E09F938F931F9287E78F93C8010296E0
:10A31000A1E0B0E0AC0FBD1F8A0F9B1F9F938F93EE
:10A320000E947B9D080F191F0FB6F894DEBF0FBE69
:10A33000CDBFC557DF4F2881CB58D040207430E0C7
:10A3400040E050E060E070E080E090E0A0E00E943B
:10A35000289431F180911B328F9380911A328F9320
:10A36000809119328F93809118328F938BE597E00B
:10A370009F938F931F9287E78F93C801029621E0E6
:10A3800030E02C0F3D1F820F931F9F938F930E94ED
:10A390007B9D080F191F0FB6F894DEBF0FBECDBF0F
:10A3A000C557DF4F2881CB58D040207830E040E0BF
:10A3B00050E060E070E080E090E0A0E00E9428942F
:10A3C00041F1F8948091C5369091C636A091C73678
:10A3D000B091C8367894BF93AF939F938F9389E6DB
:10A3E00097E09F938F931F9287E78F93C801029600
:10A3F000A1E0B0E0AC0FBD1F8A0F9B1F9F938F930E
:10A400000E947B9D080F191F0FB6F894DEBF0FBE88
:10A41000CDBF20E0C457DF4F3881CC58D0403170D9
:10A4200040E050E060E070E080E090E0A0E00E945A
:10A43000289409F098C620E0C457DF4F3881CC58E3
:10A44000D040327040E050E060E070E080E090E0AA
:10A45000A0E00E94289409F0E6C620E0C457DF4F30
:10A460003881CC58D040347040E050E060E070E07B
:10A4700080E090E0A0E00E94289409F005C720E069
:10A48000C457DF4F3881CC58D040387040E050E09E
:10A4900060E070E080E090E0A0E00E94289409F085
:10A4A00023C720E0C457DF4F3881CC58D0403071EB
:10A4B00040E050E060E070E080E090E0A0E00E94CA
:10A4C000289409F071C720E0C457DF4F3881CC5879
:10A4D000D040307240E050E060E070E080E090E01A
:10A4E000A0E00E94289409F08FC720E030E040E00F
:10A4F00050E0C157DF4F6881CF58D040647070E0A2
:10A5000080E090E0A0E00E94289409F0ABC720E032
:10A51000C956DF4F3881C759D04040E050E060E075
:10A5200070E080E090E0A0E00E94289411F00C948C
:10A53000A05A20E0C856DF4F3881C859D04040E0CB
:10A5400050E060E070E080E090E0A0E00E9428949D
:10A5500011F00C94CF5AC357DF4F5881CD58D040DB
:10A560005170E52E20E030E0452F50E060E070E0D3
:10A5700080E090E0A0E00E94289411F00C94FE5A34
:10A5800020E030E0C357DF4F4881CD58D0404270C3
:10A5900050E060E070E080E090E0A0E00E9428944D
:10A5A00011F00C94325B20E030E04F2D50E060E081
:10A5B00070E080E090E0A0E00E94289411F00C94FC
:10A5C000665B20E030E040E050E0C157DF4F68813B
:10A5D000CF58D040687070E080E090E0A0E00E942A
:10A5E000289411F00C94915B20E030E040E050E0C2
:10A5F000C157DF4F6881CF58D040607170E080E074
:10A6000090E0A0E00E94289411F00C94BD5B20E043
:10A6100030E040E050E060E0CE56DF4F7881C25934
:10A62000D040717080E090E0A0E00E94289411F08A
:10A630000C94E95B20E030E0C357DF4F4881CD58F0
:10A64000D040487050E060E070E080E090E0A0E032
:10A650000E94289411F00C940F5C20E030E0C35766
:10A66000DF4F4881CD58D040407150E060E070E04D
:10A6700080E090E0A0E00E94289411F00C94445CEB
:10A6800020E030E0C357DF4F4881CD58D0404072C2
:10A6900050E060E070E080E090E0A0E00E9428944C
:10A6A00011F00C94795C20E030E0C357DF4F488113
:10A6B000CD58D040407450E060E070E080E090E021
:10A6C000A0E00E94289411F00C94AE5CC357DF4FB9
:10A6D0005881CD58D0405078D52E20E030E0452F1D
:10A6E00050E060E070E080E090E0A0E00E942894FC
:10A6F00011F00C94E35CC257DF4F8881CE58D040F4
:10A700008170C82E20E030E040E0582F60E070E01B
:10A7100080E090E0A0E00E94289411F40C94F35F94
:10A720008091162E82FF06C021E046E061E083E0C2
:10A730000E942D1A20E030E04D2D50E060E070E0E6
:10A7400080E090E0A0E00E94289411F40C942B5D2E
:10A750008091162E82FF02C00C94F05C20E030E065
:10A7600040E0C257DF4F5881CE58D040527060E071
:10A7700070E080E090E0A0E00E94289411F00C943A
:10A78000605D20E030E040E0C257DF4F5881CE5896
:10A79000D040547060E070E080E090E0A0E00E9463
:10A7A000289411F00C94935D20E030E040E0C25713
:10A7B000DF4F5881CE58D040507160E070E080E0AB
:10A7C00090E0A0E00E94289411F00C94C65D20E077
:10A7D00030E040E0C257DF4F5881CE58D040507231
:10A7E00060E070E080E090E0A0E00E94289411F02A
:10A7F0000C94055E20E030E040E0C257DF4F588106
:10A80000CE58D040507460E070E080E090E0A0E06E
:10A810000E94289411F00C94445E20E030E040E067
:10A82000C257DF4F5881CE58D040587060E070E07A
:10A8300080E090E0A0E00E94289411F00C94835EE8
:10A8400020E030E040E050E0C157DF4F6881CF5852
:10A85000D040607270E080E090E0A0E00E94289418
:10A8600011F40C94B45E8091162E85FD02C00C94F8
:10A87000B45E81E00E9472696091EA367091EB36B5
:10A880008091EC369091ED360E94CC9520E030E03E
:10A8900048EC52E40E9418959F938F937F936F9397
:10A8A00081E099E09F938F931F9287E78F93C80170
:10A8B0000296A1E0B0E0AC0FBD1F8A0F9B1F9F93D3
:10A8C0008F930E947B9D080F191FC8010E943C5066
:10A8D0000FB6F894DEBF0FBECDBF892B09F047CC71
:10A8E000E1E020E030E040E050E0C157DF4F688118
:10A8F000CF58D040607470E080E090E0A0E00E940B
:10A90000289411F00C94B75E20E030E040E050E075
:10A91000C157DF4F6881CF58D040607870E080E049
:10A9200090E0A0E00E94289411F00C94FA5E20E0E0
:10A9300030E040E0C756DF4F5881C959D04060E051
:10A9400070E080E090E0A0E00E94289411F00C9468
:10A950003C5F20E030E04E2D50E060E070E080E0B1
:10A9600090E0A0E00E94289411F00C94785FC55705
:10A97000DF4F2881CB58D040C457DF4F3881CC58A7
:10A98000D040C357DF4F4881CD58D040C257DF4F2A
:10A990005881CE58D040C157DF4F6881CF58D04042
:10A9A000CE56DF4F7881C259D040CB56DF4F8881D9
:10A9B000C559D040CA56DF4F9881C659D040A0E053
:10A9C0000E94289411F00C94A55F8091640280612C
:10A9D00089838091A40B8A83FE01E00FF11F13820B
:10A9E0008091C9149091CA14A091CB14B091CC1449
:10A9F000A8014D5F5F4F7A0180FF0CC0FF924F931B
:10AA00008CE499E09F938F930E940F9D0F900F907D
:10AA10000F900F90B701CE0101960E9402818091A4
:10AA2000660282FF0AC025EC32E3A701BE016F5F18
:10AA30007F4F8EE692E00E949C658091C9149091B0
:10AA4000CA14A091CB14B091CC1482FD73980E94CB
:10AA5000837280EB9BE00E94BF7F809166029091A1
:10AA60006702A0916802B091690290FD02C00C9447
:10AA7000895F0F5F1F4F0E947C73E82E89E10E945F
:10AA80008D738091660290916702A0916802B091E7
:10AA9000690290FD02C00C94855F73988091A40BAD
:10AAA0008F5F8093A40B8A83B8016F5F7F4FCE01C5
:10AAB00001960E94028180EB9BE00E94BF7F40E0F4
:10AAC00050E065E880913316909134160E943E7AEA
:10AAD0008BE692E1CD56DF4FA881B981C359D040B2
:10AAE0008D939C931EC088E99BE00E940F78892B70
:10AAF000C1F00E9483728091660287FD2B9840E42A
:10AB000050E060E070E088E99BE00E94F17784E823
:10AB100092E1CD56DF4FE881F981C359D04091834E
:10AB2000808381E00C940360CD56DF4FA881B9810A
:10AB3000C359D0401D921C9283E00C940360B2E193
:10AB4000FB1669F080910A37F81211CBBAE006398A
:10AB50001B0709F00CCB89E097E00E944B9D809089
:10AB6000660290906702A0906802B090690291FC22
:10AB7000FECAF80180818130E1F50180F281E02D8B
:10AB80002081C557DF4F2883CB58D0403181C4572F
:10AB9000DF4F3883CC58D0404281C357DF4F4883C2
:10ABA000CD58D0405381C257DF4F5883CE58D04044
:10ABB0008481C157DF4F8883CF58D0409581CE56CE
:10ABC000DF4F9883C259D040A681CB56DF4FA88370
:10ABD000C559D040B781CA56DF4FB883C659D04057
:10ABE00060847184C057DF4F19821882C059D040E9
:10ABF00085C0823041F5F8010380F481E02DC05713
:10AC0000DF4FF983E883C059D040612C712CF1E00B
:10AC1000C557DF4FF883CB58D040C457DF4F188259
:10AC2000CC58D040C357DF4F1882CD58D04020E8D1
:10AC3000C257DF4F2883CE58D040C157DF4F18820C
:10AC4000CF58D0404CC0833039F1843009F08FCADE
:10AC5000612C712CC057DF4F19821882C059D04027
:10AC600035E0C557DF4F3883CB58D040C457DF4F4E
:10AC70001882CC58D040C357DF4F1882CD58D040EF
:10AC8000C257DF4F1882CE58D04042E0C157DF4F45
:10AC90004883CF58D04023C0612C712CC057DF4F60
:10ACA00019821882C059D04055E0C557DF4F5883EC
:10ACB000CB58D040C457DF4F1882CC58D040C35730
:10ACC000DF4F1882CD58D040C257DF4F1882CE5880
:10ACD000D04081E0C157DF4F8883CF58D040CE5657
:10ACE000DF4F1882C259D040CB56DF4F1882C5596A
:10ACF000D040CA56DF4F1882C659D04020908D02EE
:10AD000030908E0240908F0250909002C090183286
:10AD1000D0901932E0901A32F0901B322DEC3CECBE
:10AD20004CE45EE3C201B1010E943594A701960193
:10AD30000E94139518165CF0E894A0F880926602C1
:10AD400090926702A0926802B092690253C0A70174
:10AD50009601C201B1010E94F19618160CF04AC08A
:10AD60008091243290912532A0912632B0912732E1
:10AD70000196A11DB11D8093243290932532A0939A
:10AD80002632B0932732A0FCF2C96894A0F88092D2
:10AD9000660290926702A0926802B092690295E4FE
:10ADA000C557DF4F9883CB58D040A0E2C457DF4F40
:10ADB000A883CC58D040C357DF4F1882CD58D0401D
:10ADC000C257DF4F1882CE58D040B4E0C157DF4F92
:10ADD000B883CF58D040CE56DF4F1882C259D040EA
:10ADE000CB56DF4F1882C559D040CA56DF4F188264
:10ADF000C659D040C357DF4FE881CD58D040E470EA
:10AE0000FE2E20E030E04E2F50E060E070E080E069
:10AE100090E0A0E00E94289409F08C9AC557DF4F7B
:10AE2000F881CB58D040F072EF2E2F2F30E040E069
:10AE300050E060E070E080E090E0A0E00E942894A4
:10AE400011F00E940B11C457DF4F2881CC58D0401D
:10AE50002074C956DF4F2883C759D04020E0C95617
:10AE6000DF4F3881C759D04040E050E060E070E0EB
:10AE700080E090E0A0E00E94289411F00E9400265B
:10AE8000C457DF4F3881CC58D0403078C856DF4F98
:10AE90003883C859D04020E040E050E060E070E0E6
:10AEA00080E090E0A0E00E94289451F00E94A6105B
:10AEB0006093D2367093D3368093D4369093D53640
:10AEC000C557DF4F2881CB58D040217030E040E09B
:10AED00050E060E070E080E090E0A0E00E94289404
:10AEE000F1F080EE9DE19F938F9388E197E09F932F
:10AEF0008F931F9287E78F93CE0103969F938F9333
:10AF00000E947B9D6C010E943C500FB6F894DEBFFE
:10AF10000FBECDBF892B09F02AC9860102C000E00F
:10AF200010E0C557DF4F2881CB58D040227030E069
:10AF300040E050E060E070E080E090E0A0E00E943F
:10AF40002894D9F1C801029660E277E0A1E0B0E070
:10AF5000AC0FBD1F8A0F9B1F0E94699C0D5F1F4F86
:10AF60003FEDC32E36E3D32E47EE842E46E3942ED8
:10AF700052E9A52E53E0B52E67E7562EF6018191D2
:10AF80006F011F928F93BF92AF921F925F92C80181
:10AF9000029621E030E02C0F3D1F820F931F9F93FC
:10AFA0008F930E947B9D080F191F0FB6F894DEBF88
:10AFB0000FBECDBF8C149D0409F7C557DF4F288104
:10AFC000CB58D040247030E040E050E060E070E0CA
:10AFD00080E090E0A0E00E94289409F446C0C801F7
:10AFE000029664E277E0A1E0B0E0AC0FBD1F8A0FEB
:10AFF0009B1F0E94699C0C5F1F4F6E01BAE7CB0E2E
:10B00000D11C80E1F60111928A95E9F728E0A601AA
:10B0100068E980EB0E9453164601F8E08F0E911C00
:10B0200092E9A92E93E0B92E27E7522ED6018D91F1
:10B030006D011F928F93BF92AF921F925F92C801D2
:10B040000296E1E0F0E0EC0FFD1F8E0F9F1F9F9333
:10B050008F930E947B9D080F191F0FB6F894DEBFD7
:10B060000FBECDBFC814D90409F7C257DF4F3881CE
:10B07000CE58D0403078C756DF4F3883C959D040BA
:10B0800020E030E040E0C756DF4F5881C959D0403A
:10B0900060E070E080E090E0A0E00E942894E1F49D
:10B0A0008091C7149091C8149F938F9389E297E081
:10B0B0009F938F931F9287E78F93CE01800F911FED
:10B0C00003969F938F930E947B9D080F191F0FB6C5
:10B0D000F894DEBF0FBECDBF20E030E040E050E08E
:10B0E000C157DF4F6881CF58D040617070E080E079
:10B0F00090E0A0E00E94289409F44BC8E3E0F0E05F
:10B10000EC0FFD1FE00FF11F80E28083DE01A00F36
:10B11000B11FBD016C5F7F4FE5E4F2E305541243BC
:10B120009F012D5F3F4FC8018E0F9F1F43813196B6
:10B13000442309F41FC8D9018C91DB018D93BD0113
:10B14000EFCFCE01800F911F60E377E003960E945E
:10B15000699C095F1F4FC8010E943C50892B11F068
:10B160000C94B75028C86114710409F464C9F894A8
:10B170002090C5363090C6364090C7365090C836BD
:10B18000789480914A1E90914B1EA0914C1EB091D4
:10B190004D1EA2019101281B390B4A0B5B0BCA0102
:10B1A000B9010E94CA954B015C01B30180E090E0B7
:10B1B0000E94CA959B01AC01C501B4010E9418957B
:10B1C000B62EC72ED82EE92E9F938F937F936F9321
:10B1D00084E797E09F938F931F9287E78F93CE0129
:10B1E000800F911F03969F938F930E947B9D080F62
:10B1F000191F8B2D9C2DAD2DBE2D8093D73690938E
:10B20000D836A093D936B093DA3620924A1E3092BF
:10B210004B1E40924C1E50924D1E0FB6F894DEBF4E
:10B220000FBECDBF08C96114710409F416C9F894A2
:10B230008091211E9091221EA091231EB091241E68
:10B2400078949F938F9380916D028F9380916C027D
:10B250008F9381E897E09F938F931F9287E78F9357
:10B26000C8010296A1E0B0E0AC0FBD1F8A0F9B1F82
:10B270009F938F930E947B9D080F191F0FB6F89420
:10B28000DEBF0FBECDBFE9C8F8948091C93690915A
:10B29000CA36A091CB36B091CC367894BF93AF9399
:10B2A0009F938F9381E997E09F938F931F9287E7F6
:10B2B0008F93C801029621E030E02C0F3D1F820FD2
:10B2C000931F9F938F930E947B9D080F191FC801A6
:10B2D0000E943C500FB6F894DEBF0FBECDBF892B45
:10B2E00011F00C94B750CBC86114710409F4D9C89B
:10B2F000F8942090C9363090CA364090CB365090A2
:10B30000CC36789480914E1E90914F1EA091501E85
:10B31000B091511EA2019101281B390B4A0B5B0B06
:10B32000CA01B9010E94CA954B015C01B30180E0DA
:10B3300090E00E94CA959B01AC01C501B4010E9436
:10B340001895B62EC72ED82EE92E9F938F937F93F4
:10B350006F938CE997E09F938F931F9287E78F936A
:10B36000CE01800F911F03969F938F930E947B9D28
:10B37000080F191F8B2D9C2DAD2DBE2D8093DB3614
:10B380009093DC36A093DD36B093DE3620924E1ECD
:10B3900030924F1E4092501E5092511E0FB6F8949C
:10B3A000DEBF0FBECDBF7DC8672809F48CC8F894F6
:10B3B0008091251E9091261EA091271EB091281ED7
:10B3C00078949F938F9380916B028F9380916A0200
:10B3D0008F9389EA97E09F938F931F9287E78F93CC
:10B3E000C8010296A1E0B0E0AC0FBD1F8A0F9B1F01
:10B3F0009F938F930E947B9D080F191F0FB6F8949F
:10B40000DEBF0FBECDBF5FC880911C3290911D3250
:10B41000A0911E32B0911F32BF93AF939F938F9331
:10B4200089EB97E09F938F931F9287E78F93C801D3
:10B43000029621E030E02C0F3D1F820F931F9F9357
:10B440008F930E947B9D080F191FC8010E943C50DA
:10B450000FB6F894DEBF0FBECDBF892B11F00C9450
:10B46000B75043C8809127328F93809126328F93B3
:10B47000809125328F93809124328F938091233253
:10B480008F93809122328F93809121328F9380917C
:10B4900020328F9384EC97E09F938F931F9287E7DE
:10B4A000E82EEF92C8010296A1E0B0E0AC0FBD1FFC
:10B4B0008A0F9B1F9F938F930E947B9D080F191FDC
:10B4C000C8010E943C500FB6F894DEBF0FBECDBF3E
:10B4D000892B11F00C94B7508091162E9091172E55
:10B4E00093FF15C880912B328F9380912A328F93CE
:10B4F000809129328F93809128328F9388EE97E044
:10B500009F938F931F92EF92C801029621E030E043
:10B510002C0F3D1F820F931F9F938F930E947B9D43
:10B52000080F191FC8010E943C500FB6F894DEBFE7
:10B530000FBECDBF892B11F00C94B7500C948752DD
:10B5400080910D2A8F9380910C2A8F9380910B2AE2
:10B550008F9380910A2A8F938AEF97E09F938F931E
:10B560001F9287E78F93C8010296A1E0B0E0AC0F6D
:10B57000BD1F8A0F9B1F9F938F930E947B9D080F77
:10B58000191FC8010E943C500FB6F894DEBF0FBED1
:10B59000CDBF892B11F00C94B7500C949952809127
:10B5A000D5368F938091D4368F938091D3368F93F5
:10B5B0008091D2368F9385E098E09F938F931F926E
:10B5C00087E78F93C801029621E030E02C0F3D1FE2
:10B5D000820F931F9F938F930E947B9D080F191FCB
:10B5E000C8010E943C500FB6F894DEBF0FBECDBF1D
:10B5F000892B11F00C94B7500C94AB5281E00E944F
:10B600005810209185023091860240918702509116
:10B6100088020E94C4979F938F937F936F9382E1D8
:10B6200098E09F938F931F9287E78F93C8010296AC
:10B63000A1E0B0E0AC0FBD1F8A0F9B1F9F938F93BB
:10B640000E947B9D080F191FC8010E943C500FB635
:10B65000F894DEBF0FBECDBF892B11F00C94B7500C
:10B660000C94C05282E00E945810209181023091C7
:10B67000820240918302509184020E94C4979F935A
:10B680008F937F936F938FE198E09F938F931F9297
:10B6900087E78F93C801029621E030E02C0F3D1F11
:10B6A000820F931F9F938F930E947B9D080F191FFA
:10B6B000C8010E943C500FB6F894DEBF0FBECDBF4C
:10B6C000892B11F00C94B7500C94D35283E00E9454
:10B6D00058109F938F937F936F938CE298E09F9382
:10B6E0008F931F9287E78F93C8010296A1E0B0E085
:10B6F000AC0FBD1F8A0F9B1F9F938F930E947B9D52
:10B70000080F191F8C98C8010E943C500FB6F8947E
:10B71000DEBF0FBECDBF892B11F00C94B7500C9437
:10B72000E152299903C08FE595E002C083E99AE0D0
:10B730009F938F9389E398E09F938F931F9287E75E
:10B740008F93C801029621E030E02C0F3D1F820F3D
:10B75000931F9F938F930E947B9D080F191FC80111
:10B760000E943C500FB6F894DEBF0FBECDBF892BB0
:10B7700011F00C94B7500C94F4522A9903C08FE541
:10B7800095E002C083E99AE09F938F9381E498E06B
:10B790009F938F931F9287E78F93C8010296A1E032
:10B7A000B0E0AC0FBD1F8A0F9B1F9F938F930E9429
:10B7B0007B9D080F191FC8010E943C500FB6F894DA
:10B7C000DEBF0FBECDBF892B11F00C94B7500C9487
:10B7D00007538EB31F928F9389E498E09F938F93C2
:10B7E0001F9287E78F93C801029621E030E02C0F6B
:10B7F0003D1F820F931F9F938F930E947B9D080F85
:10B80000191FC8010E943C500FB6F894DEBF0FBE4E
:10B81000CDBF892B11F00C94B7500C941A53809122
:10B82000162E9091172E92FD02C00C942D5321E0FC
:10B8300042E161E080ED0E94D9669F938F937F93F0
:10B840006F9388E598E09F938F931F9287E78F937C
:10B85000C8010296A1E0B0E0AC0FBD1F8A0F9B1F8C
:10B860009F938F930E947B9D080F191FC8010E9410
:10B870003C500FB6F894DEBF0FBECDBF892B11F040
:10B880000C94B7500C942D538091162E9091172E36
:10B8900092FD02C00C94405321E042E162E080ED51
:10B8A0000E94D9669F938F937F936F9386E698E06B
:10B8B0009F938F931F9287E78F93C801029621E091
:10B8C00030E02C0F3D1F820F931F9F938F930E9498
:10B8D0007B9D080F191FC8010E943C500FB6F894B9
:10B8E000DEBF0FBECDBF892B11F00C94B7500C9466
:10B8F00040538091162E9091172E92FD02C00C9409
:10B90000535321E042E163E080ED0E94D9669F93AA
:10B910008F937F936F9384E798E09F938F931F9209
:10B9200087E78F93C8010296A1E0B0E0AC0FBD1F7E
:10B930008A0F9B1F9F938F930E947B9D080F191F57
:10B94000C8010E943C500FB6F894DEBF0FBECDBFB9
:10B95000892B11F00C94B7500C9453538091162EF0
:10B960009091172E92FD02C00C94665321E042E1A3
:10B9700064E080ED0E94D9669F938F937F936F93CD
:10B9800082E898E09F938F931F9287E78F93C80177
:10B99000029621E030E02C0F3D1F820F931F9F93F2
:10B9A0008F930E947B9D080F191FC8010E943C5075
:10B9B0000FB6F894DEBF0FBECDBF892B11F00C94EB
:10B9C000B7500C9466538091162E82FD02C00C94E1
:10B9D0007B5346E061E083E00E942D1A0C947B5378
:10B9E0008091F91E8F938091F81E8F938091F71E9E
:10B9F0008F938091F61E8F9380E998E09F938F93A9
:10BA00001F9287E78F93C8010296A1E0B0E0AC0FC8
:10BA1000BD1F8A0F9B1F9F938F930E947B9D080FD2
:10BA2000191FC8010E943C500FB6F894DEBF0FBE2C
:10BA3000CDBF892B11F00C94B75020E030E040E0EE
:10BA40005C2D60E070E080E090E0A0E00E9428942F
:10BA500011F40C94AE538091162E82FD02C00C940A
:10BA6000AE538091FD1E8F938091FC1E8F93809129
:10BA7000FB1E8F938091FA1E8F9388E998E09F9325
:10BA80008F931F9287E78F93C801029621E030E0E1
:10BA90002C0F3D1F820F931F9F938F930E947B9DBE
:10BAA000080F191FC8010E943C500FB6F894DEBF62
:10BAB0000FBECDBF892B11F00C94B7500C94AE5330
:10BAC0008091162E9091172E93FD02C00C94C153B5
:10BAD00080E090E00E9478259F938F937F936F93EF
:10BAE00083EA98E09F938F931F9287E78F93C80113
:10BAF0000296A1E0B0E0AC0FBD1F8A0F9B1F9F9381
:10BB00008F930E947B9D080F191FC8010E943C5013
:10BB10000FB6F894DEBF0FBECDBF892B11F00C9489
:10BB2000B7500C94C1538091162E9091172E93FD0F
:10BB300002C00C94D45381E090E00E9478259F933A
:10BB40008F937F936F9383EB98E09F938F931F92D4
:10BB500087E78F93C801029621E030E02C0F3D1F4C
:10BB6000820F931F9F938F930E947B9D080F191F35
:10BB7000C8010E943C500FB6F894DEBF0FBECDBF87
:10BB8000892B11F00C94B7500C94D4538091162E3D
:10BB90009091172E93FD02C00C94E75381E090E042
:10BBA0000E9478254B015C0180E090E00E9478259E
:10BBB0009B01AC01C501B4010E9473239F938F9335
:10BBC0007F936F9384EC98E09F938F931F9287E706
:10BBD0008F93C8010296A1E0B0E0AC0FBD1F8A0FA1
:10BBE0009B1F9F938F930E947B9D080F191FC80175
:10BBF0000E943C500FB6F894DEBF0FBECDBF892B1C
:10BC000011F00C94B7500C94E7538091162E90913C
:10BC1000172E93FD02C00C94FA5381E090E00E942D
:10BC200078254B015C0180E090E00E9478259B0123
:10BC3000AC01C501B4010E94D4239F938F937F93DD
:10BC40006F938FEC98E09F938F931F9287E78F936A
:10BC5000C801029621E030E02C0F3D1F820F931F98
:10BC60009F938F930E947B9D080F191FC8010E940C
:10BC70003C500FB6F894DEBF0FBECDBF892B11F03C
:10BC80000C94B7500C94FA538091162E9091172E65
:10BC900093FD02C00C940D5481E090E00E94782541
:10BCA0004B015C0180E090E00E9478259B01AC0193
:10BCB000C501B4010E9439249F938F937F936F93A2
:10BCC0008DED98E09F938F931F9287E78F93C80124
:10BCD0000296A1E0B0E0AC0FBD1F8A0F9B1F9F939F
:10BCE0008F930E947B9D080F191FC8010E943C5032
:10BCF0000FB6F894DEBF0FBECDBF892B11F00C94A8
:10BD0000B7500C940D548091162E9091172E94FDDF
:10BD100002C00C9420540E94921E9F938F937F9395
:10BD20006F9380EF98E09F938F931F9287E78F9395
:10BD3000C801029621E030E02C0F3D1F820F931FB7
:10BD40009F938F930E947B9D080F191FC8010E942B
:10BD50003C500FB6F894DEBF0FBECDBF892B11F05B
:10BD60000C94B7500C942054E0E00C9471548091E2
:10BD7000162E85FD02C00C948454E11103C081E0AD
:10BD80000E9472696091EE367091EF368091F036C4
:10BD90009091F1360E94CA9520E030E040E85AE3E5
:10BDA0000E94C4979F938F937F936F9382E199E052
:10BDB0009F938F931F9287E78F93C801029621E08C
:10BDC00030E02C0F3D1F820F931F9F938F930E9493
:10BDD0007B9D080F191FC8010E943C500FB6F894B4
:10BDE000DEBF0FBECDBF892B11F00C94B750E1E040
:10BDF0000C9484548091162E85FD02C00C949754A7
:10BE0000E11103C081E00E9472696091F236709185
:10BE1000F3368091F4369091F5360E94CA9520E071
:10BE200030E040E85BE30E94C4979F938F937F9339
:10BE30006F9384E299E09F938F931F9287E78F938C
:10BE4000C8010296A1E0B0E0AC0FBD1F8A0F9B1F96
:10BE50009F938F930E947B9D080F191FC8010E941A
:10BE60003C500FB6F894DEBF0FBECDBF892B11F04A
:10BE70000C94B7500C949754C057DF4FA881B981E8
:10BE8000C059D04016968C9116971F928F93159695
:10BE90008C9115971F928F9313968C9113971F92E5
:10BEA0008F9312968C911F928F9385E399E09F93C5
:10BEB0008F931F9287E78F93C8010296E1E0F0E02D
:10BEC000EC0FFD1F8E0F9F1F9F938F930E947B9DF2
:10BED000080F191FC8010E943C500FB6F894DEBF2E
:10BEE0000FBECDBF892B11F00C94B7500C94A95400
:10BEF000779A8091C9149091CA14A091CB14B091F3
:10BF0000CC1492FF22C0749A20C08E2D0E948D7393
:10BF1000739A8091C7149091C814892B11F00E94D4
:10BF2000BA718091A40B8F5F8093A40B8091C91488
:10BF30009091CA14A091CB14B091CC1482FD02C090
:10BF40000C94B750739A0C94B7508091C914909187
:10BF5000CA14A091CB14B091CC1482FD0CC0809176
:10BF6000660280FD08C081FD02C00C94E5541D9955
:10BF700002C00C94E55440E050E060E070E0CE0177
:10BF800001960E94C30E8091FF1E90E02091BF1485
:10BF90003091C0148217930710F40C94E55440E0DC
:10BFA00050E062E180E192E00E943E7A0C94E55418
:10BFB000E5E8FE120C94915500E010E00C94415518
:10BFC00088E99BE00E940F78892B11F40C9491551D
:10BFD0000E94BA718091660287FD02C00C94B7502E
:10BFE0002B9A0C94B75020E030E04D2D50E060E0EB
:10BFF00070E080E090E0A0E00E94289411F00C94A2
:10C00000A8530C94AE53C756DF4F0FB6F894DEBF5B
:10C010000FBECDBFDF91CF911F910F91FF90EF9099
:10C02000DF90CF90BF90AF909F908F907F906F9058
:10C030005F904F903F902F9008950C94A57E4F9263
:10C040005F926F927F929F92AF92BF92CF92DF9258
:10C05000EF92FF920F931F93CF93DF93CDB7DEB78D
:10C0600060970FB6F894DEBF0FBECDBF5B010E9494
:10C070007C73E82FF0E0EE0FFF1FED5EF14E808144
:10C0800091810196918380838091C9149091CA1403
:10C09000A091CB14B091CC1481FD749840906602AD
:10C0A0005090670260906802709069020E94598007
:10C0B0006C01FC018081982F92959F70913099F4CA
:10C0C0008F7051F48091F71D9091F81D0196909317
:10C0D000F81D8093F71D3EC1B50181E499E30E94EC
:10C0E0007681892B51F08091F51D9091F61D019676
:10C0F0009093F61D8093F51D2DC1D301C2013EE042
:10C10000B695A795979587953A95D1F7F82FF17041
:10C110009F2E8BEB9BE00E94157B7C01892B09F401
:10C120004BC0B501C70102960E947681892B09F4A4
:10C130003FC0870122E73EE040E054E660E070E067
:10C14000C7010F960E94BE78F6019181F7018481A4
:10C15000981321C082858F5F82878091F31D909113
:10C16000F41D01969093F41D8093F31D84E00E94CA
:10C170004281F701208530E02817390708F07AC19D
:10C1800084E00E944281F7018087F60180818F70F0
:10C19000F7018187DFC0F701128684E00E944281A7
:10C1A000F7018087F60180818F70F701818763C175
:10C1B000C7010E94767BB1CF88E092E00E946B7C41
:10C1C0007C01892B09F4C6C0B501C70102960E9403
:10C1D0006F81F60181818150F701848380E091E0D5
:10C1E000A0E0B0E083879487A587B687128684E0B5
:10C1F0000E944281F7018087F60180818F70F701EC
:10C200008187B7018BEB9BE00E94507B870122E77F
:10C210003EE040E054E660E070E0C7010F960E9407
:10C22000BE7811E0F6018181F7018483F6018081F7
:10C230008F70F701878384E00E944281F701858334
:10C2400083E00E944281F701868387818F3009F065
:10C2500010E0F6014180F7018481481A512C612CCD
:10C26000712C86E0440C551C661C771C8A95D1F70E
:10C270002385348545855685A0ECB0E00E948792E1
:10C28000BB27A92F982F872F480E591E6A1E7B1E89
:10C290004386548665867686A501B701C6010E944D
:10C2A000C30E8091FF1E90E02091BF143091C01406
:10C2B0008217930738F040E050E062E180E192E0BD
:10C2C0000E943E7A8091BF149091C014029708F4A6
:10C2D0004DC08091162E9091172E91FF2AC00E947A
:10C2E0002866C60105960E94F465F60181811F92B9
:10C2F0008F93F70186811F928F9385811F928F9371
:10C300008DE599E09F938F931F9280E18F93CE01EB
:10C3100001965C019F938F930E947B9D82E00E9417
:10C320000E66C5010E94F4650FB6F894DEBF0FBE1D
:10C33000CDBF8091660290916702A0916802B09192
:10C34000690297FD4DC08091BF149091C01402976F
:10C3500008F47AC08091C9149091CA14A091CB14AA
:10C36000B091CC1481FF89C0749A87C08091660215
:10C3700090916702A0916802B091690296FFA9CFDF
:10C38000992009F4A6CFF6019081892F8F70823011
:10C39000E8F0907F8150892B808380EB9BE00E94A6
:10C3A0001D608091F11D9091F21D01969093F21DF8
:10C3B0008093F11D8091C9149091CA14A091CB145F
:10C3C000B091CC1496FF85CF739883CF8091F71DE1
:10C3D0009091F81D01969093F81D8093F71D79CFE9
:10C3E00080EE9DE12091E01D222309F4ACCF9F93C4
:10C3F0008F9380E799E09F938F93CE0101963C0144
:10C400009F938F930E94B89D5C01B301C601029671
:10C410000E948A9C0F900F900F900F900F900F909A
:10C42000009709F490CFEFEFAE1ABE0A8A0D9B1D5C
:10C43000AC010196FA0120812032D1F362E18AE158
:10C4400092E00E943E7A7FCF112309F483CF82E0ED
:10C45000809331321092333210923232F092353270
:10C46000E092343241E352E362E182E492E00E94DE
:10C470003E7A70CF912C10E0D5CE60960FB6F8942E
:10C48000DEBF0FBECDBFDF91CF911F910F91FF9007
:10C49000EF90DF90CF90BF90AF909F907F906F9084
:10C4A0005F904F9008958115910511F00197F1F774
:10C4B0000895E091FE36F091FF3690818091FD362F
:10C4C00089230895E091FB36F091FC3690818091AC
:10C4D000FD36892B8083E0910037F0910137908100
:10C4E0008091FD36892B808308951F93CF93DF932E
:10C4F000E091FB36F091FC3690818091FD3680957D
:10C5000089238083E0910037F091013790818091F9
:10C51000FD36892B80838FE897E00E9453621FB716
:10C52000F894E0910037F091013790818091FD36C9
:10C5300080958923808389E091E00E945362E09195
:10C54000FE36F091FF36D081C091FD361FBF789442
:10C5500085E896E00E945362E091FE36F091FF3646
:10C5600090818091FD36892319F08D2F8C2301C095
:10C5700081E0DF91CF911F9108955093013740934F
:10C5800000377093FC366093FB369093FF368093B0
:10C59000FE3681E001C0880F2A95EAF78093FD36C8
:10C5A0000C947562CF93DF93C82FDFB7F894E091B6
:10C5B0000037F091013790818091FD36892B80837F
:10C5C00087E090E00E945362CC2351F0E091003765
:10C5D000F091013790818091FD3680958923808389
:10C5E00084E390E00E945362E091FE36F091FF36C2
:10C5F00090818091FD36892309F4C0E085EB90E0BD
:10C600000E945362E0910037F09101379081809150
:10C61000FD36809589238083DFBF88E790E00E9404
:10C6200053628C2FDF91CF910895CF93DF93C82F62
:10C63000D8E08C2F81700E94D262C6958111C068AB
:10C64000D150B9F78C2FDF91CF9108958FEF0C94D3
:10C650001563DF92EF92FF920F931F93CF93DF93B7
:10C66000E82E8B010E947562811135C080EF0E9417
:10C670001563D0E0C0E488EFD82EDC0E81E00E9484
:10C68000D262F82E81E00E94D262882319F0FF2046
:10C6900071F023C0F1100BC0CE1530F0F80180818D
:10C6A00080FF05C0CE1519F0DC2FFF24F3948F2DE9
:10C6B0000E94D262F80180818695FF2011F0806887
:10C6C000F8018083C150CD11D9CF0F5F1F4FC11129
:10C6D000D2CF8D2F03C08FEF01C08EEFDF91CF91AE
:10C6E0001F910F91FF90EF90DF900895EF92FF92CE
:10C6F0001F93CF93DF93182FEB010E947562209751
:10C7000071F085E50E9415637E0188E0E80EF11C5A
:10C7100089910E941563CE15DF05D1F703C08CEC1B
:10C720000E941563812FDF91CF911F91FF90EF90B1
:10C730000C9415630F931F93CF93DF93DB01ED915F
:10C74000FC911197803161F4EE7F63E0EE0FFF1FE3
:10C750006A95E1F716969C911697E91BF1093C96AC
:10C76000F7FF07C091E0EA019883F195E195F1099F
:10C7700002C0EA011882883279F414968C91982FBD
:10C780009076903649F086FF02C0EE7F05C085FFA7
:10C7900002C0EC7F01C0E87FCF0144E09695879509
:10C7A0004A95E1F7D9018C93EF70E801E88380E0C6
:10C7B000DF91CF911F910F9108950F931F93CF9306
:10C7C000DF93EC018B01B80188810E942963888383
:10C7D00081508D3F30F4F8018081883211F0803132
:10C7E00091F7DF91CF911F910F910895CF93DF9330
:10C7F000EC010E947562BE0184EB0E94766381E0C9
:10C800000E94D262C82F0E94756281E0C11101C0EE
:10C8100080E0DF91CF9108950F931F93CF93C82F9E
:10C820008B010E9475620E945962882349F0B80109
:10C8300084E40E947663C13029F00E94626202C0E3
:10C8400082E001C080E0CF911F910F9108954F9237
:10C850005F926F927F928F929F92AF92BF92CF9290
:10C86000DF92EF92FF920F931F93CF93DF93CDB799
:10C87000DEB729970FB6F894DEBF0FBECDBF6C01AF
:10C880003B015A0189010E947562B6018EEB0E943C
:10C890007663CE0101967C014E019AE0890E911CCF
:10C8A00027010E942663F70181937F01E815F905AE
:10C8B000C1F769E070E0C2010E94BD84F82E8111C9
:10C8C00008C09501A301B201F60180810E949A631C
:10C8D00002C083E0F82E8F2D29960FB6F894DEBFA4
:10C8E0000FBECDBFDF91CF911F910F91FF90EF90C1
:10C8F000DF90CF90BF90AF909F908F907F906F9080
:10C900005F904F900895EF92FF920F931F93CF93F4
:10C91000DF93CDB7DEB72B970FB6F894DEBF0FBE0F
:10C92000CDBF182F092F682F792F88E0810F0E9423
:10C930000C64882319F084E391E244C06CE872E847
:10C940008EE190E00E94EF647E0189E0E80EF11C28
:10C950009701AE01465F5F4FBE01655F7F4F812F3C
:10C96000902F0E9427648111E6CF88E0EFEEF2E07D
:10C97000DE01119601900D928A95E1F7298541E734
:10C9800052E0249FC001259F900D112464E670E0C1
:10C990000E940C928A8594E6899F600D711D112476
:10C9A000FE0131968191281303C06F5F7F4F03C052
:10C9B000EE15FF05B9F78B85882319F07195619500
:10C9C0007109CB012B960FB6F894DEBF0FBECDBF19
:10C9D000DF91CF911F910F91FF90EF900895DC01AF
:10C9E000CB0181159105A105B10529F08150904039
:10C9F000A040B040D9F708959B01AC011092B90056
:10CA000060E074E284EF90E00E942092DA01C901B4
:10CA10004097A109B109B695A795979587958093F9
:10CA2000B800089594EA9093BC0040EA56E861E0AB
:10CA300070E09091BC0097FD07C041505109610919
:10CA40007109B9F781E008959091B900987F983005
:10CA500011F09031B9F78093BB0084E88093BC005B
:10CA600080EA96E8A1E0B0E02091BC0027FD05C077
:10CA70000197A109B109C1F7E5CF8091B900887F7D
:10CA8000883111F08034F1F680E0089524EA34E82A
:10CA900044E92093BC009091BC0097FFFCCF90919B
:10CAA000B900987F983011F0903199F78093BB00CE
:10CAB0003093BC009091BC0097FFFCCF9091B900DF
:10CAC000987F903211F0983539F44093BC009091E2
:10CAD000BC0094FDFCCFDDCF08950C94126584E971
:10CAE0008093BC008091BC0084FDFCCF08958093AE
:10CAF000BB0084E88093BC008091BC0087FFFCCF22
:10CB00009091B900987F81E0983209F480E008950F
:10CB100084EC8093BC008091BC0087FFFCCF8091A7
:10CB2000BB00089584E88093BC008091BC0087FF1F
:10CB3000FCCF8091BB000895CF93DF93FC017096EA
:10CB4000EC01A991CE01A0933F01EC17FD07C1F7BD
:10CB500080913C018F7D80933C0180913C01877FD7
:10CB600080933C01DB015096FB01819180933E0153
:10CB7000EA17FB07D1F780913C01806880933C0164
:10CB800080913D0180FFFCCF4051510980913C01D3
:10CB9000806280933C0180913C01877F80933C01BF
:10CBA000141615069CF4FB01819180933E01AE178B
:10CBB000BF07D1F780913C01806880933C01809150
:10CBC0003D0180FFFCCF40515109EACFF901C90175
:10CBD000409620913E0121938E179F07D1F781E067
:10CBE00090E0DF91CF9108950F931F93CF93DF9340
:10CBF000EC018CE70E9446658CE70E9477658E0108
:10CC0000005F1F4F89910E947765C017D107D1F748
:10CC1000DF91CF911F910F910C946F65813019F4C2
:10CC200040E050E002C040EC50E060E070E08CE793
:10CC300090E00C944316813019F44EE050E002C0AD
:10CC400048E050E060E070E08CE790E00C94431620
:10CC500041E050E060E070E08CE790E00E94431615
:10CC600064ED74E180E090E00C94EF6448E350E000
:10CC700060E070E08CE790E00E94431649E350E0EA
:10CC800060E070E08CE790E00E94431644E150E0E1
:10CC900060E070E08CE790E00E94431648E750E0C7
:10CCA00060E070E08CE790E00E9443164EE550E0B3
:10CCB00060E070E08CE790E00E9443164DE650E0A3
:10CCC00060E070E08CE790E00E94431668E374E354
:10CCD0008CE090E00E94EF644CE050E060E070E097
:10CCE0008CE790E00E94431641E050E060E070E085
:10CCF0008CE790E00E94431646E050E060E070E070
:10CD00008CE790E00E94431664ED74E180E090E0CF
:10CD10000C94EF64CF93DF93CDB7DEB7A2970FB635
:10CD2000F894DEBF0FBECDBF81E1EFEFF9E0DE0189
:10CD3000529601900D928A95E1F781E1E0E1FAE0E7
:10CD4000DE01119601900D928A95E1F70E943666F8
:10CD5000CE0142960E94F46582E00E940E6664ED68
:10CD600074E180E090E00E94EF64CE0101960E94A1
:10CD7000F46560E27CE581E590E00E94EF6480E08C
:10CD80000E941B6660E27CE581E590E00E94EF6412
:10CD90004EE050E060E070E08CE790E00E944316C7
:10CDA000A2960FB6F894DEBF0FBECDBFDF91CF9134
:10CDB0000895CF92DF92EF92FF920F931F93CF933C
:10CDC000DF9300D0CDB7DEB7042F122F213031F022
:10CDD000223031F0243031F0283031F090E005C0BD
:10CDE00091E003C092E001C093E0E82FF0E08160A1
:10CDF000F82E0C3009F4E1C00E3011F49460DDC05F
:10CE0000003111F49860D9C0023109F0D6C0292F41
:10CE10002C60613009F4B6C0623011F4206207C0A2
:10CE2000633011F4206403C0643009F42066206884
:10CE3000622F70E023E030E0AE014F5F5F4FCF0123
:10CE40000E94531662E174E380E090E00E94EF6478
:10CE50008F2D0E9412650E94886589830E948865D3
:10CE60008A83023119F40E9488658B830E94886549
:10CE700087FDF1CF0E9492650E946F6562E174E3C5
:10CE800080E090E00E94EF648F2D0E9412650E9466
:10CE9000886589830E9488658A83023119F40E941B
:10CEA00092658B830E9492650E946F6569812A81D9
:10CEB000023139F5862F90E0A0E0B0E04B8130E000
:10CEC000322F2227DC0199278827820F931FA11D6B
:10CED000B11D61FF09C0840F911DA11DB11DBC01D1
:10CEE000CD018C6F9F6F06C0BC01CD01640F711D19
:10CEF000811D911D0E94CC9520E83FEF4FEF57E434
:10CF00001FC070E0762F6627620F711D072E000C80
:10CF1000880B990B0E94CC950C3029F420E030EE60
:10CF20004FEF54E40DC00E3029F420E038EF4FEFFE
:10CF300055E406C0003131F420E03EEF4FEF56E4F7
:10CF40000E9418952FE632E143E050E40E94C49716
:10CF50006B017C01612F70E080E090E00E94CC9535
:10CF60009B01AC01C701B6010E9418950F900F906C
:10CF70000F90DF91CF911F910F91FF90EF90DF9075
:10CF8000CF9008959C68692F70E023E030E0AE01F7
:10CF90004F5F5F4FCF010E94531662E174E380E060
:10CFA00090E00E94EF648F2D0E9412650E948865B8
:10CFB00089830E9488658A8356CF6130D9F490684E
:10CFC000692F70E023E030E0AE014F5F5F4FCF018B
:10CFD0000E94531662E174E380E090E00E94EF64E7
:10CFE0008F2D0E9412650E94886589830E94886542
:10CFF0008A833CCF292F10CF8F929F92AF92BF92FE
:10D00000CF92DF92EF92FF920F931F93EDECF4E13A
:10D010000081118120E030E06B017C0144E0F59457
:10D02000E794D794C7944A95D1F7C01AD10AE20A77
:10D03000F30ADC01CB0153E0B595A7959795879549
:10D040005A95D1F7000F111F221F331F4C015D01AC
:10D05000801A910AA20AB30AA5019401A281B381A0
:10D060000E9492924B015C017BE0B594A794979447
:10D0700087947A95D1F7A7019601C701B6010E945E
:10D08000DC919B01AC01ACE0559547953795279510
:10D09000AA95D1F7A481B5810E949292DC01CB01BF
:10D0A0001EE0B595A795979587951A95D1F7A50197
:10D0B0009401280F391F4A1F5B1F21A332A343A3EA
:10D0C00054A3A5E0B0E00E948792DC01CB01805818
:10D0D0009F4FAF4FBF4F692F7A2F8B2F992787FD17
:10D0E0009A951F910F91FF90EF90DF90CF90BF9096
:10D0F000AF909F908F900895CF92DF92EF92FF9222
:10D100001F93CF93DF93CDB7DEB76A970FB6F8942E
:10D11000DEBF0FBECDBF182F21E030E0CE0101965B
:10D120007C01AC0160ED70E08EEE90E00E94531641
:10D130008981803609F0C8C046EB50E060EE70E0AF
:10D140008EEE90E00E9443163CE2C32EDD24D39481
:10D1500088EE93E00E94606F91E0C91AD108C1F790
:10D160008AE1F70111928A95E9F72AE130E0A701F7
:10D1700068E870E08EEE90E00E94531689819A81F3
:10D180009093CE148093CD148C8190E0982F8827B3
:10D190002B81822B9093D0148093CF148E8190E0BA
:10D1A000982F88272D81822B9093D2148093D114AD
:10D1B0008F8198859093D4148093D3148A8590E0BE
:10D1C000982F88272985822B9093D6148093D51485
:10D1D0008C8590E0982F88272B85822B9093D814EC
:10D1E0008093D7148E8590E0982F88272D85822BE9
:10D1F0009093DA148093D914888990E0982F882727
:10D200002F85822B9093DC148093DB148A8990E025
:10D21000982F88272989822B9093DE148093DD1420
:10D220008C8990E0982F88272B89822B9093E0148B
:10D230008093DF148E8990E0982F88272D89822B88
:10D240009093E2148093E114888D90E0982F8827C2
:10D250002F89822B9093E4148093E3148A8D80931A
:10D26000E51428E030E0A70161EE70E08EEE90E07A
:10D270000E9453168A8190E0982F88272981822B5B
:10D280009093E7148093E6148B818093E8148D814A
:10D290002C81F0E12F9F90011124982F9F70292B52
:10D2A0003093EA142093E9142E812F7030E1839F8C
:10D2B000C0011124822B9093EC148093EB148F8186
:10D2C0008093ED141093F2146A960FB6F894DEBFB3
:10D2D0000FBECDBFDF91CF911F91FF90EF90DF90F8
:10D2E000CF9008952F923F924F925F926F927F92CC
:10D2F0008F929F92AF92BF92CF92DF92EF92FF9266
:10D300000F931F93CF93DF93CDB7DEB7A4970FB6DC
:10D31000F894DEBF0FBECDBF9E012F5F3F4F790156
:10D3200098E0D9011D929A95E9F7813009F015C36B
:10D330008091F214813009F010C341E050E062EFB7
:10D3400070E08EEE90E00E94431640E050E065EF02
:10D3500070E08EEE90E00E94431646E250E064EFEB
:10D3600070E08EEE90E00E94431600E416E088EE36
:10D3700093E00E94606F01501109C9F70CE211E0BF
:10D3800021E030E0AE01475F5F4F63EF70E08EEE6B
:10D3900090E00E945316898589708987882341F01F
:10D3A00088EE93E00E94606F0150110949F7D5C2E1
:10D3B00028E030E0A70167EF70E08EEE90E00E9479
:10D3C0005316F981FAA32A812BA33B813CA3CF807A
:10D3D000D884DC24CD24DC24E12CF12C6C81862F34
:10D3E00090E0A0E0B0E0AC01BD01ECE0440F551FBF
:10D3F000661F771FEA95D1F78D8190E0A0E0B0E03D
:10D40000F4E0880F991FAA1FBB1FFA95D1F7842B50
:10D41000952BA62BB72B2E8122952F70BC01CD0109
:10D42000622B0E94FC676093EA367093EB36809320
:10D43000EC369093ED368090EE149090EF14A0901F
:10D44000F014B090F114D501C4019C52A140B1096F
:10D450008A879B87AC87BD87AEE0CC0CDD1CEE1CB9
:10D46000FF1CAA95D1F78091E9149091EA14092E36
:10D47000000CAA0BBB0B14E1880F991FAA1FBB1F3E
:10D480001A95D1F7C81AD90AEA0AFB0AA091EB1437
:10D49000B091EC142A853B854C855D850E94929263
:10D4A000C61AD70AE80AF90A90E4D90EE11CF11C61
:10D4B0000FE0F594E794D794C7940A95D1F7A0911B
:10D4C000E814B0E00E9487922B013C018BE0759438
:10D4D0006794579447948A95D1F7A0E85A0E611C37
:10D4E000711CA091ED140A2E000CBB0B0E949292AD
:10D4F0002AE095958795779567952A95D1F7A301A9
:10D5000092010E94DC91DC01CB013AE0B595A79530
:10D51000979587953A95D1F79C01AD01405E5F4F95
:10D52000A091E614B091E7140E949292DC01CB0125
:10D53000905EAF4FBF4FBC01CD014EE095958795F2
:10D54000779567954A95D1F7A70196010E94DC91DE
:10D550006B017C015FE095958795779567955A9566
:10D56000D1F79B01AC010E94DC919B01AC0167E00B
:10D5700055954795379527956A95D1F7A091E5146C
:10D58000B0E00E948792DC01CB0174E0B595A795CD
:10D59000979587957A95D1F7A7019601281B390BA6
:10D5A0004A0B5B0BDA01C90157FF03C080E090E032
:10D5B000DC0181309105A10539E1B30724F080E059
:10D5C00090E0A0E0B9E12CE0B595A79597958795F7
:10D5D0002A95D1F78093EE369093EF36A093F036EC
:10D5E000B093F13675016401FF0CCC08DC2C760198
:10D5F0009401A5016C2D7C2D8C2D9C2D345F414018
:10D60000510961097109810991092A873E874F876C
:10D61000588B698B7A8B8B8B9C8B59016A017B01B0
:10D620008C010E949A922D8B3E8B4F8B5D8F6E8F5B
:10D630007F8F88A399A33091D6142091D514932F6E
:10D64000990F990B492F592F692F792F892F0E94F4
:10D650009A920CE00E94CA93922E832E742E652E0D
:10D66000562E472E382E292E3091D8142091D714BB
:10D67000932F990F990BAD88BE88CF88DD8CEE8CE7
:10D68000FF8C08A119A1492F592F692F792F892FB4
:10D690000E949A9208E00E94E393A92CB82CC72C10
:10D6A000D62CE52CF42C032D122D0E9401947058D9
:10D6B0008F4F9F4F2090D3143090D4145101C12C20
:10D6C000D12CE12CF12C00E010E00E949A9201E2B2
:10D6D0000E94E393288F398F4A8F5B8F6C8F272EA0
:10D6E000382E492EA0E00E94289409F42AC13091D6
:10D6F000DE142091DD14932F990F990BAD88BE880D
:10D70000CF88DD8CEE8CFF8C08A119A1492F592FF1
:10D71000692F792F892F0E949A922D8B3E8B4F8BE8
:10D72000552E3B014C013091DC142091DB14932FDA
:10D73000990F990BAA84BE84CF84D888E988FA8887
:10D740000B891C89492F592F692F792F892F0E9406
:10D750009A9201E10E94CA93AD88BE88CF88D52CE9
:10D76000730184010E94019459016A017B01582EC2
:10D77000192FBBA14B2F50E060E070E0E4E0440FB4
:10D78000551F661F771FEA95D1F78CA182958F7080
:10D79000482BEAA18E2F90E0A0E0B0E0FCE0880FDB
:10D7A000991FAA1FBB1FFA95D1F7482B592B6A2B3B
:10D7B0007B2B80E090E0A0E1B0E0841B950BA60BF2
:10D7C000B70B3C014D01990C6608762C43019C0176
:10D7D000AD01662D762D862D962D0FE10E94CA9300
:10D7E00039014A01B62FA72FF82FE92F3091DA140B
:10D7F0002091D914932F990F990B492F592F692FE5
:10D80000792F892F03E20E94CA93052D0E9401946B
:10D8100059016A017B018C019301A4016B2F7A2FBE
:10D820008F2F9E2F0E941694E5E3AE2EFCE0BF2EB4
:10D83000C12CD12CE12CF12C00E010E00E949A9236
:10D84000A88CB98CCA8CDB8CEC8CF22C032D142D9B
:10D850000E94F5922A873E874F87588B698B7A8B77
:10D860008B8B9C8B0DE00E94E393922E832E742E63
:10D87000652E562E472E382E292E3091E4142091F5
:10D88000E314932F990F990BA92CB82CC72CD62CE5
:10D89000E52CF42C032D122D492F592F692F792FA8
:10D8A000892F0E949A920E949A9209E10E94E39322
:10D8B000AA84BE84CF84D888E988FA880B891C8919
:10D8C0000E94019419012A013B014C013091E2149C
:10D8D0002091E114932F990F990B492F592F692FFC
:10D8E000792F892F0E949A9203E10E94E3935901B4
:10D8F0006A017B018C019101A201B301C4010E9464
:10D90000019408E00E94E39359016A017B01E82F2A
:10D91000192F3091E0142091DF14932F990F990B58
:10D92000492F592F692F792F892F04E00E94CA931C
:10D930000E2F0E940194722F632F942F852F9B012D
:10D9400004C030E020E090E080E03093F236209395
:10D95000F3369093F4368093F536A4960FB6F89488
:10D96000DEBF0FBECDBFDF91CF911F910F91FF9012
:10D97000EF90DF90CF90BF90AF909F908F907F906F
:10D980006F905F904F903F902F900895CF93E6E473
:10D99000F1E0C081908180812081C07C2295269514
:10D9A00026952370C20F969596959073C90F829510
:10D9B0008C70C80F1F92CF938AE094E19F938F934E
:10D9C0000E94239D0F900F900F900F908C2FCF915E
:10D9D0000895CF93C82F81E29AE09F938F930E947E
:10D9E0000F9D0F900F90C0FF04C08EE29AE00E943E
:10D9F0004B9DC1FF04C08DE39AE00E944B9DC2FF86
:10DA000004C08CE49AE00E944B9DC3FF04C08BE5E8
:10DA10009AE00E944B9DC4FF05C08AE69AE0CF9130
:10DA20000C944B9DCF9108951F93CF93DF9383B1B7
:10DA300081708093043746E069E180E00E94427083
:10DA400080E00E9497700E941C6F85E79AE09F9388
:10DA50008F938FEE93E19F938F930E94239D8EB3BC
:10DA60000E94E96C0E94977A0E94CE7960E070E093
:10DA700089EB92E00E946A7A0E94B278E091D00A23
:10DA8000F091D10A19950E94C66C90E00E94C8706E
:10DA90000E945B8182E080934139809342390E94E9
:10DAA0006D6E41E459E3BC018DEC9BEA0E949273D8
:10DAB0000E94DF6D0E947F730E94716E0E949274BB
:10DAC0000E94E47FE0914A0BF0914B0B1995E09195
:10DAD000220BF091230B1995E091060BF091070BA7
:10DAE00019950E949474182FC091560BD091570B22
:10DAF000FE0119950F900F900F900F90892B49F010
:10DB0000FE011995BC0180E890E00E94F891EB01BC
:10DB100002C0C0E8D0E00E947C731F921F93DF9385
:10DB2000CF931F928F938091490B8F938091480BD5
:10DB30008F938091210B8F938091200B8F938DEB8E
:10DB400093E19F938F930E94239D80EB93E19F939A
:10DB50008F930E94239D8FE993E19F938F930E945F
:10DB6000239D60E070E085EE92E00E946A7A60E0BA
:10DB700070E087E992E00E946A7A8DEE99E00E9457
:10DB8000CF7687E993E19F938F930E94239D8DB772
:10DB90009EB742960FB6F8949EBF0FBE8DBFDF9121
:10DBA000CF911F91089580E88093610010926100E9
:10DBB0000E94146D0E94DE790E94BA70FBCFEF9232
:10DBC000FF920F931F93CF93DF93CDB7DEB7A0974C
:10DBD0000FB6F894DEBF0FBECDBF83E690E00E9483
:10DBE000D49F182F282F35EF380F303108F0982F99
:10DBF0009095291709F463C089E194E19F938F936D
:10DC00000E94239DEEE5F4E18E010F5F1F4FCE01D0
:10DC100009960F900F90D801780124912D93319699
:10DC2000A817B907D1F7F89448E050E06FE770E023
:10DC3000C8010E94DA9FE0E5F4E1CE010F96D80119
:10DC400024912D933196A817B907D1F74EE050E0F3
:10DC500061E770E0C8010E94DA9FE6E4F4E1CE01DA
:10DC60000B962491D8012D938D013196A817B907F1
:10DC7000C1F74AE050E067E670E0C7010E94DA9F12
:10DC80006DEC7BEA81E690E00E94F29F60E070E03C
:10DC90008FE590E00E94F29F60E08EE590E00E94A8
:10DCA000E49F60E070E085E690E00E94F29F1AE158
:10DCB0006AE175EE83E690E00E94F29F7894812FEE
:10DCC000A0960FB6F894DEBF0FBECDBFDF91CF9107
:10DCD0001F910F91FF90EF9008958FE590E00C94C5
:10DCE000D49F8EE590E00C94CC9F83B1817090E03E
:10DCF0000895209880E090E0089580E090E00895F5
:10DD0000CF93DF93EC01888199818737910509F4DE
:10DD100057C08E37910509F470C0892B09F084C073
:10DD20000E94C77980930A371092F6141092F51466
:10DD30008091F5149091F614FC01EE0FFF1FED5643
:10DD4000FD4F0190F081E02D3097B1F0DC01A85F2C
:10DD5000B84C1C920480F581E02D60E070E080E812
:10DD600090E019958091F5149091F6140196909396
:10DD7000F6148093F514DCCF8093F71487E790E0D6
:10DD800039C0FC01E85FF84C208127FD22C080915A
:10DD9000F5149091F61401969093F6148093F5146F
:10DDA0008091F5149091F6142091F71430E08217C9
:10DDB00093073CF38091F3149091F414892BF1F2C2
:10DDC0001092F4141092F3141092F6141092F514A9
:10DDD000E7CF880F991FFC01ED56FD4F408151811F
:10DDE00060910A3780E090E00E943E7A892B49F4E6
:10DDF0008EE790E0998388831BC080910A37861351
:10DE000017C0E091F514F091F614E85FF84C8081AA
:10DE10008F7780838091F3149091F41401969093FE
:10DE2000F4148093F314B3CF1982188283E001C0F5
:10DE300081E0DF91CF910895F8941092B60016BC5E
:10DE400089E787BD82E084BD95E095BD95B395BB1C
:10DE500080936E00789408950F931F936091FA1445
:10DE60007091FB148091FC149091FD140091FA14B0
:10DE70001091FB142091FC143091FD146017710770
:10DE80008207930759F71F910F9108950F931F93DE
:10DE90006091133770911437809115379091163730
:10DEA00000911337109114372091153730911637A0
:10DEB000601771078207930759F71F910F91089513
:10DEC000009731F0880F991F880F991F0197F1F77C
:10DED00008951F920F920FB60F9211240BB60F9256
:10DEE0002F933F934F935F936F937F938F939F9362
:10DEF000AF93BF93EF93FF938091FA149091FB142B
:10DF0000A091FC14B091FD140196A11DB11D809348
:10DF1000FA149093FB14A093FC14B093FD14809119
:10DF2000F9148F5F8093F91487FF15C01092F914CC
:10DF30008091133790911437A0911537B09116370F
:10DF40000196A11DB11D8093133790931437A093B0
:10DF50001537B09316378091B2388823E1F080915D
:10DF6000F8148F5F8093F81487FF15C01092F8148F
:10DF700080910B3790910C37A0910D37B0910E37EF
:10DF80000196A11DB11D80930B3790930C37A09380
:10DF90000D37B0930E370E941A78892B11F00E942A
:10DFA0003B77FF91EF91BF91AF919F918F917F91BF
:10DFB0006F915F914F913F912F910F900BBE0F90FA
:10DFC0000FBE0F901F9018951F920F920FB60F92D1
:10DFD00011240BB60F922F933F934F935F936F9340
:10DFE0007F938F939F93AF93BF93EF93FF93809112
:10DFF000C600E0911937F0911A37309709F019955A
:10E00000FF91EF91BF91AF919F918F917F916F9110
:10E010005F914F913F912F910F900BBE0F900FBECC
:10E020000F901F9018951F920F920FB60F92112408
:10E030000BB60F922F933F934F935F936F937F9302
:10E040008F939F93AF93BF93EF93FF938091CE00F5
:10E05000E0911737F0911837309709F01995FF9133
:10E06000EF91BF91AF919F918F917F916F915F9150
:10E070004F913F912F910F900BBE0F900FBE0F90BD
:10E080001F90189581110EC01092C5006093C400B6
:10E0900088E98093C1004093C20010921A37109211
:10E0A00019370895813069F41092CD006093CC0047
:10E0B00088E98093C9004093CA00109218371092E3
:10E0C00017370895811107C08091C00085FFFCCFEC
:10E0D0006093C6000895813031F48091C80085FFB7
:10E0E000FCCF6093CE000895CF93C82F8A3031F4CF
:10E0F0006DE08091FE140E94627002C08D3029F0A4
:10E100006C2F8091FE140E94627080E090E0CF91AD
:10E110000895811105C070931A37609319370895D7
:10E12000813021F4709318376093173708958093E6
:10E13000FE1481EA92E090935E3B80935D3B0895EC
:10E1400084B7877F84BF0FB6F894A895809160004C
:10E15000886180936000109260000FBE08959FE078
:10E1600088E10FB6F894A895809360000FBE909355
:10E1700060000895A89508950FB6F894A895809129
:10E180006000886180936000109260000FBE089567
:10E190000C94E2980C94DE988091203790E00895DA
:10E1A0008091390181FF09C0809139018D7F809371
:10E1B000390189E190E00197F1F723E040E06FE158
:10E1C00082E491E00E94EF7585E090E00197F1F71D
:10E1D00008959091390191FD0AC0282F803108F0EF
:10E1E0002FE040E06FE085E491E00C94EF75089536
:10E1F0008091390181FD09C040E06FE181E491E047
:10E200000E94E4758F7E813019F080E090E00895DF
:10E2100081E090E008958091390181FF02C081E0A2
:10E22000089540E06FE181E491E00E94E4758F3150
:10E2300021F08F7E8150823090F780E008958091A8
:10E24000390181FD04C00E940B718823C1F3089538
:10E250001092B2388091390181FD8BC00E941F71EC
:10E260008091390181FD85C00E94D0708091390173
:10E270008260809339018091EA388823D9F18091B6
:10E280009400909195004091FB385091FC38841790
:10E290009507A0F48091C7389091C838A091C938EB
:10E2A000B091CA38875F924CAF4FBF4F8093C73849
:10E2B0009093C838A093C938B093CA38209194007D
:10E2C00030919500241B350B8091C7389091C83848
:10E2D000A091C938B091CA38820F931FA11DB11DFA
:10E2E0008093C7389093C838A093C938B093CA3880
:10E2F0001092EA388091EC388823D9F1809194000B
:10E30000909195004091FF385091003984179507FE
:10E31000A0F48091CF389091D038A091D138B091AD
:10E32000D238875F924CAF4FBF4F8093CF389093D6
:10E33000D038A093D138B093D23820919400309146
:10E340009500241B350B8091CF389091D038A09147
:10E35000D138B091D238820F931FA11DB11D809387
:10E36000CF389093D038A093D138B093D238109250
:10E37000EC3808958091B238882321F00E940B7107
:10E380000E94287180E090E0089522E0260F27FF88
:10E390000CC08091B0389091B13801969093B1380B
:10E3A0008093B0388FEF9FEF0895AB01BC018FEFE2
:10E3B00094E10E94509C80E090E0089540E06FE17D
:10E3C00081E491E00C94E475282F40E06FEF86E53E
:10E3D00091E00E94EF750895CF93DF9398EF980F27
:10E3E000923038F0982F9F7E963019F0893109F0DD
:10E3F0004BC09091390191FD4AC0C82F0E941F71F6
:10E400000E94DE71D82FC81709F43BC0C83029F428
:10E41000809139010E94D07027C0C93119F486312A
:10E4200081F404C0C63169F4893159F429E040E02F
:10E430006FE182E491E00E94EF7585E090E0019742
:10E44000F1F72C2F40E06FE182E491E00E94EF753C
:10E45000D83031F48FEF0E94E47181ED92E002C078
:10E4600085E090E00197F1F70E94DE71C81749F04E
:10E47000C63019F4813071F404C0C63159F48131C9
:10E4800049F480E490E008C082E490E005C084E4B0
:10E4900090E002C083E490E0DF91CF9108958091F5
:10E4A000940090919500909300398093FF3881E01B
:10E4B0008093EC388093B2389091390191FF1EC05F
:10E4C00020919400309195003093FC382093FB38D4
:10E4D0008093EA388093AD382FB7789480913901D2
:10E4E000809139018D7F8093390180E197E23091ED
:10E4F000AD38332311F00197D1F72FBF86E10E9489
:10E50000EC710C941F718091B238811102C00E948D
:10E510004F7281E090E008950F931F93CF93DF93A4
:10E520001F92CDB7DEB78091B238882361F0809119
:10E53000390181FF02C080E07BC00E940B718823FB
:10E54000D1F300E003C00E94837201E08091940047
:10E55000909195009093FA388093F93811E01093D8
:10E56000E93880E88093550186E00E94EC711093B1
:10E5700021378FB789837894109247018091213792
:10E580008111FCCF89818FBF8091470111E08E30CE
:10E5900008F010E0119586E10E94EC71109255018F
:10E5A0008091E9388823D9F1809194009091950069
:10E5B0004091F9385091FA3884179507A0F480916A
:10E5C000C3389091C438A091C538B091C638875FE0
:10E5D000924CAF4FBF4F8093C3389093C438A093F1
:10E5E000C538B093C6382091940030919500241B13
:10E5F000350B8091C3389091C438A091C538B09143
:10E60000C638820F931FA11DB11D8093C33890930C
:10E61000C438A093C538B093C6381092E9380111B8
:10E620000E94BA71812F829586958695837081703C
:10E6300090E00F90DF91CF911F910F9108958FEF90
:10E6400080934E0121E044E060EF8CE691E00E946F
:10E65000EF7525E041E06EE08CE691E00E94EF75F9
:10E6600080E880936F018091460180936D0121E0E5
:10E6700045E060E284E491E00C94EF75CF93DF9382
:10E68000C9EFD7E0CE010197F1F70E94E375109230
:10E6900027371092A93710922B38109226371092F4
:10E6A0002537E9E3F1E080818E7F808380818D7F53
:10E6B000808381EC93E00197F1F780818160808312
:10E6C00023E040E06FE182E491E00E94EF75219742
:10E6D000F1F780915D0180915E010E941F7360E0FF
:10E6E00070E08FEA92E00E946A7A0E944F7281E0A5
:10E6F00090E0DF91CF910895809180150895CF9398
:10E70000C82F0E941F71C09380152C2F40E06FE12D
:10E7100088E491E0CF910C94EF750E947F7386E0BE
:10E720000C94EC71EF92FF920F931F93CF93DF93B2
:10E730007C018B01EA011F936F93FF928F9386EA0E
:10E740009AE09F938F930E940F9DE0926201F09256
:10E75000630100936001109361010F900F900F907F
:10E760000F900F900F902097C1F0888180936B01DC
:10E77000898180936A018A81809369018B8180936A
:10E7800068018C81809367018D81809366018E8101
:10E79000809365018F8180936401DF91CF911F91F8
:10E7A0000F91FF90EF9008958FEA92E00E948B7A8C
:10E7B00081E0809320378091223790912337019612
:10E7C000909323378093223781E090E008950F9350
:10E7D0001F93CF9320912637C2E8C29F9001112446
:10E7E000F901E95DF84C4081442309F44FC047FD2D
:10E7F00009C0433038F050E08A0102501109601717
:10E80000710710F4108242C0B901685D784C0E9413
:10E81000509C80912637C89FF0011124E95DF84C87
:10E82000DF01A058BF4F9C9190931B3710828F5FE0
:10E83000833018F48093263702C010922637E09177
:10E84000263782E8E89FF0011124E95DF84C8081C9
:10E85000882319F00E94D47302C01092203760916F
:10E86000470160931C3780911F37882311F0681788
:10E8700010F460931F3770E084E00E94378160914C
:10E880001B3770E083E00E94378102C000E010E097
:10E89000C801CF911F910F9108950F931F93CF93AC
:10E8A000DF931F92CDB7DEB78C01FC01808191818F
:10E8B000009709F18334954029F0F8011182108204
:10E8C00083E02AC06238E1F40E94EF808FB7898329
:10E8D000F8940E94598060E870E00E94E7732981F3
:10E8E0002FBF1816190674F40E945480E091500B43
:10E8F000F091510B199583E495E0F80191838083A1
:10E9000081E00AC080911D3790911E370196909347
:10E910001E3780931D37EFCF0F90DF91CF911F915E
:10E920000F9108950C94E9708091390181FD06C022
:10E9300040E06FE085E491E00C94E47580E1089597
:10E94000EF92FF921F93CF93DF931F92CDB7DEB765
:10E95000182F8091390181FD07C00E941F7180919D
:10E96000B23881111CC05AC08091940090919500DA
:10E970009093FC388093FB3881E08093EA38809351
:10E98000AD38809139018D7F8093390180E197E224
:10E990002091AD38222309F30197D1F7DECF809182
:10E9A000EC388823D9F180919400909195004091A2
:10E9B000FF385091003984179507A0F48091CF3823
:10E9C0009091D038A091D138B091D238875F924CD5
:10E9D000AF4FBF4F8093CF389093D038A093D138AA
:10E9E000B093D2382091940030919500241B350BC0
:10E9F0008091CF389091D038A091D138B091D23851
:10EA0000820F931FA11DB11D8093CF389093D038F2
:10EA1000A093D138B093D2381092EC3889E10E949B
:10EA2000EC7186E00E944281892B51F00E9494741F
:10EA3000E82E86E00E94428181500E94E97002C067
:10EA4000E12CF12C80919400909195009093FE38E8
:10EA50008093FD3881E08093EB388FB78983F894F9
:10EA600080913901826080933901809139018D7FD5
:10EA70008093390162E0610F8FEF94E10E94357657
:10EA800089818FBF8091AE389091AF380196909375
:10EA9000AF388093AE380E941F7145E060EE82E48B
:10EAA00091E00E94E475182F86E00E944281892B34
:10EAB00019F08E2D0E94E9708091EB388823D9F1EE
:10EAC00080919400909195004091FD385091FE38CE
:10EAD00084179507A0F48091CB389091CC38A09101
:10EAE000CD38B091CE38875F924CAF4FBF4F8093F7
:10EAF000CB389093CC38A093CD38B093CE382091BA
:10EB0000940030919500241B350B8091CB38909167
:10EB1000CC38A091CD38B091CE38820F931FA11D73
:10EB2000B11D8093CB389093CC38A093CD38B0935F
:10EB3000CE381092EB388091B238882371F08091F2
:10EB4000940090919500909300398093FF3881E074
:10EB50008093EC380E944F7202C00E9428711230DC
:10EB600028F48CE00E94428110E00BC0133031F099
:10EB7000153031F0173029F411E003C012E001C064
:10EB800013E0812F90E00F90DF91CF911F91FF90C4
:10EB9000EF900895CF93DF93EB010E94C57100972A
:10EBA00029F4CE010E94A074009751F02091B03852
:10EBB0003091B1382F5F3F4F3093B1382093B03848
:10EBC000DF91CF9108950895FC0180816823862FFD
:10EBD00090E002C0959587954A95E2F70895CF9306
:10EBE000DF931F92CDB7DEB7FC01922F8FB78983D9
:10EBF000F8942081562F50955223292F01C0220FBF
:10EC00004A95EAF72623252B208389818FBF0F9011
:10EC1000DF91CF910895CF93DF93E0917B012DEFAA
:10EC20002E0F2D3740F0FC011082E058FF4F10826C
:10EC30003196108217C0DC01ED932E2FC0E8D1E091
:10EC400038813D93215021962111FACFE150F0E017
:10EC5000E058FE4F2181FC01E058FF4F20833196A0
:10EC600021E02083DF91CF9108956093800162506D
:10EC7000E1E8F1E0DC012D91CD0120836150319676
:10EC80006111F8CF08951F920F920FB60F921124C1
:10EC90000BB60F922F933F934F935F936F937F9396
:10ECA0008F939F93AF93BF93EF93FF93809147010F
:10ECB00080931C378091253722E8829FC001112460
:10ECC000895D984C0E940B76809125378F5F833049
:10ECD00018F48093253702C0109225370E94D47310
:10ECE000FF91EF91BF91AF919F918F917F916F9124
:10ECF0005F914F913F912F910F900BBE0F900FBEE0
:10ED00000F901F9018951F920F920FB60F9211241B
:10ED10001092AD380F900FBE0F901F9018951F9254
:10ED20000F920FB60F921124109224370F900FBE3E
:10ED30000F901F9018951F920F920FB60F921124EB
:10ED40000F900FBE0F901F9018951F920F920FB645
:10ED50000F9211240F900FBE0F901F9018951F92C5
:10ED60000F920FB60F9211240F900FBE0F901F90AD
:10ED700018951F920F920FB60F9211240F900FBE8D
:10ED80000F901F9018951F920F920FB60F9211249B
:10ED9000109221370F900FBE0F901F901895CF93B0
:10EDA000DF93EC0189919991009729F060E070E080
:10EDB0000E946A7AF7CFDF91CF910895CF92DF92C8
:10EDC000EF92FF920F931F93809185159091861576
:10EDD000892B49F410928115109282151092831597
:10EDE0001092841541C00E942C6F8B019C01E09110
:10EDF0008515F091861540815181628173818481EE
:10EE00009581A681B781840F951FA61FB71F801B10
:10EE1000910BA20BB30B0084F185E02D3097C1F06C
:10EE2000C080D180E280F380448155816681778102
:10EE30004C0D5D1D6E1D7F1D401B510B620B730B36
:10EE4000481759076A077B0730F7DB01CA01E3CF90
:10EE5000800F911FA21FB31F80938115909382157D
:10EE6000A0938315B09384151F910F91FF90EF909D
:10EE7000DF90CF90089589EB92E00C948B7AEF921B
:10EE8000FF920F931F93CF93DF938C01FC0180813E
:10EE90009181009799F089359105D9F0F801118297
:10EEA000108283E068C0828593854817590709F06E
:10EEB00049C00084F185E02D3097A9F7109286159E
:10EEC0001092851589E590E0F8019183808381E0B7
:10EED00052C0673891F16238A9F7C0918515D09179
:10EEE0008615E12CF12C209769F3CE010E94E67A79
:10EEF000892BF1F0AE0168E88A859B850E943E7AF5
:10EF0000892BA1F41B861A8688859985E114F10462
:10EF100021F0F7019187808704C090938615809334
:10EF20008515198618860E94DE76D7CF0E943B771A
:10EF30007E010884D985C02DD6CFE0918515F0914A
:10EF40008615BACFF0938615E0938515A085B18517
:10EF5000109709F4B7CF1A968D919C911B9748177B
:10EF6000590739F418968D919C911997918780874C
:10EF7000EDCFFD01EBCFDF91CF911F910F91FF906E
:10EF8000EF900895CF93DF93EC010E943B772A85A1
:10EF90003B859091851580918615232B91F0E92F63
:10EFA000F82F309771F0EC17FD0739F48091331684
:10EFB000909134169387828710C00084F185E02DEC
:10EFC000F0CF20913316309134163B872A879887EB
:10EFD0008987D0938615C0938515DF91CF910C94C6
:10EFE000DE76CF93DF93EC010E94B87ACE01DF91F9
:10EFF000CF910C94C277CF93DF93EC010E94C87A33
:10F00000CE01DF91CF910C94C277CF93DF93EC01C7
:10F010000E94DA7ACE01DF91CF910C94C27721E081
:10F0200030E0FC0182859385892B11F020E030E0EF
:10F03000C901089581E090E02091851530918615F1
:10F04000232B11F480E090E00895CF93DF93EC013F
:10F05000E0918515F0918615E817F90769F4888520
:10F06000998590938615809385150DC0808591852F
:10F07000C817D90721F0FC013097C1F706C0888571
:10F080009985918780870E94DE76198618861B866F
:10F090001A86DF91CF910895EF92FF920F931F93FD
:10F0A000CF93DF938C017A01FC01808191810097DD
:10F0B00041F08A34910511F1F8011182108283E048
:10F0C0004AC088E895E10E94157BEC01209761F029
:10F0D0004E815F8168857985CE0102960E94F17725
:10F0E0000990D881C02DF2CF81E0809387158AE402
:10F0F00090E0F8019183808381E02DC06838E1F7CA
:10F1000088E895E10E94157BEC01209781F3CE0100
:10F110000296E816F906D9F4BE0188E895E10E9446
:10F12000357BE0903316F09034168E859F85909352
:10F13000341680933316E889F989309719F08A8953
:10F140009B891995F0923416E0923316D0CF09902E
:10F15000D881C02DDACFDF91CF911F910F91FF9011
:10F16000EF9008951092871588E895E10E94117B31
:10F1700060E070E083EC92E00C946A7AEF92FF9288
:10F180000F931F93CF93DF93EC01E0903316F09031
:10F190003416FF86EE86398B288B1B8B0A8B809169
:10F1A0008715882379F083EC92E09093341680934E
:10F1B0003316CE0102960E94F177F0923416E09257
:10F1C000331604C04E835F8368877987BE0188E861
:10F1D00095E10E94357BBE0188E895E1DF91CF91F2
:10F1E0001F910F91FF90EF900C94507BCF93DF9382
:10F1F000EC0180918715882329F0CE0102960E94A8
:10F20000257804C01B861A861D861C86BE0188E8E8
:10F2100095E1DF91CF910C94357B1F93CF93DF93D2
:10F22000DC011496ED91FC9115973097E1F0162FC3
:10F23000EC01909334168093331682E08887CD01D9
:10F2400006961995082E000C990B0297029710F05C
:10F25000133839F4BE01CE01DF91CF911F910C9488
:10F260003D7981E08887DF91CF911F910895FC015E
:10F27000208520FD0C940D790895CF92DF92EF92B6
:10F28000FF920F931F93CF93DF93E0903316F0908C
:10F2900034160091351610913616F801E817F90763
:10F2A00039F0309709F44BC00190F081E02DF6CF92
:10F2B000009709F444C06B01EC018885882309F1AB
:10F2C00018860115110561F00C171D0729F0AE0114
:10F2D00067E8C8010E943779F80100811181F1CFF8
:10F2E000EC81FD81309769F0CC15DD0551F0D093AC
:10F2F0003416C093331640E050E063E8CE01069622
:10F300001995E0913516F0913616CE17DF0741F4C6
:10F310008881998190933616809335160CC0FC0134
:10F32000309749F080819181C817D907C1F788814A
:10F33000998191838083F0923416E0923316DF91A5
:10F34000CF911F910F91FF90EF90DF90CF90089594
:10F350001F93CF93DF9310928F15C0913516D091E4
:10F36000361611E0209779F08985882341F01887B7
:10F37000198640E050E062E8CE010E940D790990C4
:10F38000D881C02DEFCFDF91CF911F91089580914B
:10F39000321691E0980F9093321608958AE8809380
:10F3A00032161092301610923116109236161092B4
:10F3B00035161092341610923316089580918F15D9
:10F3C00081110E94A87990913116992309F44EC0B9
:10F3D000E09130162E2F30E085E0E89FF0011124F7
:10F3E000E057FA4E608160938E15418152815093AF
:10F3F0008D1540938C150380F481E02D2F5F3F4FD6
:10F400002F713327209330169150909331163097F7
:10F4100031F5809135169091361690938B15809327
:10F420008A1580918A1590918B15892BF9F080911E
:10F430008F1581110E94A87940918C1550918D15DE
:10F4400060918E1580918A1590918B150E94377965
:10F45000E0918A15F0918B1580819181DECF613822
:10F4600011F481E08087CF010E94377980918F1558
:10F470002091311690E0820F911D08959C0190918A
:10F4800031169032A9F0E0913016E90FEF7185E066
:10F49000E89FF0011124E057FA4E608352834183C4
:10F4A000348323839F5F9093311680E090E008952A
:10F4B00081E090E00895CF93DF93C0913316D0910F
:10F4C00034160E943779D0933416C0933316DF91E7
:10F4D000CF910895AB013091351620913616E32F68
:10F4E000F22FE817F907B1F0309721F00190F08181
:10F4F000E02DF7CF009771F0FC01308321839093CA
:10F5000036168093351621E020871782168261E82F
:10F510000C945B7A0895009749F0FC0120852150F6
:10F52000223020F421E0218720938F1508950C9438
:10F530004D8580913716909138160097C1F0109242
:10F54000381610923716DC0114966D917C91159740
:10F550001296ED91FC9113971995E0913716F09161
:10F560003816309721F0808191810C946785089539
:10F57000CF93DF93EC014C835D836E837F830E9486
:10F580002C6F688379838A839B83DF91CF91089561
:10F59000FC01408151816281738184819581A681C2
:10F5A000B781840F951FA61FB71F80839183A28305
:10F5B000B3830895CF93DF93EC010E942C6F68838F
:10F5C00079838A839B83DF91CF910895CF92DF92D5
:10F5D000EF92FF92CF93DF93EC010E942C6FC880D3
:10F5E000D980EA80FB80DC01CB018C199D09AE0932
:10F5F000BF090196A11DB11D21E030E0CC80DD8066
:10F60000EE80FF80C816D906EA06FB0610F020E05F
:10F6100030E0C901DF91CF91FF90EF90DF90CF9064
:10F620000895FC01118210820895FC01808191816E
:10F630000895DC01ED91FC91309741F0808191813A
:10F64000009711F0FC01FACFCF01089580E090E01F
:10F650000895DC01ED91FC911197309721F0208104
:10F6600031812D933C93CF010895DC01ED91FC9104
:10F670003097A9F0A0E0B0E0208131816E177F07BC
:10F6800041F4109709F4DC012D933C931182108210
:10F690000895DF012115310511F0F901EDCF08952D
:10F6A0000F931F93CF93DF938C01EB010E94357B67
:10F6B00019821882C8010E94197B009711F4F80181
:10F6C00001C0FC01D183C083DF91CF911F910F91C5
:10F6D0000895DC01ED91FC9180E090E0309729F0F5
:10F6E00001960190F081E02DF9CF0895009721F067
:10F6F000FC0180819181089580E090E008952F922F
:10F700003F924F925F926F927F928F929F92AF92B1
:10F71000BF92CF92DF92EF92FF920F931F93CF93FE
:10F72000DF93CDB7DEB768970FB6F894DEBF0FBE94
:10F73000CDBFE3EBF8E354A445A436A427A490A4DA
:10F7400081A472A463A4248D2983858D8A83B68CB9
:10F75000A78C908D9B83218D2C83828D8D83938D9F
:10F760009E8324892F83858988879689998727890D
:10F770002A8780898B8791899C8722892D87838915
:10F780008E8794859F872585288B8685898B97858D
:10F790009A8B20852B8B81858C8B92859D8B2385E5
:10F7A0002E8BF480E580D680C78080818F8B9181FD
:10F7B000988F128103810E94466F2F923F924F9241
:10F7C0005F926F927F928F929F92AF92BF922A81A7
:10F7D0002F9329812F932E812F932D812F932C816D
:10F7E0002F932B812F932A852F9329852F9328855B
:10F7F0002F932F812F932E852F932D852F932C853B
:10F800002F932B852F932A892F9329892F9328892A
:10F810002F932F852F932E892F932D892F932C890A
:10F820002F932B892F93CF92DF92EF92FF920F931A
:10F830001F93288D2F932F892F939F938F937F93BF
:10F840006F93E1E4F9E381811F928F9380811F928E
:10F850008F9386E694E19F938F930E94239D0FB62A
:10F86000F894DEBF0FBECDBF68960FB6F894DEBF2A
:10F870000FBECDBFDF91CF911F910F91FF90EF9001
:10F88000DF90CF90BF90AF909F908F907F906F90C0
:10F890005F904F903F902F900895CF93DF93EC01AE
:10F8A0004A815B8160E070E08C819D810E94599C5F
:10F8B000288139818A819B81289FA001299F500D31
:10F8C000389F500D112460E070E08E819F81DF91A0
:10F8D000CF910C94599CFC018281938120E030E00F
:10F8E00028173907D1F0A481B581A20FB31F4C911D
:10F8F000411110C081E08C9380819181289FA001EB
:10F90000299F500D389F500D112486819781840FB7
:10F91000951F08952F5F3F4FE3CF80E090E008955B
:10F92000FC01868197814281538120E030E02417D9
:10F930003507D1F08617970781F4A481B581A20F0E
:10F94000B31F8C91181614F481508C938481958187
:10F95000FC01E20FF31F80810895A081B1818A0F1D
:10F960009B1F2F5F3F4FE3CF8FEF0895FC01268150
:10F97000378162177307A0F0A281B3814081518162
:10F98000A49FC001A59F900DB49F900D1124280F36
:10F99000391F81E090E06217730720F080E008953E
:10F9A00080E090E00895CF92DF92EF92FF920F9364
:10F9B0001F93CF93DF937C018B016A0189E396E16A
:10F9C0000E94157BEC01892B51F0EC81FD81309771
:10F9D00011F0C8011995CE010E94767BF3CFA601E4
:10F9E000B801C701DF91CF911F910F91FF90EF9068
:10F9F000DF90CF900C94B37E0F931F93CF93DF9340
:10FA00000E94FF7E8C0189E396E10E94157BEC0148
:10FA1000892B49F0EA81FB81309709F01995CE01D5
:10FA20000E94767BF4CF0115110539F0C801DF91F2
:10FA3000CF911F910F910C94A77EDF91CF911F91D1
:10FA40000F910895CF92DF92EF92FF920F931F9341
:10FA50000E94E47F0E94EF800E94BF7E0E94FD7E94
:10FA6000C12C88E0D82E87E0E82EF12C00E01EE1C2
:10FA700020E030E040E052E060E070E082E090E0C2
:10FA80000E94517E1F910F91FF90EF90DF90CF90D9
:10FA90000895CF93DF93EC010E94127F009761F0ED
:10FAA0000E947280E091240BF091250BBE0183ED42
:10FAB0009CE7199581E090E0DF91CF91089508953A
:10FAC0000F931F93CF93DF93CAE7D6E14881598103
:10FAD0006A817B8100E010E02AE83DE78AE596E153
:10FAE0000E94BE780E94CA70BC0180E090E028812C
:10FAF00039814A815B810E942092AB01BC012FEACF
:10FB00003DE786E496E10E94BE78DF91CF911F9198
:10FB10000F91089580917A1690917B16A0917C1692
:10FB2000B0917D16409176165091771660917816B7
:10FB300070917916880F991FAA1FBB1F4817590784
:10FB40006A077B0710F4DB01CA0180937A16909351
:10FB50007B16A0937C16B0937D160C94607DCF939A
:10FB6000DF930E94EF800E945980EC011982188275
:10FB70000E94C87E28813981009719F1FC014085D7
:10FB80004423F9F0FC0142815381F901EE0FFF1F7C
:10FB9000EE0FFF1FEC0FFD1F53834283FC014481D6
:10FBA00055812F5F3F4FF901EE0FFF1FEE0FFF1F33
:10FBB000EC0FFD1F51834083398328830E94767B9D
:10FBC000D9CFC901880F991F880F991F02960E94EB
:10FBD000548088819981892B31F08BE396E1DF9104
:10FBE000CF910C94BF7FDF91CF910895AF92BF92D8
:10FBF000CF92DF92EF92FF920F931F93CF93DF93F9
:10FC00001F921F92CDB7DEB75B010E9459808C0115
:10FC1000FC01E080F180FA82E9820E94A1809701D4
:10FC2000220F331F220F331F2E5F3F4F8217930780
:10FC300098F0C12CD12CCE14DF0471F0F80144816E
:10FC4000558162817381C5010E94CC7EFFEFCF1A7E
:10FC5000DF0A0C5F1F4FEFCF0F900F90DF91CF9116
:10FC60001F910F91FF90EF90DF90CF90BF90AF90DA
:10FC700008950F93013099F480916E1690916F164C
:10FC8000A0917016B091711680937A1690937B169E
:10FC9000A0937C16B0937D160F910C94607D0F910C
:10FCA00008954F925F926F927F928F929F92AF9240
:10FCB000BF92CF92DF92EF92FF920F931F932A0190
:10FCC0003B01480159014AE05BE0BC018BE396E14E
:10FCD0000E94A27FEBE3F6E143AA54AA65AA76AAA2
:10FCE00087AA90AEA1AEB2AEC3AED4AEE5AEF6AECC
:10FCF00089E39EE71F910F91FF90EF90DF90CF90E7
:10FD0000BF90AF909F908F907F906F905F904F903B
:10FD10000C94C37EEF92FF920F931F93CF93DF93C8
:10FD20008C01EB017A010E94367FF801F086E782B0
:10FD30006EE07BE0CE01DF91CF911F910F91FF909C
:10FD4000EF900C945A7F0C943E7F0C94497DDC011B
:10FD50001796ED91FC9118970190F081E02D309766
:10FD600009F019940895DC011796ED91FC9118970C
:10FD70000280F381E02D309709F01994089582E80C
:10FD800096E10C94117B90938116809380160895D0
:10FD900082E896E10C94157BEF92FF920F931F93EC
:10FDA000CF93DF938C01EB017A0182E896E10E9408
:10FDB000157B0097D9F0DC0112962D913C91139799
:10FDC0002C173D0781F41696ED91FC91179730970B
:10FDD00069F09701AE01B801DF91CF911F910F91AA
:10FDE000FF90EF9019940E94767BE3CFDF91CF9143
:10FDF0001F910F91FF90EF9008950C94327FCF9355
:10FE0000DF93E091600BF091610B1995EC01892B68
:10FE100029F06A817B8181E00E943781CE01DF91E8
:10FE2000CF9108950F931F93CF93DF93EC01E0914F
:10FE3000620BF091630B19958C016A817B8181E0E3
:10FE40000E94378181E090E0012B11F480E090E086
:10FE5000DF91CF911F910F910895E091640BF09184
:10FE6000650B199484E896E10C94117BFC01738373
:10FE70006283BC0184E896E10C94507BBC0184E869
:10FE800096E10C94357BCF93DF93EC0184E896E107
:10FE90000E94157B009749F0FC01228133812C17C9
:10FEA0003D0729F00E94767BF5CF80E090E0DF915E
:10FEB000CF9108950F931F93CF93DF938B010E94EF
:10FEC000437FEC01892B31F01D830C83C8010E9414
:10FED0002D7F8E83DF91CF911F910F910895DC01CB
:10FEE0001996ED91FC911A970280F381E02D3097DD
:10FEF00009F0199408950F931F93CF93DF931F92E6
:10FF00001F92CDB7DEB78C0188E10E945581BC01FC
:10FF1000CE0101960E946F81D8011996ED91FC9156
:10FF20001A970190F081E02D309729F0BE016F5FA4
:10FF30007F4FC80119950F900F90DF91CF911F91BE
:10FF40000F910895EF92FF920F931F93CF93DF933A
:10FF50008C01EB017A0140E15BE00E948A7EF801AE
:10FF6000F286E18664E17BE0CE01DF91CF911F91C3
:10FF70000F91FF90EF900C945A7F0C94A37ECF9337
:10FF8000DF93EC0161E479E388E10E944B81CE01CB
:10FF9000DF91CF910C94A57EE0914C0BF0914D0B2D
:10FFA0001994E091080BF091090B1994E091520B10
:10FFB000F091530B1994E091540BF091550B199457
:10FFC00080E090E0089508958DEC92E00E944D7CD1
:10FFD0008DED92E00E944D7C85ED92E00C944D7C7D
:10FFE0000F931F93CF93DF93EC01BC018DED92E053
:10FFF0000E94B67C892BA9F00990D881C02DFE0102
:020000021000EC
:1000000061917191CF010E940281BE016E547F4FB8
:10001000CE018E579F4FDF91CF911F910F910C947E
:100020002681BE0185ED92E00E94B67C892BD1F03D
:100030000E94EF80688179818A819B810E94028180
:100040008CA990E00E94B3800CA910E00E9460800F
:10005000BE016C5F7F4FA801DF91CF911F910F917F
:100060000C94509CDF91CF911F910F910895209196
:10007000991D30919A1D2817390798F04091971DC6
:100080005091981D480F591F5093981D4093971DEC
:10009000281B390B30939A1D2093991D81E090E025
:1000A000089580E090E0089590939A1D8093991DA3
:1000B00008958091971D9091981D8C5E924E0895A1
:1000C0008091961D90E08C51934E089581E090E0D0
:1000D0002091E21C3091E31C24513D4111F480E059
:1000E00090E008950E946680892B61F06091E21C87
:1000F0007091E31C4091991D50919A1D84E19DE1FE
:100100000C94509C2091971D3091981D211531051C
:10011000B9F08091991D90919A1DC096E4E1FDE19E
:10012000AF01445E5C414817590734F4DF01A20F68
:10013000B31F4C914193F4CF1092981D1092971DCC
:1001400008958091991D90919A1D08958091961D12
:1001500090E3981B2091991D30919A1DA901490F98
:10016000511DCA0108951F93CF93DF931091961DDF
:10017000212F30E02817390774F0EC010E94A68087
:100180008C0F9D1F8138910530F41C1B1093961D18
:1001900081E090E002C080E090E0DF91CF911F917C
:1001A00008950F931F93CF93DF93E1E1F9E3119249
:1001B000119289E3E134F807D1F7C9E0D9E301E10D
:1001C00019E36EE27BE0CE010E946F8122960C174C
:1001D0001D07B9F7DF91CF911F910F9108951092EC
:1001E000981D1092971D10929A1D1092991D80E3F0
:1001F0008093961D84E19DE19093E31C8093E21C23
:100200000C94D180EF92FF920F931F93CF93DF93C3
:100210008C017B010E94EF80E701C138D10510F00D
:10022000C0E8D0E0AE01B8018091E21C9091E31CDF
:100230000E94509CD0939A1DC093991DCE01DF91CE
:10024000CF911F910F91FF90EF900895FC0190E3E3
:10025000A1E1B9E301900D929A95E1F788E0FB01E5
:10026000A9E0B9E301900D928A95E1F70895E82F8E
:10027000F0E0EE0FFF1FEF5EF64C7183608381E0CC
:1002800090E00895E82FF0E0EE0FFF1FEF5EF64CD0
:1002900080819181089590E0880F991F8752974C33
:1002A0000E946F8181E090E0089590E0880F991F8F
:1002B0008752974C0895E091D00AF091D10A199590
:1002C000E0914A0BF0914B0B1995E091220BF091C4
:1002D000230B1995E091060BF091070B1994FB0184
:1002E00020813181FC0131832083089542E050E078
:1002F0000E94439C21E030E0892B11F020E030E0A7
:10030000C9010895BC0181E499E30C946F8182EBEB
:100310009DE10E940F78892B21F082EB9DE10C94E6
:1003200005780895E0919E1DF0919F1D309709F08A
:10033000199480E00895EF92FF920F931F93CF934B
:10034000DF938C01EA01FC0180819181009741F0EB
:100350008A33934081F1F8011182108283E0F8C062
:1003600080E024E0829FF0011124E056F24E1182D9
:1003700010828F5F8430A9F780939D1D8091331682
:10038000909134169093B11D8093B01D0E94C7794F
:100390008093433940E450E060E070E082EB9DE1FF
:1003A0000E94F1770E942F868AE393E0F8019183FF
:1003B000808381E0CDC06230D9F48091443990913E
:1003C0004539892B89F380915539863029F48091FC
:1003D0006D3981FD0E94878181E00E94768680913F
:1003E000443990914539892BF9F20E94F582DCCF8E
:1003F000633060F5611114C02097B1F2D093423A96
:10040000C093413A83E00E9476868091443990916E
:100410004539892B11F00E9492810E948781C4CFB7
:10042000613011F6209709F4BFCFD0933E3AC093C4
:100430003D3A85E00E947686809144399091453915
:10044000892B09F4B1CF0E949281AECF673809F0B1
:1004500040C010929C1D80EAE82E8DE1F82E80911C
:100460009C1D8430C0F4F70182819381C817D9079D
:1004700049F4808191810E945B86F701118210828C
:1004800013821282F4E0EF0EF11C80919C1D8F5FAD
:1004900080939C1DE4CFE3E4FAE3848D958DC81727
:1004A000D90719F4158E148E118EB0962AE3E33C09
:1004B000F20799F7E9EDFAE381859285C817D90724
:1004C00011F4158214823D968BE3EB35F807A1F702
:1004D0006BCF683809F068CFC25BDD4109F064CFAB
:1004E00082EB9DE10E940F78892B09F45DCF109279
:1004F0009C1DE0919C1DE43008F056CF20E2E29F65
:10050000F0011124ED5BF54C818D8823D9F082EB4D
:100510009DE10E94057880919C1DE0E28E9FC001C4
:1005200011248D5B954C9093423A8093413A82E03E
:100530000E9476868091443990914539892B11F03B
:100540000E94928180919C1D8F5F80939C1DD1CFD2
:10055000DF91CF911F910F91FF90EF900895CF936E
:10056000DF93A091413AB091423A109719F0ED0112
:100570006C9605C0C0913D3AD0913E3A2996809143
:100580003C3A86FF23C010929B1D80E0E0EAFDE12B
:100590008430C1F04081518114962D913C91159782
:1005A0004217530761F4228133812115310539F057
:1005B00080939B1D398328831B821A8205C0349641
:1005C0008F5FE6CF80939B1D0E94878188819981F0
:1005D000009741F04A815B8160914339DF91CF916F
:1005E0000C945B7ADF91CF9108950F931F93CF9373
:1005F000DF9380915539863009F07AC08091443973
:1006000090914539803F910508F472C08897EC01BC
:10061000D695C7959E01220F331F8E0128173907E3
:1006200010F40F5F1F4FCE01889690934539809349
:10063000443990934E3980934F391092713910920A
:1006400070390E9429868095909590937139809396
:10065000703910925739109256390E941886809539
:10066000909590935739809356390E949281C80192
:100670008896909345398093443990934E3980936E
:100680004F3980913F3A9091403ABC016C0F7D1FE9
:10069000A8010E94509CBE0184E699E30E94C58592
:1006A00080914839809364398091493980936539C4
:1006B00080914A398093663980914B3980936739AC
:1006C00010927139109270390E9429868095909508
:1006D000909371398093703910925739109256392E
:1006E0000E9418868095909590935739809356393B
:1006F000DF91CF911F910F910C949281E091E00ACC
:10070000F091E10A199480E090E00895AF92BF92D1
:10071000CF92DF92EF92FF920F931F93CF93DF93CD
:10072000CDB7DEB7E1970FB6F894DEBF0FBECDBFF1
:100730007C016B01CE0101965C0181E3F501119210
:100740008A95E9F781E089838CE00E9442818C835D
:100750001D821F828091BE1D91E0980F9093BE1D57
:10076000898713E018878DEC9BEA9B878A8789E14C
:100770000E9455816EE27BE00E947681892B31F0E8
:1007800082E08E838FEF8C878D8709C089E10E947C
:100790005581BC01CE010C960E946F811E838DECA9
:1007A0009BEA9D8B8C8B61E479E3CE0146960E9497
:1007B0006F810E9459809FA78EA70E94A18099AB4C
:1007C00088ABC5010E9400908C011127C8010E94CE
:1007D000B380892B31F10E946080A801BC01C50162
:1007E0000E9423900091D60A1091D70A0E94A680F9
:1007F0005C010E946080B501F8011995E114F104D3
:1008000081F0009739F0019761F441E050E064E035
:1008100070E004C041E050E060E070E0C601F70124
:100820001995E1960FB6F894DEBF0FBECDBFDF91EC
:10083000CF911F910F91FF90EF90DF90CF90BF90DD
:10084000AF9008950F931F93CF93DF9341155105F8
:1008500079F0FA018B01EC01828193810E94F07F93
:10086000B801CE01DF91CF911F910F910C94868337
:10087000DF91CF911F910F910895EF92FF920F9307
:100880001F93CF93DF93CDB7DEB7E1970FB6F89400
:10089000DEBF0FBECDBF0E94A1807C010E945980A7
:1008A0008E010F5F1F4FA801B7010E941291892B83
:1008B00009F441C088A999A99701281B390BC901DE
:1008C0000E943780892BB9F18E8181110CC0BE0145
:1008D0006A5E7F4F88E10E944B81E091260BF09188
:1008E000270B199528C02A853B852D3C9BEA3907A3
:1008F00019F02F3F3F4FF9F4823019F0E8E0F0E0B3
:1009000002C0E2E0F0E0E00FF11FE017F107F9F2BA
:10091000319783858F3FC9F3BE01645F7F4F89E1C3
:100920000E944B8189E10E94558161E479E30E9434
:100930007681892B61F6E1960FB6F894DEBF0FBE83
:10094000CDBFDF91CF911F910F91FF90EF90089550
:100950000E94CA708093BE1DE091E00AF091E10A06
:100960001994892B29F0E091E00AF091E10A04C082
:10097000E091E20AF091E30A1994FC01680F791FF3
:1009800080E048E1E617F70781F0219198E0382FE1
:100990003227532F517030FD84278695513009F44A
:1009A00080682695915099F7EDCF08951F920F9288
:1009B0000FB60F9211240BB60F922F933F934F93C4
:1009C0005F936F937F938F939F93AF93BF93EF93B7
:1009D000FF9380919400909195009093F6388093C6
:1009E000F53881E08093E73880917100807D8093B5
:1009F00071000E94997A8091E7388823D9F180911B
:100A00009400909195004091F5385091F6388417F4
:100A10009507A0F48091BB389091BC38A091BD3867
:100A2000B091BE38875F924CAF4FBF4F8093BB38B9
:100A30009093BC38A093BD38B093BE3820919400F9
:100A400030919500241B350B8091BB389091BC38B8
:100A5000A091BD38B091BE38820F931FA11DB11D6A
:100A60008093BB389093BC38A093BD38B093BE3808
:100A70001092E738FF91EF91BF91AF919F918F91C5
:100A80007F916F915F914F913F912F910F900BBE8E
:100A90000F900FBE0F901F9018959FB7F894E1E745
:100AA000F0E08081807D808388B38F6288BB109264
:100AB0009000E1E9F0E0108210929200109295000F
:100AC000109294008081856080839FBF08959C016F
:100AD0009FB7F894309399002093980088B38F6261
:100AE00088BBE1E7F0E08081826080839FBF08954A
:100AF000FB0141505109460F571FE417F50778F4E1
:100B0000208130E0322F22276181260F311D820F94
:100B1000931F8217930708F401963296EECFE417DD
:100B2000F50751F4208130E0322F2227820F931FE6
:100B30008217930708F401960895CF93DF93C0912D
:100B40004E39D0E0DC2FCC2720914F3930E02451B2
:100B50003109C20FD31F48E050E068E579E39E01F8
:100B6000280F311DC9010E947885AE0160E679E346
:100B70000E947885009721F098278927982702C03E
:100B80008FEF9FEFDF91CF910895FC012381260F16
:100B900020934B39A72FBB2792819A0F90934A3904
:100BA000318130934939408140934839E92FF0E051
:100BB000EA17FB0748F481E0830F809349398111DC
:100BC00003C04F5F4093483930E077272617370737
:100BD00088F49F5F90934A3991110CC080914939F4
:100BE0008F5F80934939811105C0809148398F5FAB
:100BF0008093483908952091413A3091423ABC019E
:100C0000C90108960E94C585E091413AF091423AA7
:100C1000A8E4B9E38C91808711968C911197818714
:100C200012968C911297828713968C9183870895E0
:100C300044E150E06CE479E380E090E00E94788544
:100C4000009721F098278927982708958FEF9FEF25
:100C5000089586E00C949D8581E10C949D8580E04B
:100C6000E82FF0E0EE0FFF1FED53F54C11821082DC
:100C70008F5F8430A9F780E090E2899FF001112412
:100C8000ED5BF54C118E8F5F8430B1F780E094E01E
:100C90009093C31D8093C21D80E09DE0989FF0015A
:100CA0001124E752F54C158214828F5F8A30B1F718
:100CB0008093C11D08959C0190E09430A1F0E92F2C
:100CC000F0E081E0890FEE0FFF1FED53F54C4081FE
:100CD00051814217530729F49093C11D118210824C
:100CE0000895982FEACF9093C11D0895AF92BF92B7
:100CF000CF92DF92EF92FF920F931F93CF93DF93E8
:100D0000843009F4DFC1C091413AD091423A24E7DE
:100D100039E33093403A20933F3A30934739209358
:100D20004639833059F4898D8F70833009F06AC059
:100D300088899989892B09F0BFC67EC0823009F065
:100D40007FC08091C71D8F5F8093C71D811113C025
:100D50008091C61D8F5F8093C61D81110CC080914C
:100D6000C51D8F5F8093C51D811105C08091C41D75
:100D70008F5F8093C41D10924539109244391092B0
:100D8000D83A1092D73A898D982F9D7F953041F4AB
:100D90008A8D8F5F8A8F843109F08EC6198E8CC63A
:100DA000882309F489C628893989232B09F440C08E
:100DB0009A8D2FEF290F2A8F91117EC69B8D983027
:100DC00031F02FEF280F223048F4953039F4198E86
:100DD00080E880933C3A0E94AF8228C5953038F471
:100DE00023E0092E01C0220F0A94EAF701C020E394
:100DF0002A8F9F5F9B8F8F708330A1F048F48130E2
:100E000009F43AC3823009F057C610926D3937C3DE
:100E1000863009F4A8C4883009F4A5C4843009F0E8
:100E20004BC6A1C484E080933C3A0E94AF8230C597
:100E30008F70833009F040C688E080933C3AEBC461
:100E4000853019F5E0913D3AF0913E3A84819581E3
:100E5000892B09F431C61092423A1092413A88E641
:100E600099E39093403A80933F3A90934739809327
:100E700046391092D83A1092D73A109245391092CA
:100E8000443988E080933C3A1BC180914C398534C9
:100E900009F012C600914E3910E0102F0027809102
:100EA0004F39080F111D80914439909145398017B1
:100EB000910708F401C61093453900934439809195
:100EC00052398F7309F0F8C5F0905339F110F4C519
:100ED0008091D33A9091D43AC091580BD091590B4C
:100EE0008C179D0759F44091D53A5091D63A2091EC
:100EF0005A0B30915B0B42175307A1F020915C39DC
:100F000030915D398217930709F0D6C520915E397B
:100F100030915F398091D53A9091D63A28173907A8
:100F200009F0CAC50E941886019609F0C5C58091CE
:100F30005539863009F429C18131E9F1813009F050
:100F4000BBC580916039883009F0B6C51092603910
:100F50008091623990916339873F6FEF960710F067
:100F6000099601C008969093633980936239809105
:100F7000583990915939A0915A39B0915B39809381
:100F80005C3990935D39A0935E39B0935F3980915D
:100F9000D33A9091D43AA091D53AB091D63A809371
:100FA000583990935939A0935A39B0935B3980E4FA
:100FB000809354395EC50C51110910934539009343
:100FC000443988E699E39093403A80933F3A809180
:100FD000663990916739892B29F00E942C860196F9
:100FE00009F06AC5209162393091633921153105C4
:100FF00009F462C589ED9AE390933E3A80933D3AB5
:10100000A0906039B0906139E0905A0BF0905B0B82
:1010100040915C0B50915D0BA0915839B0915939BA
:1010200000915A3910915B3960915E0B70915F0BA2
:10103000E0913D3AF0913E3A8BE3EB35F80708F04A
:101040003BC584819581009721F12817390709F55F
:1010500086819781009719F08A159B05D1F48081CC
:101060009181C817D90729F4C280D380CE14DF0438
:10107000B1F08417950729F4C280D380C616D7062D
:1010800071F08A179B0729F4828193810817190749
:1010900031F03D96F0933E3AE0933D3AC9CF10923D
:1010A000423A1092413A82E080933C3A88E699E3D2
:1010B00090934739809346391092D83A1092D73A94
:1010C0000E94AF828091D73A9091D83A009709F464
:1010D000F3C49C01245E3F4F30934539209344393B
:1010E00030934E3920934F39E0913D3AF0913E3A9A
:1010F00020852093543921E120935539089698276B
:1011000089279827909365398093643910926739BD
:10111000109266398481958190936139809360390A
:101120008681978190936339809362398091D33A15
:101130009091D43AA091D53AB091D63A809358394B
:1011400090935939A0935A39B0935B39808191813A
:10115000A281B38180935C3990935D39A0935E390D
:10116000B0935F3984E799E39093403A80933F3A94
:101170000E942C8680959095009711F48FEF9FEF39
:10118000909367398093663974C40E9429860196CA
:1011900009F092C44091623950916339411551056B
:1011A00009F48AC48091603990916139009709F4FB
:1011B00083C46091583970915939E0915A39F0914E
:1011C0005B39C3E4DAE3298D2223A9F0AC81BD8128
:1011D0004A175B0781F4AE81BF818A179B0759F4D8
:1011E000A881B9816A177B0731F4AA81BB81EA170C
:1011F000FB0709F45CC1A0962AE3C33CD20719F7A8
:1012000080916D398F738230D9F45093C01D409313
:10121000BF1D80E0843091F0E82FF0E0EE0FFF1F5B
:10122000ED53F54C208131818F5F4217530791F7C1
:101230001092C11D80E0C0E0D0E07CC08093C11D51
:1012400080916D3982FD38C484E180936D3988E2E4
:1012500090E0909345398093443980E580936C39D0
:101260003091673980916B39809367392091663965
:1012700080916A398093663920936A3990916539F3
:101280008091693980936539909369398091643987
:101290008093C11D409168394093643980936839C7
:1012A0003F5F30936B3931110DC02F5F20936A3946
:1012B000211108C09F5F90936939911103C08F5F1E
:1012C0008093683980916039909161399093C01D05
:1012D0008093BF1D20916239309163393093613919
:1012E00020936039909363398093623980915839A3
:1012F00090915939A0915A39B0915B3980935C39FA
:1013000090935D39A0935E39B0935F398091D33A61
:101310009091D43AA091D53AB091D63A8093583969
:1013200090935939A0935A39B0935B3987C397305A
:1013300089F08F5F8430C1F060E2869F90011124B4
:10134000F901ED5BF54C918D9111F1CF8093C11DA9
:10135000EF010FC0209721F0428D9A8D941748F726
:10136000E901CD5BD54CE5CF8093C11D209709F4F1
:10137000A3C3D093423AC093413A83E08A8F888FC7
:101380001E8A84E08F8B1B8E809162399091633925
:101390009D838C8380916039909161399F838E8386
:1013A0008091583990915939A0915A39B0915B394F
:1013B00088839983AA83BB8381E0898F8091C41D30
:1013C0008C878091C51D8D878091C61D8E878091E9
:1013D000C71D8F8781E090E0998B888B809167395A
:1013E0008B87809166398A8780916539898780915A
:1013F0006439888781E090E00E94FB8580916C3998
:10140000982F907F9135C0F182958F7090E005976D
:10141000880F991F880F991FEF2DF0E0E817F90743
:101420004CF5E45BF64C20A5222321F1213011F488
:10143000F394F2CF2230C9F421A52430B1F4F09214
:10144000C11D82A590E0982F882723A5822B909319
:10145000C01D8093BF1D893C910510F088EC90E081
:101460009B8B8A8B9D8B8C8B07C021A5222311F02F
:10147000F20ED2CFF092C11D80E180936D39809140
:101480006D39826080936D3982E08093743984E095
:10149000809375391092763988EC809377398CE295
:1014A00090E0909345398093443980E675C2D0939B
:1014B000423AC093413A10923C3A80916D39782F6C
:1014C0007470F72E82FF03C0198E80E20EC29091D5
:1014D0006C3992959F70990F990F9093C11D091BBC
:1014E0001109045111091093453900934439922F81
:1014F0009F70923029F4982F9F73923139F41FC056
:10150000913021F4982F9F739230C9F0012B19F478
:10151000982F9370A1F0209164399885291332C2D5
:1015200020916539998529132DC2209166399A85B4
:10153000291328C2209167399B85291323C284FF70
:1015400049C0688979896115710509F443C0CE01E4
:101550000C960E94C58530916839809148393813BE
:1015600039C02091693980914939281333C090914D
:101570006A3980914A3998132DC080916B39409116
:101580004B39841327C03C872D879E878F878B8D8F
:10159000811119C09E89888D2A8D821B292F26953D
:1015A00026952695821B980F9E8B87FD81952F8906
:1015B000322F36953695231B820F8F8B96959695F5
:1015C0009695890F888F81E080933C3A888D8A8F29
:1015D000198A188A298DE22FEF708E2F90E0FC0176
:1015E0003197E830F10508F067C28827E656FF4FCB
:1015F0008F4F0C94619280913C3A80FF14C083E03D
:10160000898F80E480933C3A198A188A8091443902
:1016100090914539009709F4FAC022E420933C3AAE
:101620000E94FB85F4C080916D398F73823009F080
:1016300043C222CF80913C3A80FF60C080916D39D7
:101640008F73823109F05AC080916C39982F907F46
:101650009135C0F182958F7090E00597880F991FA2
:10166000880F991FEF2DF0E0E817F9074CF5E45BC0
:10167000F64C20A5222321F1213011F4F394F2CF6E
:101680002230C9F421A52430B1F4F092C11D82A505
:1016900090E0982F882723A5822B9093C01D8093DC
:1016A000BF1D893C910510F088EC90E09B8B8A8BE4
:1016B0009D8B8C8B07C021A5222311F0F20ED2CF77
:1016C000F092C11D83E0898F809164398887809171
:1016D00065398987809166398A87809167398B87D8
:1016E00081E090E00E94FB8582E480933C3A198A75
:1016F000188A109245391092443989C080E280934B
:101700003C3A0E94AF82E091413AF091423A118E08
:1017100097CD80916D3980FF28C024FD26C088892F
:101720009989892B09F0C8C1809144399091453934
:1017300001960E94FB8580913C3A982F906190938E
:101740003C3A2091443930914539232B19F082617C
:1017500080933C3A0E94AF8281E090E0998B888B25
:1017600088E0898F1B8E81E10EC185FF1CC08091AE
:1017700072399091733998278927982740913F3A79
:101780005091403A480F591F5093403A40933F3A86
:101790004091443950914539BA01681B790B7093D7
:1017A0004539609344394091443950914539411548
:1017B000510551F024FD08C090913C3A92609093FD
:1017C0003C3ACA010E94FB8580916E3990E0982FC7
:1017D000882720916F39820F911D9093C01D8093AF
:1017E000BF1D2C893D892817390710F0892B21F45A
:1017F0003093C01D2093BF1D8091BF1D9091C01DCF
:101800009B8B8A8B80913C3A837009F455C110926E
:10181000D83A1092D73A0E94AF8280913C3A85FF25
:1018200007C01092D83A1092D73A198E84E1ABC013
:1018300084FF0AC01092D83A1092D73A81E090E023
:10184000998B888B84E08DCF2091D73A3091D83A0C
:1018500021153105E1F080FF02C0198A188A8889B4
:101860009989009781F48A899B898217930720F4CC
:101870009093D83A8093D73A8091D73A9091D83ABA
:10188000998B888B04C09093D83A8093D73A1B8E5B
:1018900080914639909147399093403A80933F3AEE
:1018A0008091D73A9091D83A892B59F088899989B3
:1018B000009739F08896909345398093443988E1B0
:1018C0000BC080913C3A81FFF7C088E290E0909392
:1018D00045398093443980E180936D395CC08091B3
:1018E0003C3A80FFE9C0198E80E180933C3A0E9427
:1018F000AF82E2C08091443990914539009711F050
:101900000E94FB8590916D3980913C3A90FF0BC00D
:1019100080FF06C087E0898F1A8E198A188A19C03D
:1019200086E0898F16C080FF1EC085E0898F198AE6
:10193000188AC2C08091443990914539009711F0BE
:101940000E94FB8580916D3980FF0DC087E0898FF3
:101950001A8E81E090E00E94FB8580E180933C3A02
:101960000E94AF820FC08091443990914539892BF4
:1019700049F4A2C080913C3A80FF9EC087E0898FE5
:101980001A8E9AC080E180936D3988E290E090933E
:1019900045398093443980E580936C3988858093FC
:1019A00068398985809369398A8580936A398B85FE
:1019B00080936B398C85809364398D8580936539EC
:1019C0008E85809366398F858093673986E0809312
:1019D00055398C819D8190936139809360398E81D6
:1019E0009F8190936339809362398091D33A90912B
:1019F000D43AA091D53AB091D63A80935839909381
:101A00005939A0935A39B0935B3988819981AA8159
:101A1000BB8180935C3990935D39A0935E39B0931C
:101A20005F39898D84FF05C010926F3910926E392D
:101A300005C010926E3988EC80936F3980E48093F2
:101A40005439809144399091453990934E3980931F
:101A50004F39109273391092723910927139109275
:101A600070390E9429868095909590937139809362
:101A7000703985E480934C3910924D391092533966
:101A8000109252398091C81D9091C91D0196909372
:101A9000C91D8093C81D909350398093513910927D
:101AA0005739109256390E941886809590959093D8
:101AB00057398093563904C01092453910924439F1
:101AC00010923C3ADF91CF911F910F91FF90EF90D0
:101AD000DF90CF90BF90AF900895FC0180E090E040
:101AE0002081222329F02181820F911D3296F8CF87
:101AF0000895EF92FF920F931F93CF93DF937A0194
:101B00002830310514F5DB014D915C9154274527B0
:101B1000542702C0440F551FEA94E2F7452F55277A
:101B2000F901EA59F44FC081D0E04C235D2368E00D
:101B300070E0EB01C21BD30BFA0102C0F695E795EA
:101B4000CA95E2F7DC01EC9376C0D90153E0B59574
:101B5000A7955A95E1F7E114F10431F0AB01FC01CE
:101B60008C010A0F1B1F2FC0FB01AC017B01EA0E89
:101B7000FB1EEE16FF0629F06191EA016993AE01A2
:101B8000F8CF8901077011270115110509F453C019
:101B9000FC01EA0FFB1FD7012C9130E0D801AA59B4
:101BA000B44F9C91492F50E042235323C8E0D0E02A
:101BB0009E01201B310BEA0102C0D695C7952A95DC
:101BC000E2F7C08338C0E017F10781F0EA018881AD
:101BD00099819827892798270E2C02C0880F991F72
:101BE0000A94E2F791934F5F5F4FEDCF2770332751
:101BF0002115310501F1A60FB71F8D919C919827F2
:101C00008927982702C0880F991FEA94E2F7892F45
